:100000000C9461470C9482470C942AD20C9482473A
:100010000C9482470C9482470C9482470C9482473C
:100020000C9482470C9482470C9482470C9455D4CC
:100030000C9482470C9482470C94B8B40C94824779
:100040000C9482470C9482470C9482470C9482470C
:100050000C9482470C9482470C9482470C948247FC
:100060000C9482470C9444D20C94D3D10C948247C4
:100070000C94AACB0C944CCB0C9488CB0C94824758
:100080000C94F5D20C9482470C9482470C948247CE
:100090000C9482470C9482470C9482470C948247BC
:1000A0000C9482470C9482470C9482470C9493BB27
:1000B0000C9437BC0C9482470C9482470C94A9B6DC
:1000C0000C9482470C9482470C9482470C9482478C
:1000D0000C9482470C9482470C9482470C9482477C
:1000E0000C942EA60C9482470C9482470C94824761
:1000F0000C9482470C9482470C9482470C9482475C
:100100000C946ABB0C940EBC0C9441BB0C94E5BBE4
:100110000C9482470C9482470C9482470C9482473B
:100120000C9482470C9482470C9482470C9482472B
:100130000C9482470C940DB60C9482470C94824721
:100140000C9482470C9482470C9482470C9482470B
:100150000C9482470C9482470C9424A60C948247FA
:100160000C9482470C9482470C9482470C948247EB
:100170000C9482470C9482470C9482470C948247DB
:100180000C9482470C9482470C9482470C948247CB
:100190000C9482470C9482470C9482470C948247BB
:1001A0000C94BCBB0C9460BC0C9482470C948247AA
:1001B0000C945BB60C9482470C9482470C94824753
:1001C0000C9482470C9482470C9482470C9482478B
:1001D0000C9482470C9482470C9482470C9482477B
:1001E0000C9482470C94824761716B7175717F71B9
:1001F0008A719077907790779077907790719077D9
:100200009077907790779077907792719C71A671A4
:10021000B071BA7190779077907790779077907768
:10022000C47190771A7290779077907790779077E3
:1002300090779077597290777575907790779077DF
:100240009077907790779077907775759077907793
:10025000907786728B7295729F72A172AB72B67232
:100260009077C17290779077FE72907790779077C1
:100270009077907790779077907790779077907746
:1002800090779077907790770873907790779077C2
:1002900090779077907790779077907712734F73ED
:1002A0008C73D573DF73F873F87302740C7416745F
:1002B00020742A742F74397443748E778E778E77F6
:1002C0008E778E778E778E778E778E778E778E7706
:1002D0008E778E778E778E778E778E778E778E77F6
:1002E0008E7702748E778E778E778E778E778E7775
:1002F0008E778E778E778E778E778E778E778E77D6
:100300008E778E778E774D74577461746B748E7799
:100310008E778E778E778E778E778E778E77F8734F
:100320001B77DA76DE76E676C276C676CE76D2763B
:10033000F27607770F77137717777377EA76E67495
:10034000F77408759077907780745271907719756B
:100350002A753B757575E9735D7590779174907723
:100360004C75A2747574907790779077B374C47459
:10037000D574DABAE2BAEABAF2BAFABA02BB0ABB7E
:1003800012BBFDBD62BD6ABD72BD7ABD82BD8ABDB4
:1003900092BD9ABDA2BDAABDB2BDBABDC2BDCABD05
:1003A000E2BDE2BDE2BDE2BDE2BDE2BDE2BDE2BD55
:1003B000E2BDE2BDE2BDE2BDE2BDE2BDE2BDE2BD45
:1003C000E2BDE2BDE2BDE2BDE2BDE2BDE2BDE2BD35
:1003D000E2BDE2BDE2BDE2BDE2BDE2BDE2BDE2BD25
:1003E000E2BDE2BDE2BDD2BDDABD084AD73B3BCE9D
:1003F000016E84BCBFFDC12F3D6C74319ABD568324
:100400003DDA3D00C77F11BED9E4BB4C3E916BAADB
:10041000AABE000000803F05A84CCDB2D44EB9382A
:1004200036A9020C50B9918688083CA6AAAA2ABE11
:10043000000000803F07634236B79BD8A71A39688F
:100440005618AEBAAB558C1D3CB7CC5763BD6DED9D
:10045000FD753EF6177231BF000000803F080000B6
:1004600000BE922449123EABAAAA2ABECDCCCC4CE7
:100470003E00000080BEABAAAAAA3E00000000BF5A
:10048000000000803F0000000000084178D3BB431B
:1004900087D1133D190E3CC3BD4282AD2B3E68ECA3
:1004A0008276BED98FE1A93E4C80EFFFBE01C4FF2A
:1004B0007F3F0000000000000C94E4AD0C94E35674
:1004C0000C9407770C94DABD0C9492710C94F55649
:1004D0000C94AF630C94BCC10C94E6C70C94757477
:1004E0000C9483A70C94FAC90C9453CE0C9412BBB1
:1004F0000C94A35A0C948DBA0C94E2BD0C94DE7645
:100500000C949D5B0C947B5A0C94FB560C9448CF36
:100510000C947F5A0C946B710C94B1BA0C94BA7110
:100520000C94CABD0C94695B0C9442680C94F85D01
:100530000C9412730C94F2BA0C9439740C9498477E
:100540000C94AABD0C948E470C940C570C94B1C219
:100550000C949F590C94175F0C94AF5A0C949357BA
:100560000C9432BD0C9484470C9417770C944C5D1A
:100570000C948FA70C9475710C947F710C94FDBD35
:100580000C94B0710C944D740C94E0AD0C94027406
:100590000C94705D0C940F770C94F2760C947B6342
:1005A0000C94C7590C94AB720C94935A0C94DA6364
:1005B0000C949F5A0C94895B0C940C740C948E7759
:1005C0000C94E9560C94D2BD0C942B570C94A4AD0A
:1005D0000C94EDCC0C94207A0C94A5BA0C94886EF3
:1005E0000C948A920C94855B0C94DE5A0C940ABB92
:1005F0000C944C570C94F54A0C9488CA0C94E973EB
:100600000C949B5A0C942C580C94B9590C947377F5
:100610000C94D6560C94AB5A0C94815B0C94A8584D
:100620000C949ABD0C94C0AD0C94B3740C941757F1
:100630000C94B75E0C94F8730C942D540C94EF56F4
:100640000C94DA760C941E6D0C94B35A0C94BFCEB5
:100650000C948B720C9428630C94755B0C949174BD
:100660000C94ADBA0C944A640C9491BA0C94426BFD
:100670000C9440790C9465570C94FD5A0C94558455
:100680000C9436570C9490770C94BF5A0C94EA76DD
:100690000C94B17F0C94D7470C94DCAD0C94735A36
:1006A0000C94C8780C94EABA0C9408730C94025811
:1006B0000C947BA70C9480740C948FAD0C94617196
:1006C0000C94FABA0C943CAF0C942F740C94F5670C
:1006D0000C949F720C94B2BD0C944BAC0C94E8AD8E
:1006E0000C94D5740C9416740C9447AC0C94CA6E8C
:1006F0000C9420630C9495580C9496BA0C9493A780
:100700000C946F680C942CBD0C94DF730C9445AC66
:100710000C94F4590C944A6B0C942C630C948A71CD
:100720000C94875A0C947ABD0C94A6710C9484682E
:100730000C944CB90C9477A70C94CE590C94016E80
:100740000C94A2740C94BABD0C9432BA0C948BA77E
:100750000C948D5B0C94CA790C9424630C94655BA7
:100760000C94D5590C94D2760C94A2BD0C94E84705
:100770000C94DEB90C94285D0C946B740C94E676A2
:100780000C94CE5C0C942A740C9448790C94577495
:100790000C9472BD0C94D05D0C9420800C94F77472
:1007A0000C94A55B0C948E5E0C946E590C94C474DE
:1007B0000C94E2770C948B790C944C750C94DE5E5F
:1007C0000C9413770C94CE760C94A15B0C94C172AC
:1007D0000C94D25D0C948F5A0C94AF670C94A1C703
:1007E0000C94A4600C944F730C94D4C10C9413AF6C
:1007F0000C948C730C9495720C94FB810C9420795E
:100800000C94BBC10C94F5680C94135A0C94975D2E
:100810000C9428D00C945D750C94675E0C941B7737
:100820000C9440B90C9486720C94C4CF0C94CAB941
:100830000C94C6760C941D5E0C94CB570C946F5A96
:100840000C94245D0C9481620C945ABA0C94775ADF
:100850000C940BAC0C94B15B0C94835A0C940DACBF
:100860000C94BC5B0C9482BD0C949C710C946163E1
:100870000C94975A0C940DC20C9465620C94F8B9C0
:100880000C94DABA0C9489BA0C94CF620C94D57398
:100890000C94425E0C946ABD0C94B75A0C94205789
:1008A0000C9441570C94E2BA0C944CBD0C94A17278
:1008B0000C94915B0C9416590C9430630C9467CA99
:1008C0000C94E6740C941B790C941A720C944C7969
:1008D0000C9459720C9443740C9401570C942C672B
:1008E0000C94F9CA0C94F5790C9411CF0C94A75A76
:1008F0000C9402BB0C9473A70C9462BD0C94757598
:100900000C94A9BA0C9473D10C9424800C9492BDCD
:100910000C94C4710C941C6E0C9487A70C94C2BDEB
:100920000C9450790C94E7CA0C9412640C94BFCDCB
:100930000C94F0C10C946E4E0C94FE720C94995B66
:100940000C942A750C94715B0C94205B0C948B5A5C
:100950000C949A590C94BB5A0C948ABD0C94795BF4
:100960000C94955B0C94015B0C9495630C947C57F0
:100970000C94C2760C947FA70C9450BD0C94246800
:100980000C947D5B0C946D5B0C9428800C944479E2
:100990000C940FAC0C9465580C9419750C94B672A9
:1009A0000C94D2770C9408750C94C0590C949071E7
:1009B0000C9420740C9461740C9434B90C9497A723
:1009C0000C943B750C9452710C947CA85B25732598
:1009D000735D20257320257320706F736974696FB0
:1009E0006E2531382E336625730A005B2573257317
:1009F0005D202573202573206F666673657425322C
:100A0000302E336625730A005B257325735D202520
:100A100073207A65726F206261636B6F6666253141
:100A2000392E336625730A005B257325735D2025F7
:100A300073206C61746368206261636B6F66662506
:100A400031382E336625730A005B257325735D20CC
:100A50002573206C617463682076656C6F636974BC
:100A6000792531332E306625732F6D696E0A005B50
:100A7000257325735D20257320736561726368207B
:100A800076656C6F636974792531322E3066257313
:100A90002F6D696E0A005B257325735D2025732019
:100AA000737769746368206D617825313764205BE2
:100AB000303D6F66662C313D686F6D696E672C3214
:100AC0003D6C696D69742C333D6C696D69742B687C
:100AD0006F6D696E675D0A005B257325735D202568
:100AE0007320737769746368206D696E253137648C
:100AF000205B303D6F66662C313D686F6D696E67B7
:100B00002C323D6C696D69742C333D6C696D697470
:100B10002B686F6D696E675D0A005B257325735DD9
:100B2000202573207261646975732076616C756528
:100B30002532302E346625730A005B257325735DDC
:100B4000202573206A756E6374696F6E2064657604
:100B5000696174696F6E2531342E346625732028DF
:100B60006C61726765722069732066617374657267
:100B7000290A005B257325735D202573206A657241
:100B80006B20686F6D696E672531362E3066257370
:100B90002F6D696E5E33202A2031206D696C6C697F
:100BA0006F6E0A005B257325735D202573206A65CF
:100BB000726B206D6178696D756D2531352E3066EB
:100BC00025732F6D696E5E33202A2031206D696C8C
:100BD0006C696F6E0A005B257325735D2025732099
:100BE00074726176656C206D696E696D756D253105
:100BF000372E336625730A005B257325735D202528
:100C0000732074726176656C206D6178696D756DA5
:100C10002531372E336625730A005B257325735DF6
:100C20002025732076656C6F63697479206D617817
:100C3000696D756D2531312E306625732F6D696EA6
:100C40000A005B257325735D202573206665656446
:100C500072617465206D6178696D756D2531312E15
:100C6000306625732F6D696E0A005B257325735DF1
:100C70002025732061786973206D6F646525313894
:100C8000642025730A005B6D615D20206D696E2014
:100C9000617263207365676D656E742531382E331C
:100CA0006625730A005B736C5D2020736F66742089
:100CB0006C696D697420656E61626C6525313264A2
:100CC0000A005B63745D202063686F7264616C204E
:100CD000746F6C6572616E63652531372E346625DD
:100CE000730A005B6A615D20206A756E6374696FC8
:100CF0006E20616363656C65726174696F6E25381F
:100D00002E306625730A005B6764695D2064656642
:100D100061756C742067636F6465206469737461C6
:100D20006E6365206D6F6465253264205B303D47DE
:100D300039302C313D4739315D0A005B6770615DA8
:100D40002064656661756C742067636F64652070EC
:100D500061746820636F6E74726F6C253364205BFE
:100D6000303D4736312C313D4736312E312C323D26
:100D70004736345D0A005B67636F5D2064656661BA
:100D8000756C742067636F646520636F6F72642095
:100D900073797374656D253364205B312D3620289B
:100DA0004735342D473539295D0A005B67756E5D1F
:100DB0002064656661756C742067636F6465207577
:100DC0006E697473206D6F6465253564205B303DFA
:100DD0004732302C313D4732315D0A005B67706C21
:100DE0005D2064656661756C742067636F6465205F
:100DF000706C616E6525313064205B303D47313762
:100E00002C313D4731382C323D4731395D0A0025C0
:100E10006320776F726B206F66667365743A253155
:100E2000322E336625730A002563206D616368697D
:100E30006E6520706F736E3A2531312E33662573DF
:100E40000A00256320706F736974696F6E3A2531EB
:100E5000352E336625730A00546F6F6C206E756DE6
:100E60006265722020202020202020202025640A76
:100E700000466565642072617465206D6F64653A33
:100E800020202020202025730A0044697374616E9D
:100E90006365206D6F64653A202020202020202586
:100EA000730A0050617468204D6F64653A202020F9
:100EB000202020202020202025730A00506C616E05
:100EC000653A2020202020202020202020202020C3
:100ED0002025730A004D6F74696F6E206D6F646515
:100EE0003A20202020202020202025730A00436F54
:100EF0006F7264696E6174652073797374656D3A9D
:100F000020202025730A00556E6974733A20202032
:100F100020202020202020202020202025730A00AF
:100F2000486F6D696E672073746174653A20202084
:100F3000202020202025730A0046656564686F6CB8
:100F4000642073746174653A20202020202025736A
:100F50000A004D6F74696F6E2073746174653A2076
:100F60002020202020202025730A004379636C650F
:100F70002073746174653A202020202020202020D6
:100F800025730A00526177206D616368696E652080
:100F900073746174653A20202025730A004D6163E3
:100FA00068696E652073746174653A202020202082
:100FB000202025730A004C696E65206E756D626590
:100FC000723A2531302E30660A004665656420721B
:100FD0006174653A2531362E336625732F6D696E3F
:100FE0000A0056656C6F636974793A2531372E3380
:100FF0006625732F6D696E0A0050101F10FF0F4792
:101000003935202D20756E6974732D7065722D72BF
:1010100065766F6C7574696F6E206D6F64650047DF
:101020003934202D20756E6974732D7065722D6DA5
:10103000696E757465206D6F64652028692E652E54
:10104000206665656472617465206D6F6465290052
:10105000473933202D20696E766572736520746977
:101060006D65206D6F6465008C106C104739312000
:101070002D20696E6372656D656E74616C206469A4
:101080007374616E6365206D6F646500473930204D
:101090002D206162736F6C7574652064697374616F
:1010A0006E6365206D6F646500DD10C510AF10477D
:1010B0003634202D20636F6E74696E756F757320E2
:1010C0006D6F6465004736312E31202D20657861C3
:1010D00063742073746F70206D6F646500473631E0
:1010E000202D2065786163742070617468206D6FB5
:1010F00064650017110811F910473139202D205966
:101100005A20706C616E6500473138202D20585A86
:1011100020706C616E6500473137202D20585920B2
:10112000706C616E6500A311911178115711301127
:10113000473830202D2063616E63656C206D6F74BD
:10114000696F6E206D6F646520286E6F6E6520611B
:1011500063746976652900473320202D20636F75FD
:101160006E74657220636C6F636B77697365206161
:101170007263206665656400473220202D20636C11
:101180006F636B7769736520617263206665656460
:1011900000473120202D206C696E656172206665E4
:1011A000656400473020202D206C696E65617220D7
:1011B000747261766572736520287365656B2900AA
:1011C0006A12501236121C120212E811CE11473563
:1011D00039202D20636F6F7264696E6174652073AE
:1011E000797374656D203600473538202D20636F84
:1011F0006F7264696E6174652073797374656D20B4
:101200003500473537202D20636F6F7264696E613A
:1012100074652073797374656D203400473536200A
:101220002D20636F6F7264696E61746520737973CA
:1012300074656D203300473535202D20636F6F7244
:1012400064696E6174652073797374656D20320012
:10125000473534202D20636F6F7264696E61746549
:101260002073797374656D203100473533202D204C
:101270006D616368696E6520636F6F7264696E612A
:1012800074652073797374656D009D1297129012C6
:10129000486F6D696E6700486F6D6564004E6F74CE
:1012A00020486F6D656400D112CC12C712C112BC08
:1012B00012B312456E6420486F6C6400486F6C6412
:1012C00000446563656C00506C616E0053796E6319
:1012D000004F666600E412E012DB12486F6C640097
:1012E00052756E0053746F70000E130413FE12F7E4
:1012F00012F3124A6F6700486F6D696E6700507293
:101300006F6265004D616368696E696E67004F6664
:10131000660044133E13381333132F13291320137D
:1013200053687574646F776E004379636C6500452C
:101330006E640053746F7000416C61726D00526591
:1013400061647900496E697469616C697A696E6774
:1013500000A713A1139B13961392138E1389138363
:10136000137D1376137213691353687574646F7762
:101370006E004A6F6700486F6D696E67004379635E
:101380006C650050726F626500486F6C6400527546
:101390006E00456E640053746F7000416C61726D35
:1013A00000526561647900496E697469616C697A9B
:1013B000696E6700CE13B813473231202D206D6956
:1013C0006C6C696D65746572206D6F646500473281
:1013D00030202D20696E63686573206D6F64650031
:1013E0000814FD13F113E8135B7261646975735D92
:1013F000005B696E686962697465645D005B737443
:10140000616E646172645D005B64697361626C65E6
:10141000645D0022141E1419142064656700206D99
:101420006D0020696E002A2A2A204E4F54494345F8
:10143000202A2A2A20526573657474696E672062B7
:10144000617564207261746520746F202573005B80
:10145000626175645D20555342206261756420723B
:1014600061746525313564205B313D393630302C6F
:10147000323D31393230302C333D33383430302C3A
:10148000343D35373630302C353D31313532303022
:101490002C363D3233303430305D0A005B72786D6B
:1014A0005D2073657269616C205258206D6F6465B0
:1014B00025313564205B303D636861725F6D6F6418
:1014C000652C313D6C696E655F6D6F64655D0A000A
:1014D0005B65785D2020656E61626C6520666C6F6F
:1014E0007720636F6E74726F6C25313064205B30CF
:1014F0003D6F66662C313D584F4E2F584F46462C57
:10150000323D5254532F4354535D0A005B65655D71
:101510002020656E61626C65206563686F253138D7
:1015200064205B303D6F66662C313D6F6E5D0A0056
:101530005B65635D2020657870616E64204C462099
:10154000746F2043524C46206F6E205458253664E9
:10155000205B303D6F66662C313D6F6E5D0A0092F8
:10156000158D15871581157B1574156D1532333062
:1015700034303000313135323030003537363030AC
:1015800000333834303000313932303000393630C1
:1015900030003000737973006662000000000702BB
:1015A0004079975DD05D6E3C6626DC4373797300AD
:1015B00066760000000007034479975DD05D723CB9
:1015C000EC51783F737973006870000000000700E9
:1015D0004879975DDE5E7A3C0000803F7379730046
:1015E00068760000000007004C79975D20797E3C0A
:1015F000000000417379730069640000000004007A
:101600005079C878D05D6A3C0000000000000000FE
:101610007469640000000100F0C14C5D8E5EA43C62
:1016200000000000000000006E000000000001004B
:101630006F5A65578E5EE93400000000000000001C
:101640006C696E65000001006F5A7C578E5EE9344C
:10165000000000000000000076656C000000000241
:10166000D5599357D05D6A3C00000000000000008F
:101670006665656400000002F459CB57D05D6A3C92
:10168000000000000000000073746174000000009E
:10169000735AD656D05D6A3C00000000000000007E
:1016A0006D61637300000000775AE356D05D6A3CB9
:1016B0000000000000000000637963730000000078
:1016C0007B5AE956D05D6A3C000000000000000033
:1016D0006D6F7473000000007F5AEF56D05D6A3C56
:1016E0000000000000000000686F6C640000000053
:1016F000835AF556D05D6A3C0000000000000000EF
:10170000756E6974000000008B5A0157D05D6A3C09
:101710000000000000000000636F6F720000000016
:101720008F5A0C57D05D6A3C00000000000000009A
:101730006D6F6D6F00000000935A1757D05D6A3CC3
:101740000000000000000000706C616E00000000EE
:10175000975A2057D05D6A3C00000000000000004E
:1017600070617468000000009B5A2B57D05D6A3C82
:1017700000000000000000006469737400000000B5
:101780009F5A3657D05D6A3C000000000000000000
:1017900066726D6F00000000A35A4157D05D6A3C2D
:1017A0000000000000000000746F6F6C000000007B
:1017B000A75A4C57D05D6A3C000000006D706F0066
:1017C0006D706F7800000003B15B2C58D05D6A3CEF
:1017D000000000006D706F006D706F7900000003F5
:1017E000B15B2C58D05D6A3C000000006D706F004A
:1017F0006D706F7A00000003B15B2C58D05D6A3CBD
:10180000000000006D706F006D706F6100000003DC
:10181000B15B2C58D05D6A3C000000006D706F0019
:101820006D706F6200000003B15B2C58D05D6A3CA4
:10183000000000006D706F006D706F6300000003AA
:10184000B15B2C58D05D6A3C00000000706F7300E3
:10185000706F737800000003A55B0258D05D6A3C8E
:1018600000000000706F7300706F73790000000358
:10187000A55B0258D05D6A3C00000000706F7300E9
:10188000706F737A00000003A55B0258D05D6A3C5C
:1018900000000000706F7300706F73610000000340
:1018A000A55B0258D05D6A3C00000000706F7300B9
:1018B000706F736200000003A55B0258D05D6A3C44
:1018C00000000000706F7300706F7363000000030E
:1018D000A55B0258D05D6A3C000000006F66730093
:1018E0006F66737800000003BC5B6558D05D6A3C8E
:1018F000000000006F6673006F66737900000003DC
:10190000BC5B6558D05D6A3C000000006F667300E8
:101910006F66737A00000003BC5B6558D05D6A3C5B
:10192000000000006F6673006F66736100000003C3
:10193000BC5B6558D05D6A3C000000006F667300B8
:101940006F66736200000003BC5B6558D05D6A3C43
:10195000000000006F6673006F6673630000000391
:10196000BC5B6558D05D6A3C00000000686F6D008C
:10197000686F6D6500000000875AFB569F596A3CEE
:1019800000000000686F6D00686F6D780000000057
:10199000A55B285DD05DBE3400000000686F6D005F
:1019A000686F6D7900000000A55B285DD05DBF34D5
:1019B00000000000686F6D00686F6D7A0000000025
:1019C000A55B285DD05DC03400000000686F6D002D
:1019D000686F6D6100000000A55B285DD05DC134BB
:1019E00000000000686F6D00686F6D62000000000D
:1019F000A55B285DD05DC23400000000686F6D00FB
:101A0000686F6D6300000000A55B285DD05DC33486
:101A100000000000707262007072626500000000D9
:101A2000BBC1285DD05DC43400000000707262004C
:101A30007072627800000003BBC1975DD05DC53451
:101A40000000000070726200707262790000000392
:101A5000BBC1975DD05DC9340000000070726200A8
:101A60007072627A00000003BBC1975DD05DCD3417
:101A7000000000007072620070726261000000037A
:101A8000BBC1975DD05DD134000000007072620070
:101A90007072626200000003BBC1975DD05DD534F7
:101AA0000000000070726200707262630000000348
:101AB000BBC1975DD05DD934000000006A6F67003C
:101AC0006A6F677800000000BBC1245DB959E33438
:101AD000000000006A6F67006A6F6779000000000D
:101AE000BBC1245DC059E334000000006A6F670089
:101AF0006A6F677A00000000BBC1245DC759E334F8
:101B0000000000006A6F67006A6F676100000000F4
:101B1000BBC1245DCE59E334000000007077720031
:101B20007077723100000000B1BADEB9D05D6A3C56
:101B300000000000707772007077723200000000C1
:101B4000B1BADEB9D05D6A3C000000007077720067
:101B50007077723300000000B1BADEB9D05D6A3C24
:101B6000000000007077720070777234000000008F
:101B7000B1BADEB9D05D6A3C00000000310000005F
:101B8000316D6100000003008DBA285DD25DF05A0E
:101B90000000404031000000317361000000030389
:101BA00091BA975D34B9FB5A6666E63F3100000092
:101BB0003174720000000B0496BA975D40B9FF5A69
:101BC0000000B44331000000316D690000000300E3
:101BD000A5BA285D4CB9F15A00000041310000005F
:101BE00031706F0000000300A9BA285DF85DF55A56
:101BF0000000803F3100000031706D0000000300E4
:101C0000ADBA285DCAB9F65A0000004032000000A3
:101C1000326D6100000003008DBA285DD25D0F5B5C
:101C20000000004032000000327361000000030336
:101C300091BA975D34B91A5B6666E63F32000000E0
:101C40003274720000000B0496BA975D40B91E5BB7
:101C50005C8F224132000000326D690000000300F9
:101C6000A5BA285D4CB9105B0000004132000000AD
:101C700032706F0000000300A9BA285DF85D145BA4
:101C80000000803F3200000032706D000000030051
:101C9000ADBA285DCAB9155B0000004033000000F2
:101CA000336D6100000003008DBA285DD25D2E5BAC
:101CB0000000803F33000000337361000000030325
:101CC00091BA975D34B9395B6666E63F3300000030
:101CD0003374720000000B0496BA975D40B93D5B07
:101CE0005C8F224133000000336D69000000030067
:101CF000A5BA285D4CB92F5B0000004133000000FD
:101D000033706F0000000300A9BA285DF85D335BF3
:101D10000000803F3300000033706D0000000300BE
:101D2000ADBA285DCAB9345B000000403400000041
:101D3000346D6100000003008DBA285DD25D4D5BFB
:101D40000000000034000000347361000000030351
:101D500091BA975D34B9585B6666E63F340000007F
:101D60003474720000000B0496BA975D40B95C5B56
:101D70005C8F224134000000346D690000000300D4
:101D8000A5BA285D4CB94E5B00000041340000004C
:101D900034706F0000000300A9BA285DF85D525B43
:101DA000000000003400000034706D0000000300EB
:101DB000ADBA285DCAB9535B00000040780000004E
:101DC00078616D0000000300205B9558A8587A33B5
:101DD0000000803F7800000078766D0000000B0066
:101DE000695B975DCF627F330080BB447800000061
:101DF0007866720000000B00655B975DCF627B33F5
:101E00000080BB447800000078746E0000000B0373
:101E1000715B975DCF62873300000000780000009F
:101E200078746D0000000B036D5B975DCF628333A8
:101E300000000A4378000000786A6D0000000B0083
:101E4000755B975D16598B330000FA4378000000EC
:101E5000786A680000000B00795B975D6E598F33DC
:101E600000007A4478000000786A640000000B04E7
:101E70007D5B975DCF6297330AD7233C78000000E3
:101E800078736E0000000300855B285D32BD9E32D2
:101E90000000803F780000007873780000000300A5
:101EA000895B285D32BD9F32000000007800000091
:101EB0007873760000000B008D5B975DCF629F33D7
:101EC0000000FA4378000000786C760000000B00F8
:101ED000915B975DCF62A3330000C841780000009A
:101EE000786C620000000B03955B975DCF62A733AF
:101EF0000000A04078000000787A620000000B0328
:101F0000995B975DCF62AB33000000007900000061
:101F100079616D0000000300205B9558A858AF332D
:101F20000000803F7900000079766D0000000B0012
:101F3000695B975DCF62B4330080BB4479000000D9
:101F40007966720000000B00655B975DCF62B0336D
:101F50000080BB447900000079746E0000000B0320
:101F6000715B975DCF62BC33000000007900000018
:101F700079746D0000000B036D5B975DCF62B83321
:101F80000000E64279000000796A6D0000000B0055
:101F9000755B975D1659C0330000FA437900000065
:101FA000796A680000000B00795B975D6E59C43355
:101FB00000007A4479000000796A640000000B0494
:101FC0007D5B975DCF62CC330AD7233C790000005C
:101FD00079736E0000000300855B285D32BDA0327E
:101FE0000000803F79000000797378000000030052
:101FF000895B285D32BDA13200000000790000003D
:102000007973760000000B008D5B975DCF62D4334F
:102010000000FA4379000000796C760000000B00A4
:10202000915B975DCF62D8330000C8417900000012
:10203000796C620000000B03955B975DCF62DC3327
:102040000000A04079000000797A620000000B03D4
:10205000995B975DCF62E033000040407A0000005A
:102060007A616D0000000300205B9558A858E433A6
:102070000000803F7A0000007A766D0000000B00BF
:10208000695B975DCF62E9330080BB447A00000052
:102090007A66720000000B00655B975DCF62E533E6
:1020A0000080BB447A0000007A746E0000000B03CD
:1020B000715B975DCF62F13300008CC27A00000043
:1020C0007A746D0000000B036D5B975DCF62ED339A
:1020D000000000007A0000007A6A6D0000000B002A
:1020E000755B975D1659F5330000FA437A000000DE
:1020F0007A6A680000000B00795B975D6E59F933CE
:1021000000007A447A0000007A6A640000000B0440
:102110007D5B975DCF6201340AD7233C7A000000D3
:102120007A736E0000000300855B285D32BDA23229
:10213000000000007A0000007A73780000000300BD
:10214000895B285D32BDA3320000803F7A00000029
:102150007A73760000000B008D5B975DCF620934C7
:102160000000FA437A0000007A6C760000000B0051
:10217000915B975DCF620D340000C8417A0000008A
:102180007A6C620000000B03955B975DCF6211349F
:102190000000A0407A0000007A7A620000000B0381
:1021A000995B975DCF62153400000000610000006C
:1021B00061616D0000000300205B9558A858193438
:1021C000000040406100000061766D0000000300E7
:1021D000695B975DDE5E1E340000B4446100000060
:1021E0006166720000000300655B975DDE5E1A3475
:1021F0000000B4446100000061746E00000003033D
:10220000715B975DCF622634000080BF61000000E3
:1022100061746D00000003036D5B975DDE5E223428
:10222000000080BF61000000616A6D0000000300D3
:10223000755B975D16592A340000FA43610000006F
:10224000616A680000000300795B975D6E592E3467
:102250000000FA4361000000616A640000000304AA
:102260007D5B975DDE5E36340AD7233C610000005B
:102270006172610000000B03815B975DDE5E3A34A2
:10228000CF2E65426100000061736E000000030004
:10229000855B285D32BDA4320000803F61000000F4
:1022A0006173780000000300895B285D32BDA532B0
:1022B0000000000061000000617376000000030070
:1022C0008D5B975DDE5E3E340000164461000000C9
:1022D000616C760000000300915B975DDE5E423426
:1022E0000000C84261000000616C6200000003034E
:1022F000955B975DDE5E46340000A0406100000003
:10230000617A620000000303995B975DDE5E4A34E8
:10231000000000406200000062616D0000000300E8
:10232000205B9558A8584E34000000006200000061
:1023300062766D0000000300695B975DDE5E5334DA
:102340000000B444620000006266720000000300F6
:10235000655B975DDE5E4F340000B44462000000B0
:1023600062746E0000000303715B975DCF625B34A3
:10237000000080BF6200000062746D000000030373
:102380006D5B975DDE5E5734000080BF6200000029
:10239000626A6D0000000300755B975D16595F343B
:1023A0000000FA4362000000626A6400000003005B
:1023B0007D5B975DDE5E6B340AD7233C62000000D4
:1023C0006272610000000B03815B975DDE5E6F341B
:1023D000CF2E65426300000063616D0000000300C2
:1023E000205B9558A858833400000000630000006B
:1023F00063766D0000000300695B975DDE5E8834E4
:102400000000B44463000000636672000000030033
:10241000655B975DDE5E84340000B44463000000B9
:1024200063746E0000000303715B975DCF629034AC
:10243000000080BF6300000063746D0000000303B0
:102440006D5B975DDE5E8C34000080BF6300000032
:10245000636A6D0000000300755B975D1659943444
:102460000000FA4363000000636A64000000030098
:102470007D5B975DDE5EA0340AD7233C63000000DD
:102480006372610000000B03815B975DDE5EA43424
:10249000CF2E65427031000070316672710003000A
:1024A00073A7975DDE5ECC590000C8427031000012
:1024B000703163736C00030077A7975DDE5ED059BF
:1024C00000E0F6457031000070316373680003006E
:1024D0007BA7975DDE5ED45900004846703100004E
:1024E000703163706C0003037FA7975DDE5ED8597F
:1024F000B81E053E70310000703163706800030340
:1025000083A7975DDE5EDC597B142E3E70310000A0
:10251000703177736C00030087A7975DDE5EE0592A
:102520000000000070310000703177736800030014
:102530008BA7975DDE5EE45900000000703100005B
:10254000703177706C0003038FA7975DDE5EE859EA
:10255000CDCCCC3D70310000703177706800030342
:1025600093A7975DDE5EEC59CDCCCC3D7031000079
:102570007031706F6600030397A7975DDE5EF059B8
:10258000CDCCCC3D673534006735347800000B0383
:102590009D5B975DCF62EA32000000006735340032
:1025A0006735347900000B039D5B975DCF62EE3297
:1025B00000000000673534006735347A00000B03F3
:1025C0009D5B975DCF62F2320000000067353400FA
:1025D0006735346100000B039D5B975DCF62F63277
:1025E00000000000673534006735346200000B03DB
:1025F0009D5B975DCF62FA320000000067353400C2
:102600006735346300000B039D5B975DCF62FE323C
:1026100000000000673535006735357800000B0392
:102620009D5B975DCF620233000000006735350087
:102630006735357900000B039D5B975DCF620633EC
:1026400000000000673535006735357A00000B0360
:102650009D5B975DCF620A3300000000673535004F
:102660006735356100000B039D5B975DCF620E33CC
:1026700000000000673535006735356200000B0348
:102680009D5B975DCF621233000000006735350017
:102690006735356300000B039D5B975DCF62163392
:1026A0000000A0C1673536006735367800000B039F
:1026B0009D5B975DCF621A330000000067353600DE
:1026C0006735367900000B039D5B975DCF621E3343
:1026D00000000000673536006735367A00000B03CE
:1026E0009D5B975DCF6222330000000067353600A6
:1026F0006735366100000B039D5B975DCF62263323
:1027000000000000673536006735366200000B03B5
:102710009D5B975DCF622A3300000000673536006D
:102720006735366300000B039D5B975DCF622E33E8
:1027300000000000673537006735377800000B036D
:102740009D5B975DCF623233000000006735370034
:102750006735377900000B039D5B975DCF62363399
:1027600000000000673537006735377A00000B033B
:102770009D5B975DCF623A330000000067353700FC
:102780006735376100000B039D5B975DCF623E3379
:1027900000000000673537006735376200000B0323
:1027A0009D5B975DCF6242330000000067353700C4
:1027B0006735376300000B039D5B975DCF6246333F
:1027C00000000000673538006735387800000B03DB
:1027D0009D5B975DCF624A3300000000673538008B
:1027E0006735387900000B039D5B975DCF624E33F0
:1027F00000000000673538006735387A00000B03A9
:102800009D5B975DCF625233000000006735380052
:102810006735386100000B039D5B975DCF625633CF
:1028200000000000673538006735386200000B0390
:102830009D5B975DCF625A3300000000673538001A
:102840006735386300000B039D5B975DCF625E3395
:1028500000000000673539006735397800000B0348
:102860009D5B975DCF6262330000000067353900E1
:102870006735397900000B039D5B975DCF62663346
:1028800000000000673539006735397A00000B0316
:102890009D5B975DCF626A330000000067353900A9
:1028A0006735396100000B039D5B975DCF626E3326
:1028B00000000000673539006735396200000B03FE
:1028C0009D5B975DCF627233000000006735390071
:1028D0006735396300000B039D5B975DCF627633EC
:1028E00000000000673932006739327800000103C8
:1028F0009D5B975DD05D5B3500000000673932005D
:1029000067393279000001039D5B975DD05D5F35CB
:1029100000000000673932006739327A0000010395
:102920009D5B975DD05D6335000000006739320024
:1029300067393261000001039D5B975DD05D6735AB
:10294000000000006739320067393262000001037D
:102950009D5B975DD05D6B350000000067393200EC
:1029600067393263000001039D5B975DD05D6F3571
:102970000000000067323800673238780000010339
:10298000A15B975DD05D73350000000067323800B1
:102990006732387900000103A15B975DD05D773520
:1029A00000000000673238006732387A0000010307
:1029B000A15B975DD05D7B35000000006732380079
:1029C0006732386100000103A15B975DD05D7F3500
:1029D00000000000673238006732386200000103EF
:1029E000A15B975DD05D8335000000006732380041
:1029F0006732386300000103A15B975DD05D8735C6
:102A000000000000673330006733307800000103B6
:102A1000A15B975DD05D8B3500000000673330000F
:102A20006733307900000103A15B975DD05D8F357E
:102A300000000000673330006733307A0000010384
:102A4000A15B975DD05D93350000000067333000D7
:102A50006733306100000103A15B975DD05D97355E
:102A6000000000006733300067333062000001036C
:102A7000A15B975DD05D9B3500000000673330009F
:102A80006733306300000103A15B975DD05D9F3524
:102A9000000000006A6964006A6964610000000067
:102AA000BBC1705DB75E943C000000006A696400C1
:102AB0006A69646200000000BBC1705DB75E983C4B
:102AC000000000006A6964006A6964630000000035
:102AD000BBC1705DB75E9C3C000000006A69640089
:102AE0006A69646400000000BBC1705DB75EA03C11
:102AF00000000000737973006A61000000000F009D
:102B0000BF5A975DCF62B8320050C34773797300E4
:102B10006374000000000F04DE5A975DCF62BC3280
:102B20000AD7233C73797300736C00000000070020
:102B3000FD5A285DD25DC032000000007379730039
:102B400073740000000007004CBD285D2CBD93325B
:102B50000000803F737973006D740000000007026D
:102B600089BA975DF8B9EC5A0000004000000000F7
:102B70006D65000000000000BCC15ABA5ABA6A3C38
:102B800000000000000000006D6400000000000074
:102B9000BCC132BA32BA6A3C0000000073797300DB
:102BA000656A0000000007002080285DF85D863C13
:102BB0000000803F737973006A7600000000070010
:102BC0002480285DB17F5E3F000040407379730030
:102BD0006A730000000007002880285DF85D603FF0
:102BE0000000803F737973007476000000000700D6
:102BF000B1C2285DF85D5F5C0000803F73797300AF
:102C00007176000000000700E8AD285D425E255A9D
:102C10000000000073797300737600000000070065
:102C20004BAC285D1D5E325A0000803F7379730003
:102C3000736900000000070047AC4C5D0FAC335ACD
:102C400000007A4373797300656300000000070099
:102C50002063285DDA63703200000000737973002E
:102C600065650000000007002463285D4A64713236
:102C70000000000073797300657800000000070011
:102C80002863285D1264723200000040737973007B
:102C900072786D00000007002C63285DF85D7332C8
:102CA0000000803F73797300626175640000040066
:102CB0003063285D81626E320000A0400000000099
:102CC000737200000000000045AC0BAC0DAC6A3C18
:102CD0000000000000000000717200000000000011
:102CE000DCAD8FADD05D6A3C00000000000000004C
:102CF0007169000000000000E0ADA4ADD05D6A3C49
:102D00000000000000000000716F000000000000E3
:102D1000E4ADC0ADD05D6A3C0000000000000000E2
:102D20006572000000000000BBC17CA8D05D6A3C59
:102D300000000000000000007166000000000000BC
:102D4000BBC1245D9A596A3C0000000000000000ED
:102D50007278000000000000F0C16562D05D6A3C3E
:102D600000000000000000006D736700000000001C
:102D7000BCC1245DD05D6A3C000000000000000082
:102D8000636C656172000000BBC16E4E6E4E6A3CA2
:102D90000000000000000000746573740000000073
:102DA000BBC1CA7950BD6A3C0000000000000000B1
:102DB0006465666100000000BBC1F579CE5C6A3CC9
:102DC0000000000000000000626F6F74000000004F
:102DD000BBC1207A1B796A3C0000000000000000A3
:102DE00068656C7000000000BBC18B79D05D6A3CE7
:102DF000000000000000000068000000000000006B
:102E0000BBC18B79D05D6A3C000000007379730010
:102E100067706C0000000700AB5A285D1D5ECE3263
:102E2000000000007379730067756E0000000700F2
:102E3000AF5A285DF85DCF320000803F7379730090
:102E400067636F0000000700B35A285DD25DCD3282
:102E50000000004073797300677061000000070094
:102E6000B75A285D1D5ED0320000004073797300B0
:102E70006764690000000700BB5A285DF85DD13225
:102E80000000000000000000676300000000000078
:102E9000BBC1D277E2776A3C00000000000000006E
:102EA0006D61000000000B04015B975DCF62C532CD
:102EB000CDCCCC3D000000006664000000000300A3
:102EC000D4C1285DF85D5F3F0000000075646100BB
:102ED0007564613000000300F0C1705DB75E263C90
:102EE000000000007564610075646131000003003A
:102EF000F0C1705DB75E2A3C00000000756461009F
:102F00007564613200000300F0C1705DB75E2E3C55
:102F10000000000075646100756461330000030007
:102F2000F0C1705DB75E323C000000007564620065
:102F30007564623000000300F0C1705DB75E363C1E
:102F400000000000756462007564623100000300D7
:102F5000F0C1705DB75E3A3C00000000756462002D
:102F60007564623200000300F0C1705DB75E3E3CE4
:102F700000000000756462007564623300000300A5
:102F8000F0C1705DB75E423C0000000075646300F4
:102F90007564633000000300F0C1705DB75E463CAD
:102FA0000000000075646300756463310000030075
:102FB000F0C1705DB75E4A3C0000000075646300BC
:102FC0007564633200000300F0C1705DB75E4E3C73
:102FD0000000000075646300756463330000030043
:102FE000F0C1705DB75E523C000000007564640083
:102FF0007564643000000300F0C1705DB75E563C3C
:103000000000000075646400756464310000030012
:10301000F0C1705DB75E5A3C00000000756464004A
:103020007564643200000300F0C1705DB75E5E3C01
:1030300000000000756464007564643300000300E0
:10304000F0C1705DB75E623C000000005F74650017
:103050005F746578000000020DC2975DD05D9557E2
:10306000000000005F7465005F7465790000000275
:103070000DC2975DD05D9957000000005F74650038
:103080005F74657A000000020DC2975DD05D9D57A8
:10309000000000005F7465005F746561000000025D
:1030A0000DC2975DD05DA157000000005F74650000
:1030B0005F746562000000020DC2975DD05DA55788
:1030C000000000005F7465005F746563000000022B
:1030D0000DC2975DD05DA957000000005F747200BB
:1030E0005F747278000000020DC2975DD05DBA581F
:1030F000000000005F7472005F74727900000002CB
:103100000DC2975DD05DBE58000000005F74720074
:103110005F74727A000000020DC2975DD05DC258E4
:10312000000000005F7472005F74726100000002B2
:103130000DC2975DD05DC658000000005F7472003C
:103140005F747262000000020DC2975DD05DCA58C4
:10315000000000005F7472005F7472630000000280
:103160000DC2975DD05DCE58000000005F74730003
:103170005F747331000000020DC2975DD05D255869
:10318000000000005F7073005F7073310000000288
:103190000DC2975DD05D3558000000005F6373007D
:1031A0005F637331000000020DC2975DD05D45582A
:1031B000000000005F6573005F657331000000026E
:1031C0000DC2975DD05D5558000000005F78730018
:1031D0005F787331000000020DC2975DD05D875BA0
:1031E000000000005F6665005F6665310000000258
:1031F0000DC2975DD05D6558000000005F747300DC
:103200005F747332000000020DC2975DD05D2958D3
:10321000000000005F7073005F70733200000002F6
:103220000DC2975DD05D3958000000005F637300E8
:103230005F637332000000020DC2975DD05D495894
:10324000000000005F6573005F65733200000002DC
:103250000DC2975DD05D5958000000005F78730083
:103260005F787332000000020DC2975DD05D9F5BF6
:10327000000000005F6665005F66653200000002C6
:103280000DC2975DD05D6958000000005F74730047
:103290005F747333000000020DC2975DD05D2D583E
:1032A000000000005F7073005F7073330000000265
:1032B0000DC2975DD05D3D58000000005F63730054
:1032C0005F637333000000020DC2975DD05D4D58FF
:1032D000000000005F6573005F657333000000024B
:1032E0000DC2975DD05D5D58000000005F787300EF
:1032F0005F787333000000020DC2975DD05DB75B4D
:10330000000000005F6665005F6665330000000234
:103310000DC2975DD05D6D58000000005F747300B2
:103320005F747334000000020DC2975DD05D3158A8
:10333000000000005F7073005F70733400000002D3
:103340000DC2975DD05D4158000000005F637300BF
:103350005F637334000000020DC2975DD05D515869
:10336000000000005F6573005F65733400000002B9
:103370000DC2975DD05D6158000000005F7873005A
:103380005F787334000000020DC2975DD05DCF5BA3
:10339000000000005F6665005F66653400000002A3
:1033A0000DC2975DD05D7158000000000000000064
:1033B0005F64616D00000000BBC1135A135A6A3C80
:1033C00000000000000000007365303000000200C3
:1033D000BBC14C5D675E3E5A00000000000000006B
:1033E0007365303100000200BBC14C5D675E405A1E
:1033F0000000000000000000736530320000020091
:10340000BBC14C5D675E425A000000000000000036
:103410007365303300000200BBC14C5D675E445AE7
:10342000000000000000000073653034000002005E
:10343000BBC14C5D675E465A000000000000000002
:103440007365303500000200BBC14C5D675E485AB1
:10345000000000000000000073653036000002002C
:10346000BBC14C5D675E4A5A0000000000000000CE
:103470007365303700000200BBC14C5D675E4C5A7B
:1034800000000000000000007365303800000200FA
:10349000BBC14C5D675E4E5A00000000000000009A
:1034A0007365303900000200BBC14C5D675E505A45
:1034B00000000000000000007365313000000200D1
:1034C000BBC14C5D675E525A000000000000000066
:1034D0007365313100000200BBC14C5D675E545A18
:1034E000000000000000000073653132000002009F
:1034F000BBC14C5D675E565A000000000000000032
:103500007365313300000200BBC14C5D675E585AE1
:10351000000000000000000073653134000002006C
:10352000BBC14C5D675E5A5A0000000000000000FD
:103530007365313500000200BBC14C5D675E5C5AAB
:10354000000000000000000073653136000002003A
:10355000BBC14C5D675E5E5A0000000000000000C9
:103560007365313700000200BBC14C5D675E605A75
:103570000000000000000000736531380000020008
:10358000BBC14C5D675E625A000000000000000095
:103590007365313900000200BBC14C5D675E645A3F
:1035A00000000000000000007365323000000200DF
:1035B000BBC14C5D675E665A000000000000000061
:1035C0007365323100000200BBC14C5D675E685A12
:1035D00000000000000000007365323200000200AD
:1035E000BBC14C5D675E6A5A00000000000000002D
:1035F0007365323300000200BBC14C5D675E6C5ADC
:10360000000000000000000073653234000002007A
:10361000BBC14C5D675E6E5A0000000000000000F8
:103620007365323500000200BBC14C5D675E705AA5
:103630000000000000000000736532360000020048
:10364000BBC14C5D675E725A0000000000000000C4
:103650007365323700000200BBC14C5D675E745A6F
:103660000000000000000000736532380000020016
:10367000BBC14C5D675E765A000000000000000090
:103680007365323900000200BBC14C5D675E785A39
:1036900000000000000000007379730000000000CB
:1036A000BBC1A460175F6A3C00000000000000007E
:1036B0007031000000000000BBC1A460175F6A3CCD
:1036C00000000000000000003100000000000000C9
:1036D000BBC1A460175F6A3C00000000000000004E
:1036E0003200000000000000BBC1A460175F6A3C0C
:1036F0000000000000000000330000000000000097
:10370000BBC1A460175F6A3C00000000000000001D
:103710003400000000000000BBC1A460175F6A3CD9
:103720000000000000000000780000000000000021
:10373000BBC1A460175F6A3C0000000000000000ED
:103740007900000000000000BBC1A460175F6A3C64
:1037500000000000000000007A00000000000000EF
:10376000BBC1A460175F6A3C0000000000000000BD
:103770006100000000000000BBC1A460175F6A3C4C
:1037800000000000000000006200000000000000D7
:10379000BBC1A460175F6A3C00000000000000008D
:1037A0006300000000000000BBC1A460175F6A3C1A
:1037B0000000000000000000673534000000000039
:1037C000BBC1A460175F6A3C00000000000000005D
:1037D0006735350000000000BBC1A460175F6A3C7C
:1037E0000000000000000000673536000000000007
:1037F000BBC1A460175F6A3C00000000000000002D
:103800006735370000000000BBC1A460175F6A3C49
:1038100000000000000000006735380000000000D4
:10382000BBC1A460175F6A3C0000000000000000FC
:103830006735390000000000BBC1A460175F6A3C17
:1038400000000000000000006739320000000000A6
:10385000BBC1A460175F6A3C0000000000000000CC
:103860006732380000000000BBC1A460175F6A3CEB
:10387000000000000000000067333000000000007E
:10388000BBC1A460175F6A3C00000000000000009C
:103890006D706F0000000000BBC1A460175F6A3C40
:1038A0000000000000000000706F730000000000C6
:1038B000BBC1A460175F6A3C00000000000000006C
:1038C0006F66730000000000BBC1A460175F6A3C14
:1038D0000000000000000000686F6D0000000000A4
:1038E000BBC1A460175F6A3C00000000000000003C
:1038F0007072620000000000BBC1A460175F6A3CE8
:10390000000000000000000070777200000000005E
:10391000BBC1A460175F6A3C00000000000000000B
:103920006A6F670000000000BBC1A460175F6A3CBB
:1039300000000000000000006A6964000000000050
:10394000BBC1A460175F6A3C0000000000000000DB
:103950007564610000000000BBC1A460175F6A3C91
:10396000000000000000000075646200000000001C
:10397000BBC1A460175F6A3C0000000000000000AB
:103980007564630000000000BBC1A460175F6A3C5F
:1039900000000000000000007564640000000000EA
:1039A000BBC1A460175F6A3C00000000000000007B
:1039B0005F74650000000000BBC1A460175F6A3C33
:1039C00000000000000000005F74720000000000B2
:1039D000BBC1A460175F6A3C00000000000000004B
:1039E0005F74730000000000BBC1A460175F6A3CF5
:1039F00000000000000000005F7073000000000085
:103A0000BBC1A460175F6A3C00000000000000001A
:103A10005F63730000000000BBC1A460175F6A3CD5
:103A200000000000000000005F657300000000005F
:103A3000BBC1A460175F6A3C0000000000000000EA
:103A40005F78730000000000BBC1A460175F6A3C90
:103A500000000000000000005F666500000000003C
:103A6000BBC1A460175F6A3C0000000000000000BA
:103A70006D00000000000000BBC19563D05D6A3C92
:103A800000000000000000007100000000000000C5
:103A9000BBC17B63D05D6A3C0000000000000000F9
:103AA0006F00000000000000BBC16163D05D6A3C94
:103AB00000000000000000002400000000000000E2
:103AC000BBC1AF63D05D6A3C00000000486F6D6908
:103AD0006E67206572726F72202D202563206178D9
:103AE00069732073657474696E6773206D6973639D
:103AF0006F6E666967757265640050726F62696E99
:103B000067206572726F72202D20256320617869AD
:103B1000732063616E6E6F74206D6F7665206475BF
:103B200072696E672070726F62696E67005B6964AC
:103B30005D202054696E7947204944253330730A4B
:103B4000005B68765D202068617264776172652031
:103B500076657273696F6E2531362E32660A005BA8
:103B600068705D2020686172647761726520706C96
:103B70006174666F726D2531352E32660A005B66A0
:103B8000765D20206669726D776172652076657258
:103B900073696F6E2531362E32660A005B66625D90
:103BA00020206669726D77617265206275696C6448
:103BB0002531382E32660A00456E74657220246203
:103BC0006F6F743D3120746F20656E746572207460
:103BD000686520626F6F74206C6F616465722E0A75
:103BE000000A0A0A2323232054696E794720424F92
:103BF0004F54204C4F414445522048656C7020235F
:103C000023230A00456E7465722024646566613D55
:103C10003120746F20726573657420746865207339
:103C2000797374656D20746F2074686520666163B4
:103C3000746F72792064656661756C742076616C4E
:103C40007565732E0A546869732077696C6C206FF0
:103C5000766572777269746520616E792063686138
:103C60006E67657320796F752068617665206D6178
:103C700064652E0A000A0A0A2323232054696E79F8
:103C80004720524553544F52452044454641554CD8
:103C900054532048656C70202323230A00496E7614
:103CA0006F6B652073656C66207465737420627930
:103CB00020656E746572696E672024746573743D47
:103CC0004E207768657265204E206973206F6E659F
:103CD000206F663A0A202024746573743D312020D9
:103CE000736D6F6B6520746573740A20202474658E
:103CF00073743D322020686F6D696E672074657340
:103D00007420202028796F75206D7573742074726B
:103D1000697020686F6D696E672073776974636876
:103D20006573290A202024746573743D3320207341
:103D3000717561726520746573742020202861207C
:103D4000736572696573206F662073717561726542
:103D500073290A202024746573743D342020617215
:103D600063207465737420202020202028736F6DD9
:103D700065206C6172676520636972636C65732985
:103D80000A202024746573743D3520206477656CA7
:103D90006C207465737420202020286D6F76657305
:103DA00020737061636564206279203120736563DC
:103DB0006F6E64206477656C6C73290A202024740C
:103DC0006573743D36202066656564686F6C642099
:103DD000746573742028656E746572202120616E8D
:103DE00064207E20746F20686F6C6420616E642094
:103DF000726573746172742C20726573706563747C
:103E00006976656C79290A202024746573743D37BE
:103E100020204D20636F64657320746573742020C7
:103E2000284D20636F64657320696E7465726D69D7
:103E30006E676C65642077697468206D6F76657352
:103E4000290A202024746573743D3820204A534F7A
:103E50004E20746573742020202020286D6F7469B3
:103E60006F6E20746573742072756E207573696E41
:103E700067204A534F4E20636F6D6D616E647329E6
:103E80000A202024746573743D392020696E76659C
:103E90007273652074696D6520746573740A2020DF
:103EA00024746573743D313020726F7461727920AF
:103EB0006D6F74696F6E20746573740A20202474AA
:103EC0006573743D313120736D616C6C206D6F765C
:103ED000657320746573740A202024746573743DBF
:103EE000313220736C6F77206D6F76657320746547
:103EF00073740A202024746573743D313320636F1A
:103F00006F7264696E6174652073797374656D2076
:103F10006F66667365742074657374202847393240
:103F20002C204735342D473539290A0A54657374D6
:103F30007320617373756D6520612063656E7465B0
:103F4000726564205859206F726967696E20616ECE
:103F500064206174206C656173742038306D6D204D
:103F6000636C656172616E636520696E20616C6C63
:103F700020646972656374696F6E730A5465737443
:103F80007320617373756D65205A206861732061B9
:103F900074206C656173742034306D6D20706F73A4
:103FA00069697469766520636C656172616E6365C9
:103FB0000A54657374732073746172742077697422
:103FC000682061204730205830205930205A302056
:103FD0006D6F76650A486F6D696E6720697320742E
:103FE000686520657863657074696F6E2E204E6F0A
:103FF00020696E697469616C20706F736974696F90
:104000006E206F7220636C656172616E63652069FA
:104010007320617373756D65640A000A0A0A2323AD
:10402000232054696E79472053454C46205445530C
:10403000542048656C70202323230A00456163687F
:10404000202420636F6D6D616E642061626F766500
:1040500020616C736F20646973706C617973207474
:10406000686520746F6B656E20666F722065616392
:10407000682073657474696E6720696E205B205DCB
:1040800020627261636B6574730A546F2076696590
:10409000772073657474696E677320656E746572DA
:1040A000206120746F6B656E3A0A0A2020243C74EC
:1040B0006F6B656E3E0A0A466F72206578616D709F
:1040C0006C65202479667220746F20646973706C4B
:1040D0006179207468652059206D61782066656576
:1040E0006420726174650A0A546F2075706461748B
:1040F000652073657474696E677320656E7465728C
:1041000020746F6B656E20657175616C73207661CC
:104110006C75653A0A0A2020243C746F6B656E3E0C
:104120003D3C76616C75653E0A0A466F7220657883
:10413000616D706C6520247966723D383030207472
:104140006F20736574207468652059206D61782034
:1041500066656564207261746520746F2038303044
:10416000206D6D2F6D696E7574650A466F722063E0
:104170006F6E66696775726174696F6E20646574CD
:1041800061696C73207365653A2068747470733A62
:104190002F2F6769746875622E636F6D2F73796E48
:1041A000746865746F732F54696E79472F77696BE4
:1041B000692F54696E79472D436F6E666967757212
:1041C0006174696F6E0A00546865736520636F6D72
:1041D0006D616E64732061726520616374697665D8
:1041E00020666F7220636F6E6669677572617469AD
:1041F0006F6E3A0A2020247379732053686F7720FA
:1042000073797374656D202867656E6572616C29BA
:104210002073657474696E67730A2020243120202E
:104220002053686F77206D6F746F72203120736533
:104230007474696E677320286F7220776861746583
:10424000766572206D6F746F7220796F752077615B
:104250006E7420312C322C332C34290A20202478FF
:1042600020202053686F772058206178697320736D
:10427000657474696E677320286F72207768617443
:1042800065766572206178697320796F7520776132
:104290006E7420782C792C7A2C612C622C63290A7C
:1042A0002020246D20202053686F7720616C6C20C3
:1042B0006D6F746F722073657474696E67730A2012
:1042C00020247120202053686F7720616C6C20615E
:1042D0007869732073657474696E67730A2020248B
:1042E0006F20202053686F7720616C6C206F6666AA
:1042F0007365742073657474696E67730A20202473
:104300002420202053686F7720616C6C20736574C3
:1043100074696E67730A2020246820202053686F18
:104320007720746869732068656C702073637265A8
:10433000656E0A0A000A0A0A2323232054696E794B
:104340004720434F4E46494755524154494F4E200E
:1043500048656C70202323230A000A466F7220648C
:10436000657461696C65642054696E794720696E73
:10437000666F207365653A2068747470733A2F2FE6
:104380006769746875622E636F6D2F73796E7468D8
:1043900065746F732F54696E79472F77696B692F36
:1043A0000A466F7220746865206C617465737420AE
:1043B0006669726D77617265207365653A2068740D
:1043C0007470733A2F2F6769746875622E636F6D0E
:1043D0002F73796E746865746F732F54696E7947A3
:1043E0000A506C65617365206C6F6720616E79207F
:1043F00069737375657320617420687474703A2FE3
:104400002F7777772E73796E746865746F732E6368
:104410006F6D2F666F72756D730A486176652066E1
:10442000756E0A000A4E6F74653A2054696E7947BA
:104430002067656E657261746573206175746F6D58
:104440006174696320737461747573207265706F31
:104450007274732062792064656661756C740A54A5
:104460006869732063616E206265206469736162AC
:104470006C656420627920656E746572696E672070
:104480002473763D300A536565207468652077692A
:104490006B692062656C6F7720666F72206D6F723A
:1044A000652064657461696C732E0A0054686573D5
:1044B0006520636F6D6D616E64732061726520614C
:1044C00063746976652066726F6D20746865206319
:1044D0006F6D6D616E64206C696E653A0A205E785E
:1044E0002020202020202020202020202052657302
:1044F00065742028636F6E74726F6C207829202D8C
:1045000020736F6674776172652072657365740AD3
:1045100020203F202020202020202020202020207C
:104520004D616368696E6520706F736974696F6E41
:1045300020616E642067636F6465206D6F64656CD5
:104540002073746174650A202024202020202020FC
:104550002020202020202053686F7720616E642067
:1045600073657420636F6E66696775726174696FD5
:104570006E2073657474696E67730A202021202091
:1045800020202020202020202020204665656468EF
:104590006F6C64202D2073746F70206D6F74696F61
:1045A0006E20776974686F7574206C6F73696E67BD
:1045B00020706F736974696F6E0A20207E2020203E
:1045C000202020202020202020204379636C65209B
:1045D0005374617274202D2072657374617274203B
:1045E00066726F6D2066656564686F6C640A202072
:1045F00068202020202020202020202020205368F8
:104600006F7720746869732068656C7020736372BB
:1046100065656E0A2020246820202020202020208C
:104620002020202053686F7720636F6E666967755E
:10463000726174696F6E2068656C70207363726557
:10464000656E0A20202474657374202020202020A9
:104650002020204C6973742073656C662D7465731B
:1046600074730A202024746573743D4E202020202A
:1046700020202052756E2073656C662D74657374EE
:10468000204E0A202024686F6D653D3120202020B7
:1046900020202052756E206120686F6D696E672042
:1046A0006379636C650A202024646566613D31206E
:1046B000202020202020526573746F726520616C69
:1046C0006C2073657474696E677320746F20226642
:1046D0006163746F7279222064656661756C7473AE
:1046E0000A000A0A0A2323232054696E79472048C6
:1046F000656C70202323230A005B6A735D20206AA7
:10470000736F6E2073657269616C697A652073746A
:10471000796C65253964205B303D72656C61786524
:10472000642C313D7374726963745D0A005B6A7650
:104730005D20206A736F6E20766572626F73697494
:104740007925313564205B303D73696C656E742C5E
:10475000313D666F6F7465722C323D6D65737361A8
:104760006765732C333D636F6E666967732C343DE8
:104770006C696E656E756D2C353D766572626F7312
:10478000655D0A005B656A5D2020656E61626C652F
:10479000206A736F6E206D6F646525313364205B12
:1047A000303D746578742C313D4A534F4E5D0A009C
:1047B000E158DB58D458CF58C658BB58B058A45805
:1047C00098588A587358645857584B5837582A582D
:1047D00015580158FE57FB57EC57D757C257B357D8
:1047E000A35791577A575D5740572757115700578E
:1047F000EE56E156CF56B556B256AF56AC56A95600
:10480000A656A356A0569D569A569756945691561C
:104810008E568B568856855682567F567C567956CC
:104820007656735670566D566A566756645661567C
:104830005E565B565856555652564F564C5649562C
:104840004656435640563D563A56375634563156DC
:104850002E562B562856255622561F561C5619568C
:104860001656EF55CB55AB55915577555D55395586
:104870001C550455EE54D454B0549354815461548F
:104880004A5431540F54F653D853BC53A453925343
:1048900074535F535B53575353534F534B534753C7
:1048A00043533F533B53375333532F532B532753C8
:1048B00023531F530553EB52D852BC52AA52935262
:1048C00072526152415221520752ED51D651A351B9
:1048D0007651565134510E51E750CB50AC50925056
:1048E000785053502A501250E74FBB4F854F504FCE
:1048F0003E4F2C4F1D4F0A4FF14ECF4EBD4EAB4E8B
:10490000994E874E754E634E514E3F4E2D4E1B4E67
:10491000094EF74DE54DD34DCF4DCB4DC74DC34D52
:10492000BF4DBB4DB74DB34DAF4DAB4DA74DA34D97
:104930009F4D9B4D974D934D8F4D8B4D874D834D87
:104940006F4D514D354D0A4DE54CC04CBC4CB84CEB
:10495000B44CB04CAC4CA84CA44CA04C9C4C984CC7
:10496000944C904C8C4C884C744C584C3C4C204C87
:10497000044CE84BCC4BB04B944B784B5C4B404BCE
:10498000244B204B1C4B184B144B104B0C4B084B1F
:10499000F44ACC4AA54A7F4A524A2C4AFF49FB496D
:1049A000F749F349E049BF49AA494A6F6767696E09
:1049B00067206379636C65206661696C656400508B
:1049C000726F626520656E64706F696E74206973C2
:1049D000207374617274696E6720706F696E740001
:1049E00050726F6265206379636C65206661696CE3
:1049F00065640032343900323438003234370048CC
:104A00006F6D696E67204572726F72202D20486F3E
:104A10006D696E67207377697463686573206D696B
:104A200073636F6E6669677572656400486F6D6960
:104A30006E67204572726F72202D204E656761741B
:104A4000697665206C61746368206261636B6F6670
:104A50006600486F6D696E67204572726F72202D17
:104A60002054726176656C206D696E2026206D6120
:104A70007820617265207468652073616D650048F7
:104A80006F6D696E67204572726F72202D204C61C8
:104A90007463682076656C6F63697479206973202C
:104AA0007A65726F00486F6D696E67204572726F2C
:104AB00072202D205365617263682076656C6F6388
:104AC000697479206973207A65726F00486F6D6927
:104AD0006E67204572726F72202D20426164206FD4
:104AE00072206E6F206178697320737065636966E8
:104AF00069656400486F6D696E67206379636C65F2
:104B0000206661696C6564003233390032333800E5
:104B1000323337003233360032333500323334002B
:104B200032333300536F6674206C696D697420658D
:104B300078636565646564202D2043206D6178008D
:104B4000536F6674206C696D697420657863656560
:104B5000646564202D2043206D696E00536F667478
:104B6000206C696D6974206578636565646564208F
:104B70002D2042206D617800536F6674206C696D42
:104B80006974206578636565646564202D20422022
:104B90006D696E00536F6674206C696D6974206571
:104BA00078636565646564202D2041206D6178001F
:104BB000536F6674206C696D6974206578636565F0
:104BC000646564202D2041206D696E00536F66740A
:104BD000206C696D6974206578636565646564201F
:104BE0002D205A206D617800536F6674206C696DBA
:104BF0006974206578636565646564202D205A209A
:104C00006D696E00536F6674206C696D6974206500
:104C100078636565646564202D2059206D61780096
:104C2000536F6674206C696D69742065786365657F
:104C3000646564202D2059206D696E00536F667481
:104C4000206C696D697420657863656564656420AE
:104C50002D2058206D617800536F6674206C696D4B
:104C60006974206578636565646564202D2058202B
:104C70006D696E00536F6674206C696D6974206590
:104C8000786365656465640032313900323138001B
:104C900032313700323136003231350032313400B2
:104CA00032313300323132003231310032313000B2
:104CB000323039003230380032303700323036008E
:104CC00054726170657A6F696420706C616E6E6594
:104CD00072206661696C656420746F20636F6E7604
:104CE00065726765004C696D6974207377697463D8
:104CF0006820686974202D2053687574646F776E1E
:104D0000206F63637572726564004D616368696EDC
:104D10006520697320616C61726D6564202D20438C
:104D20006F6D6D616E64206E6F742070726F63655D
:104D300073736564004D6F7665206C6573732074C2
:104D400068616E206D696E696D756D2074696D6541
:104D5000004D6F7665206C657373207468616E20FA
:104D60006D696E696D756D206C656E67746800475E
:104D7000656E657269632054696E79472065727249
:104D80006F7200313939003139380031393700312B
:104D90003936003139350031393400313933003199
:104DA0003932003139310031393000313839003190
:104DB0003838003138370031383600313835003175
:104DC0003834003138330031383200313831003175
:104DD0003830005420776F726420697320696E76D2
:104DE000616C6964005420776F7264206973206D70
:104DF000697373696E67005220776F7264206973FC
:104E000020696E76616C6964005220776F7264204D
:104E10006973206D697373696E67005120776F72D3
:104E20006420697320696E76616C69640051207733
:104E30006F7264206973206D697373696E67004CCB
:104E400020776F726420697320696E76616C696483
:104E5000004C20776F7264206973206D69737369E9
:104E60006E67004820776F726420697320696E76E0
:104E7000616C6964004820776F7264206973206DEB
:104E8000697373696E67004520776F726420697378
:104E900020696E76616C6964004520776F726420CA
:104EA0006973206D697373696E67004420776F7250
:104EB0006420697320696E76616C696400442077B0
:104EC0006F7264206973206D697373696E67005037
:104ED00020776F7264206973206E6F742061207672
:104EE000616C696420746F6F6C206E756D626572A1
:104EF000005020776F7264206973206E6F74206198
:104F00006E20696E7465676572005020776F7264F9
:104F1000206973206E65676174697665005020773B
:104F20006F7264206973207A65726F005020776F0A
:104F3000726420697320696E76616C696400502028
:104F4000776F7264206973206D697373696E67008F
:104F50004172632073706563696669636174696F28
:104F60006E206572726F72202D20656E64706F699D
:104F70006E74206973207374617274696E67207037
:104F80006F696E740041726320737065636966694E
:104F9000636174696F6E206572726F72202D20726A
:104FA000616469757320617263206F7574206F6628
:104FB00020746F6C6572616E63650041726320736B
:104FC000706563696669636174696F6E206572728A
:104FD0006F72202D206D697373696E67206F66662E
:104FE0007365742873290041726320737065636967
:104FF0006669636174696F6E206572726F72202DCD
:10500000206D697373696E672061786973286573B1
:105010002900417263207370656369666963617416
:10502000696F6E206572726F72005370696E646C86
:1050300065206D757374206265207475726E696E7B
:105040006720666F72207468697320636F6D6D618D
:105050006E64005370696E646C65206D75737420A6
:105060006265206F666620666F72207468697320BF
:10507000636F6D6D616E64005370696E646C652062
:105080005320776F726420697320696E76616C6952
:1050900064005370696E646C65205320776F72648E
:1050A000206973206D697373696E67005370696E50
:1050B000646C6520737065656420657863656564FC
:1050C0006564206D6178696D756D005370696E64FB
:1050D0006C652073706565642062656C6F77206D08
:1050E000696E696D756D0050726F6772616D6D6587
:1050F0006420706F696E742073616D652061732028
:1051000063757272656E7420706F696E740043759A
:105110007474657220636F6D70656E736174696F0E
:105120006E2063616E6E6F7420626520656E6162D1
:105130006C6564005265717565737465642076658D
:105140006C6F636974792065786365656473206C3E
:10515000696D697473004730206F72204731206D8C
:105160007573742062652061637469766520666F6B
:10517000722047353300526F74617279206178650F
:10518000732063616E6E6F74206265207573656451
:105190002077697468207468697320636F6D6D612E
:1051A0006E6400496E76657273652074696D652062
:1051B0006D6F64652063616E6E6F7420626520752B
:1051C0007365642077697468207468697320636FFD
:1051D0006D6D616E64004665656472617465206E14
:1051E0006F74207370656369666965640053656CEC
:1051F000656374656420706C616E652069732069F5
:105200006E76616C69640053656C656374656420D7
:10521000706C616E65206973206D697373696E6768
:1052200000417869732074617267657420706F73D0
:105230006974696F6E20697320696E76616C696448
:1052400000417869732074617267657420706F73B0
:105250006974696F6E206973206D697373696E6715
:1052600000417869732069732064697361626C65B9
:1052700064004178697320697320696E76616C6996
:105280006420666F72207468697320636F6D6D614E
:105290006E6400417869732063616E6E6F74206282
:1052A000652070726573656E74004178697320774C
:1052B0006F7264206D697373696E670047636F6412
:1052C00065206D6F64616C2067726F757020766900
:1052D0006F6C6174696F6E004D20636F646520753B
:1052E0006E737570706F727465640047636F646588
:1052F00020636F6D6D616E6420756E737570706F75
:10530000727465640047656E657269632047636FF8
:10531000646520696E707574206572726F720031F9
:105320003239003132380031323700313236003113
:105330003235003132340031323300313232003113
:105340003231003132300031313900313138003101
:105350003137003131360031313500313134004AD6
:10536000534F4E20737472696E6720746F6F206C98
:105370006F6E67004A534F4E20696E7075742068D7
:10538000617320746F6F206D616E79207061697236
:1053900073004A534F4E2073796E746178206572A2
:1053A000726F7200496E7075742076616C7565203D
:1053B00072616E6765206572726F7200496E7075FA
:1053C000742065786365656473206D6178696D75B7
:1053D0006D2076616C756500496E707574206C6522
:1053E0007373207468616E206D696E696D756D20D0
:1053F00076616C756500496E7075742065786365BB
:10540000656473206D6178206C656E677468004315
:105410006F6D6D616E64206E6F7420616363657083
:1054200074656420617420746869732074696D65A3
:1054300000506172616D657465722063616E6E6F9C
:1054400074206265207265616400506172616D65EF
:1054500074657220697320726561642D6F6E6C795A
:1054600000556E737570706F72746564206E756D23
:10547000626572206F72204A534F4E2074797065B6
:1054800000426164206E756D62657220666F726D98
:10549000617400496E76616C6964206F72206D6181
:1054A0006C666F726D656420636F6D6D616E640014
:1054B000556E7265636F676E697A656420636F6DA0
:1054C0006D616E64206F7220636F6E666967206E17
:1054D000616D650047656E65726963206173736510
:1054E0007274696F6E206661696C757265004D65D6
:1054F0006D6F7279206661756C7420646574656384
:1055000074656400537461636B206F766572666CBA
:105510006F7720646574656374656400436F6E74AF
:10552000726F6C6C657220617373657274696F6EF3
:10553000206661696C7572650043616E6F6E6963A8
:10554000616C206D616368696E652061737365725B
:1055500074696F6E206661696C75726500506C616C
:105560006E6E657220617373657274696F6E20660A
:1055700061696C7572650053746570706572206145
:105580007373657274696F6E206661696C7572659C
:1055900000456E636F646572206173736572746930
:1055A0006F6E206661696C75726500494F20737576
:1055B000622D73797374656D20617373657274699C
:1055C0006F6E206661696C75726500436F6E666907
:1055D00067207375622D73797374656D20617373C1
:1055E000657274696F6E206661696C7572650049D9
:1055F0004F206D656D6F727920616C6C6F636174A3
:10560000696F6E20617373657274696F6E20666175
:10561000696C7572650038380038370038360038E4
:105620003500383400383300383200383100383033
:105630000037390037380037370037360037350044
:105640003734003733003732003731003730003617
:1056500039003638003637003636003635003634F5
:10566000003633003632003631003630003539002E
:1056700035380035370035360035350035340035DE
:1056800033003532003531003530003439003438DC
:1056900000343700343600343500343400343300FD
:1056A00034320034310034300033390033380033C1
:1056B000370033360042616420737461747573205F
:1056C0007265706F72742073657474696E670050D0
:1056D000657273697374656E6365206572726F724B
:1056E00000466C6F6174206973204E414E00466C19
:1056F0006F617420697320696E66696E69746500F4
:105700004D6F76652074696D65206973204E414E3A
:10571000004D6F76652074696D6520697320696E30
:1057200066696E6974650047656E657269632065B8
:105730007863657074696F6E207265706F72740043
:105740004661696C656420746F2067657420706CB5
:10575000616E6E657220627566666572005379735C
:1057600074656D20616C61726D202D207368757495
:1057700074696E6720646F776E00496E6974696141
:105780006C697A6174696F6E206661696C757265A7
:1057900000526561642D6F6E6C792061646472657E
:1057A000737300496E76616C69642041646472654C
:1057B000737300446976696465206279207A657242
:1057C0006F00466C6F6174696E6720706F696E74EC
:1057D000206572726F7200496E7465726E616C2022
:1057E00072616E6765206572726F7200496E7465D2
:1057F000726E616C206572726F72003139003138DF
:105800000046756E6374696F6E20697320737475DA
:105810006262656400456E746572696E6720626FCE
:105820006F74206C6F6164657200496E69746961A0
:105830006C697A696E670042756666657220667586
:105840006C6C202D20666174616C00427566666523
:10585000722066756C6C0042756666657220656DB7
:10586000707479004E6F2073756368206465766983
:105870006365004D61782066696C652073697A659F
:105880002065786365656465640046696C65206EB3
:105890006F74206F70656E00456E64206F662066C1
:1058A000696C6500456E64206F66206C696E6500EA
:1058B00048617264207265736574005465726D6925
:1058C0006E6174656400436F6D706C657465004E45
:1058D0006F6F700045616761696E004572726F722B
:1058E000004F4B005B7031706F665D2070776D20EC
:1058F0007068617365206F66662020202531352E23
:105900003366205B302E2E315D0A005B703177707C
:10591000685D2070776D20636377207068617365C0
:105920002068692531352E3366205B302E2E315D9F
:105930000A005B703177706C5D2070776D20636357
:1059400077207068617365206C6F2531352E336662
:10595000205B302E2E315D0A005B70317773685DFD
:105960002070776D206363772073706565642068AD
:10597000692531352E30662052504D0A005B70315A
:1059800077736C5D2070776D20636377207370652B
:105990006564206C6F2531352E30662052504D0ADB
:1059A000005B70316370685D2070776D20637720D5
:1059B0007068617365206869202531352E33662053
:1059C0005B302E2E315D0A005B703163706C5D20A0
:1059D00070776D206377207068617365206C6F202D
:1059E0002531352E3366205B302E2E315D0A005B6B
:1059F00070316373685D2070776D206377207370FA
:105A0000656564206869202531352E306620525046
:105A10004D0A005B703163736C5D2070776D20639D
:105A200077207370656564206C6F202531352E30CA
:105A3000662052504D0A005B70316672715D2070B5
:105A4000776D206672657175656E637920202025FB
:105A500031352E306620487A0A0053595354454D4B
:105A6000205245414459004C6F6164696E67206360
:105A70006F6E666967732066726F6D204545505280
:105A80004F4D00496E697469616C697A696E67206F
:105A9000636F6E6669677320746F204F4D43204FAC
:105AA000746865724D696C6C2073657474696E6797
:105AB00073007B226572223A7B226662223A25308D
:105AC0002E32662C227374223A25642C226D736761
:105AD000223A222573227D7D0A007B65723A7B661D
:105AE000623A25302E32662C73743A25642C6D731D
:105AF000673A222573227D7D0A005B71765D202046
:105B00007175657565207265706F72742076657247
:105B1000626F73697479253764205B303D6F666608
:105B20002C313D73696E676C652C323D74726970FF
:105B30006C655D0A00716F3A25640A0071693A2547
:105B4000640A0071723A25640A005B73765D202056
:105B5000737461747573207265706F7274207665EA
:105B600072626F73697479253664205B303D6F66AD
:105B7000662C313D66696C74657265642C323D76C5
:105B80006572626F73655D0A005B73695D202073E7
:105B9000746174757320696E74657276616C2531F9
:105BA000342E3066206D730A004D6F746F7220259D
:105BB0006320706F77657220656E61626C6564202A
:105BC00073746174653A25322E30660A005B257362
:105BD00025735D206D257320706F776572206D6170
:105BE0006E6167656D656E7425313064205B303D94
:105BF00064697361626C65642C313D616C776179B5
:105C000073206F6E2C323D696E206379636C652C56
:105C1000333D7768656E206D6F76696E675D0A004B
:105C20005B257325735D206D257320706F6C617229
:105C300069747925313864205B303D6E6F726D6117
:105C40006C2C313D726576657273655D0A005B256B
:105C50007325735D206D2573206D6963726F737496
:105C600065707325313664205B312C322C342C382E
:105C70005D0A005B257325735D206D2573207472AA
:105C80006176656C20706572207265766F6C7574D4
:105C9000696F6E2531302E346625730A005B2573DB
:105CA00025735D206D2573207374657020616E67A8
:105CB0006C652532302E336625730A005B2573250B
:105CC000735D206D2573206D617020746F20617885
:105CD000697325313564205B303D582C313D592C9A
:105CE000323D5A2E2E2E5D0A005B6D745D20206DB4
:105CF0006F746F722069646C652074696D656F756F
:105D0000742531342E3266205365630A001C5D18F9
:105D10005D135D2064656700206D6D0020696E0075
:105D20005B73745D20207377697463682074797085
:105D30006525313864205B303D4E4F2C313D4E435C
:105D40005D0A005465737420232564206E6F7420EF
:105D5000666F756E640A004E312054314D360A4E1E
:105D600032204731370A4E33204732310A4E38202D
:105D700046313830300A4E392047310A4E31303002
:105D80002047393220582D32352E313737592D33AF
:105D9000342E303732205A2D312E303030202854D6
:105DA000454D502C2052454D4F5645204C415445B1
:105DB00052290A4E33343320582D32352E35393599
:105DC000592D33342E3334390A4E33343420582D80
:105DD00032352E373031592D33342E3433360A4E86
:105DE00033343520582D32352E373931592D33344F
:105DF0002E3532300A4E33343620582D32352E3877
:105E00003634592D33342E3630310A4E3334372060
:105E1000582D32352E393230592D33342E3637390C
:105E20000A4E33343820582D32352E393630592D1C
:105E300033342E3735340A4E33343920582D323529
:105E40002E393832592D33342E3832360A4E333506
:105E50003020582D32352E393837592D33342E38DD
:105E600039350A4E33353120582D32352E393736F3
:105E7000592D33342E3936310A4E33353220582DD0
:105E800032352E393438592D33352E3032330A4ECF
:105E900033353320582D32352E393033592D3335A3
:105EA0002E3038320A4E33353420582D32352E38C4
:105EB0003431592D33352E3133380A4E33353520B0
:105EC000582D32352E373633592D33352E31393062
:105ED0000A4E33353620582D32352E363639592D67
:105EE00033352E3233390A4E33353720582D32357B
:105EF0002E353539592D33352E3238340A4E333557
:105F00003820582D32352E343333592D33352E3336
:105F100032350A4E33353920582D32352E3239314B
:105F2000592D33352E3336330A4E33363020582D23
:105F300032352E313334592D33352E3339370A4E1D
:105F400033363120582D32342E393633592D3335EE
:105F50002E3432380A4E33363220582D32342E3712
:105F60003737592D33352E3435350A4E33363320F5
:105F7000582D32342E353737592D33352E343737A7
:105F80000A4E33363420582D32342E333637592DBD
:105F900033352E3439360A4E33363520582D3234C7
:105FA0002E313434592D33352E3531310A4E3336B6
:105FB0003620582D32332E393039592D33352E3580
:105FC00032320A4E33363720582D32332E363631A0
:105FD000592D33352E3532390A4E33363820582D67
:105FE00032332E343033592D33352E3533320A4E79
:105FF00033363920582D32332E313333592D333542
:106000002E3533320A4E33373020582D32322E3867
:106010003533592D33352E3532370A2F4E3235313F
:106020003820473058302E333237592D33332E3500
:1060300032315A2D312E3030300A4E32353139203E
:106040004D3330004E31204732300A4E3520473430
:1060500030204731370A4E3130205431204D303610
:106060000A284E313520473930204730205830201B
:106070005930205A30290A4E3230205335303030D2
:10608000204D3033200A4E32352058302E303634F1
:106090002059302E333236205A300A4E34302047C1
:1060A0003031204631362E300A4E35302058302ED1
:1060B0003036342059302E3332360A4E353520589A
:1060C000302E3036302059302E3239330A4E3630A9
:1060D0002058302E3037372059302E3236370A4E7E
:1060E00036352058302E3131312059302E32353767
:1060F0000A4E37302058302E3134392059302E3264
:1061000035320A4E37352058302E31383820593044
:106110002E3235350A4E38302058302E3232372064
:1061200059302E3236380A4E38352058302E323516
:10613000372059302E3237310A4E39302058302E20
:106140003333352059302E3236350A4E3935205802
:10615000302E3431322059302E3237310A4E313020
:10616000302058302E3437342059302E3238370A08
:106170004E3130352058302E3439312059302E32BE
:1061800038390A4E3131302058302E3531372059C8
:10619000302E3237330A4E3131352058302E3534D7
:1061A000342059302E3236330A4E313230205830B6
:1061B0002E3538302059302E3236310A4E313235B4
:1061C0002058302E3539352059302E3236330A4E8C
:1061D0003133302058302E3632312059302E32377C
:1061E000340A4E3133352058302E36353920593067
:1061F0002E3330360A4E3134302058302E36373375
:106200002059302E3333350A4E3134352058302E54
:106210003637392059302E3336310A4E3135302059
:1062200058302E3637382059302E3338390A4E310F
:1062300035352058302E3637302059302E34323014
:106240000A4E3136302058302E3637302059302E15
:106250003434360A4E3136352058302E3638302018
:1062600059302E3437340A4E3137302058302E37DB
:1062700030342059302E3439370A4E3137352058D2
:10628000302E3733322059302E3531350A4E3138E1
:10629000302058302E3739342059302E3533350AD6
:1062A0004E3138352058302E3837322059302E357F
:1062B00036370A4E3139302058302E393530205992
:1062C000302E3630340A4E3139352058312E3033A5
:1062D000312059302E3634370A4E32303020583182
:1062E0002E3134392059302E3732320A4E32303581
:1062F0002058312E3330382059302E3835340A4E5C
:106300003231302058312E3433302059302E393844
:10631000340A4E3231352058312E3434372059303A
:106320002E3938360A4E3232302058312E36323835
:106330002059302E3832320A4E3232352058312E22
:106340003733322059302E3731340A4E3233302031
:1063500058322E3030392059302E3338310A4E32EF
:1063600033352058322E3131362059302E323636E0
:106370000A4E3234302058322E3232382059302EE4
:106380003135370A4E3234352058322E32383020EB
:1063900059302E3132330A4E3235302058322E33B6
:1063A00033322059302E3039340A4E3235352058A8
:1063B000322E3432332059302E3037300A4E3236B6
:1063C000302058322E3438392059302E3036350AA4
:1063D0004E3236352058322E3535372059302E3052
:1063E00036360A4E3237302058322E363237205960
:1063F000302E3038340A4E3237352058322E363966
:10640000332059302E3130390A4E3238302058324C
:106410002E3733302059302E3133330A4E3238354F
:106420002058322E3830352059302E3139300A4E2E
:106430003239302058322E3832392059302E32310C
:10644000360A4E3239352058322E383830205930FD
:106450002E3239310A4E3330302058322E3838340B
:106460002059302E3330300A4E3330352058322EFA
:106470003839382059302E3333320A4E33313020F8
:1064800058322E3930352059302E3336370A4E33B4
:1064900031352058322E3931302059302E343037B2
:1064A0000A4E3332302058322E3930382059302EAF
:1064B0003434360A4E3332352058322E39303120BA
:1064C00059302E3439350A4E3333302058322E3875
:1064D00039372059302E3439350A4E333335205868
:1064E000322E3839302059302E3532340A4E33347A
:1064F000302058322E3834322059302E3630340A7B
:106500004E3334352058322E3831342059302E361F
:1065100036350A4E3335302058322E37393420592B
:10652000302E3735300A4E3335352058322E373934
:10653000312059302E3833380A4E33363020583215
:106540002E3831392059302E3937360A4E33363508
:106550002058322E3833372059312E3034340A4EF9
:106560003337302058322E3836322059312E3131DF
:10657000320A4E3337352058322E383737205931CA
:106580002E3134350A4E3338302058322E393132DC
:106590002059312E3231370A4E3338352058322EB9
:1065A0003931372059312E3232360A4E33393020C4
:1065B00058322E3935312059312E3238310A4E3386
:1065C00039352058322E3937302059312E3239356D
:1065D0000A4E3430302058322E3939362059312E77
:1065E0003239350A4E3430352058332E303133208D
:1065F00059312E3237350A4E3431302058332E304F
:1066000032342059312E3235340A4E343135205847
:10661000332E3037302059312E3135310A4E343255
:10662000302058332E3037372059312E3133340A49
:106630004E3432352058332E3132352059312E30F8
:1066400033390A4E3433302058332E313338205901
:10665000312E3031390A4E3433352058332E323012
:10666000352059302E3930380A4E343430205833E2
:106670002E3238322059302E3739370A4E343435DD
:106680002058332E3336312059302E3639310A4EC8
:106690003435302058332E3432362059302E3539A7
:1066A000320A4E3435352058332E343536205930A1
:1066B0002E3534330A4E3436302058332E343739A1
:1066C0002059302E3439330A4E3436352058332E83
:1066D0003439342059302E3437320A4E3437302092
:1066E00058332E3530352059302E3434360A4E3456
:1066F00037352058332E3531382059302E34313744
:106700000A4E3438302058332E3533302059302E4D
:106710003339310A4E3438352058332E353634204B
:1067200059302E3330300A4E3439302058332E351C
:1067300037372059302E3235330A4E343935205808
:10674000332E3536382059302E3231320A4E35301C
:10675000302058332E3534342059302E3137360A14
:106760004E3530352058332E3534312059302E31C6
:1067700034360A4E3531302058332E3535332059D2
:10678000302E3131390A4E3531352058332E3537D8
:10679000362059302E3130360A4E353230205833BB
:1067A0002E3539372059302E3130320A4E353235B8
:1067B0002058332E3631382059302E3130390A4E98
:1067C0003533302058332E3633392059302E31327C
:1067D000390A4E3533352058332E3635302059306E
:1067E0002E3135390A4E3534302058332E36363373
:1067F0002059302E3137380A4E3534352058332E53
:106800003637382059302E3139320A4E353530205E
:1068100058332E3639392059302E3139370A4E3512
:1068200035352058332E3732332059302E31393612
:106830000A4E3536302058332E3736342059302E14
:106840003137390A4E3536352058332E3830352019
:1068500059302E3136350A4E3537302058332E38E0
:1068600038342059302E3135390A4E3537352058D5
:10687000332E3934392059302E3136350A4E3538D9
:10688000302058332E3936362059302E3137350ADC
:106890004E3538352058332E3937382059302E317F
:1068A00039340A4E3539302058332E39373820598B
:1068B000302E3232330A4E3539352058332E3936A0
:1068C000302059302E3234350A4E3630302058338D
:1068D0002E3833342059302E3331310A4E3630358C
:1068E0002058332E3736322059302E3334350A4E65
:1068F0003631302058332E3732362059302E333847
:10690000390A4E3631352058332E3730332059303E
:106910002E3435380A4E3632302058332E3638323F
:106920002059302E3533300A4E3632352058332E2A
:106930003637392059302E3533340A4E363330202D
:1069400058332E3632362059302E3638310A4E36EC
:1069500033352058332E3536382059302E383238DA
:106960000A4E3634302058332E3434342059312EE8
:106970003038300A4E3634352058332E34303520F6
:1069800059312E3136370A4E3635302058332E34B1
:1069900030342059312E3136370A4E3635352058AD
:1069A000332E3338372059312E3230380A4E3636AE
:1069B000302058332E3338342059312E3230380AB3
:1069C0004E3636352058332E3336352059312E3257
:1069D00036350A4E3637302058332E333535205968
:1069E000312E3238350A4E3637352058332E33346F
:1069F000382059312E3330380A4E3638302058334B
:106A00002E3333332059312E3335300A4E36383554
:106A10002058332E3332312059312E3339310A4E3A
:106A20003639302058332E3331312059312E34321B
:106A3000380A4E3639352058332E33333920593100
:106A40002E3432330A4E3730302058332E3434301F
:106A50002059312E3430360A4E3730352058332EF7
:106A60003531302059312E3430380A4E373130200C
:106A700058332E3538352059312E3432310A4E37BD
:106A800031352058332E3631312059312E343339B7
:106A90000A4E3732302058332E3631312059312EBC
:106AA0003434310A4E3732352058332E36313520C2
:106AB00059312E3434310A4E3733302058332E3684
:106AC00033362059312E3438380A4E373335205872
:106AD000332E3633342059312E3531370A4E373480
:106AE000302058332E3632322059312E3534330A85
:106AF0004E3734352058332E3630352059312E3527
:106B000036330A4E3735302058332E353736205934
:106B1000312E3537350A4E3735352058332E35343A
:106B2000342059312E3538310A4E3736302058331B
:106B30002E3437392059312E3539320A4E37363511
:106B40002058332E3435312059312E3539380A4EFC
:106B50003737302058332E3338372059312E3632DC
:106B6000360A4E3737352058332E333930205931D5
:106B70002E3633360A4E3738302058332E353332DE
:106B80002059312E3630320A4E3738352058332EC0
:106B90003630312059312E3539370A4E37393020C9
:106BA00058332E3636382059312E3539380A4E377B
:106BB00039352058332E3738322059312E3631327C
:106BC0000A4E3830302058332E3739342059312E80
:106BD0003631380A4E3830352058332E3836382082
:106BE00059312E3633360A4E3831302058332E394B
:106BF00031382059312E3635350A4E383135205846
:106C0000332E3934352059312E3636370A4E383244
:106C1000302058332E3936342059312E3638350A43
:106C20004E3832352058332E3936372059312E36EA
:106C300038350A4E3833302058332E3937342059FE
:106C4000312E3639390A4E3833352058332E3938FB
:106C5000342059312E3732350A4E383430205833EB
:106C60002E3938342059312E3735380A4E383435DC
:106C70002058332E3937302059312E3739300A4ECB
:106C80003835302058332E3934352059312E3831AB
:106C9000370A4E3835352058332E3931382059319E
:106CA0002E3832360A4E3836302058332E383931A5
:106CB0002059312E3832370A4E3836352058332E87
:106CC0003834322059312E3830390A4E3837302096
:106CD00058332E3739382059312E3738340A4E3848
:106CE00037352058332E3734362059312E37373246
:106CF0000A4E3838302058332E3639382059312E44
:106D00003736340A4E3838352058332E363335204E
:106D100059312E3736360A4E3839302058332E3511
:106D200035332059312E3738350A4E383935205809
:106D3000332E3437382059312E3832300A4E39301C
:106D4000302058332E3430392059312E3836340A19
:106D50004E3930352058332E3334352059312E39C1
:106D600031380A4E3931302058332E3236342059DA
:106D7000322E3032330A4E3931352058332E3234E8
:106D8000382059322E3035310A4E393230205833BE
:106D90002E3234302059322E3038310A4E393235C5
:106DA0002058332E3331362059322E3038360A4EA1
:106DB0003933302058332E3339302059322E313088
:106DC000340A4E3933352058332E34313420593279
:106DD0002E3132310A4E3934302058332E3433318B
:106DE0002059322E3135330A4E3934352058332E5E
:106DF0003433332059322E3138300A4E3935302071
:106E000058332E3432372059322E3230350A4E392B
:106E100035352058332E3431332059322E32323426
:106E20000A4E3936302058332E3339322059322E1B
:106E30003234320A4E3936352058332E333335202A
:106E400059322E3234340A4E3937302058332E32EC
:106E500037382059322E3233360A4E3937352058DA
:106E6000332E3235362059322E3234320A4E3938EA
:106E7000302058332E3233392059322E3235310AF0
:106E80004E3938352058332E3231312059322E3296
:106E900038300A4E3939302058332E3137342059A2
:106EA000322E3335360A4E3939352058332E3135A6
:106EB000392059322E3339370A4E3130303020588C
:106EC000332E3135302059322E3433380A4E31309A
:106ED00030352058332E3134302059322E34383169
:106EE0000A4E313031302058332E3133322059326E
:106EF0002E3531300A4E313031352058332E313174
:106F0000382059322E3534330A4E31303230205841
:106F1000332E3039392059322E3537360A4E31303A
:106F200032352058332E3035312059322E36333118
:106F30000A4E313033302058332E3030332059321E
:106F40002E3636360A4E313033352058322E39350A
:106F5000372059322E3638350A4E313034302058E9
:106F6000322E3930372059322E3639390A4E3130E7
:106F700034352058322E3836302059322E373131C0
:106F80000A4E313035302058322E383139205932BE
:106F90002E3732370A4E313035352058322E3736BB
:106FA000382059322E3734350A4E31303630205899
:106FB000322E3731362059322E3735370A4E31309E
:106FC00036352058322E3637352059322E37353760
:106FD0000A4E313037302058322E35373920593269
:106FE0002E3733310A4E313037352058322E35376F
:106FF000302059322E3732330A4E31303830205853
:10700000322E3535392059322E3732300A4E313052
:1070100038352058322E3533302059322E37303122
:107020000A4E313039302058322E35303120593225
:107030002E3639330A4E313039352058322E343716
:10704000312059322E3638330A4E31313030205803
:10705000322E3434332059322E3636380A4E3131FE
:1070600030352058322E3339362059322E363334CB
:107070000A4E313131302058322E333534205932D6
:107080002E3539310A4E313131352058322E3335D3
:10709000322059322E3539310A4E313132302058B2
:1070A000322E3332352059322E3534330A4E3131B7
:1070B00032352058322E3331352059322E35323187
:1070C0000A4E313133302058322E33303720593286
:1070D0002E3439380A4E313133352058322E323978
:1070E000362059322E3436340A4E3131343020585D
:1070F000322E3239332059322E3432370A4E313162
:1071000034352058322E3239352059322E33363626
:107110000A4E313135302058322E33323120593237
:107120002E3330330A4E313135352058322E333537
:10713000382059322E3234370A4E31313630205809
:10714000322E3431392059322E3230330A4E313119
:1071500036352058322E3431392059322E313739D4
:107160000A4E313137302058322E343035205932E2
:107170002E3135380A4E313137352058322E3336DC
:10718000322059322E3132330A4E313138302058C4
:10719000322E3335342059322E3130340A4E3131CB
:1071A00038352058322E3335342059322E3039318B
:1071B0000A4E313139302058322E3338302059328E
:1071C0002E3036350A4E313139352058322E343191
:1071D000302059322E3035310A4E3132303020587D
:1071E000322E3431302059322E3034370A4E31327B
:1071F00030352058322E3430352059322E30323846
:107200000A4E313231302058322E34303820593243
:107210002E3031300A4E313231352058322E343151
:10722000362059312E3939350A4E31323230205814
:10723000322E3433332059312E3938320A4E31321E
:1072400032352058322E3433382059312E393633E6
:107250000A4E313233302058322E343437205931EF
:107260002E3934380A4E313233352058322E3436E6
:10727000312059312E3933380A4E313234302058CA
:10728000322E3438302059312E3933310A4E3132D2
:1072900034352058322E3437382059312E38393988
:1072A0000A4E313235302058322E34383720593199
:1072B0002E3837350A4E313235352058322E35309A
:1072C000342059312E3835340A4E31323630205878
:1072D000322E3532372059312E3834380A4E313279
:1072E00036352058322E3534392059312E3834393C
:1072F0000A4E313237302058322E35373720593147
:107300002E3836310A4E313237352058322E36304B
:10731000342059312E3836360A4E31323830205822
:10732000322E3633312059312E3835340A4E31322F
:1073300038352058322E3634302059312E383237F5
:107340000A4E313239302058322E363430205931FD
:107350002E3739320A4E313239352058322E3632F4
:10736000392059312E3735390A4E313330302058D3
:10737000322E3631322059312E3732370A4E3133E0
:1073800030352058322E3537362059312E363934A3
:107390000A4E313331302058322E353336205931B0
:1073A0002E3636320A4E313331352058322E3437AC
:1073B000302059312E3631360A4E31333230205892
:1073C000322E3334352059312E3535310A4E313392
:1073D00032352058322E3330372059312E35323164
:1073E0000A4E313333302058322E32363020593164
:1073F0002E3438320A4E313333352058322E32345F
:10740000332059312E3437370A4E31333430205837
:10741000322E3232382059312E3436390A4E313339
:1074200034352058322E3232322059312E3434380D
:107430000A4E313335302058322E3232382059310D
:107440002E3432350A4E313335352058322E32350E
:10745000342059312E3430350A4E313336302058ED
:10746000322E3236382059312E3337330A4E3133EB
:1074700036352058322E3237392059312E333432B6
:107480000A4E313337302058322E333038205931BC
:107490002E3238370A4E313337352058322E3334B6
:1074A000302059312E3235340A4E3133383020589D
:1074B000322E3430372059312E3230310A4E3133AA
:1074C00038352058322E3434312059312E3135366A
:1074D0000A4E313339302058322E34353420593168
:1074E0002E3133310A4E313339352058322E34366D
:1074F000302059312E3130360A4E31343030205858
:10750000322E3436342059312E3130320A4E313455
:1075100030352058322E3437312059312E30333621
:107520000A4E313431302058322E3436362059301C
:107530002E3937310A4E313431352058322E343518
:10754000312059302E3839370A4E313432302058F4
:10755000322E3431352059302E3739310A4E3134FC
:1075600032352058322E3430332059302E373637CA
:107570000A4E313433302058322E333838205930C7
:107580002E3736350A4E313433352058322E3330CB
:10759000362059302E3834310A4E313434302058A8
:1075A000322E3232322059302E3931310A4E3134B6
:1075B00034352058322E3131342059302E39393576
:1075C0000A4E313435302058322E30303220593185
:1075D0002E3037360A4E313435352058312E393079
:1075E000352059312E3133390A4E31343630205856
:1075F000312E3735342059312E3232330A4E313460
:1076000036352058312E3633372059312E3237381F
:107610000A4E313437302058312E35383220593126
:107620002E3330310A4E313437352058312E35352E
:10763000382059312E3331350A4E31343830205804
:10764000312E3436302059312E3335320A4E313412
:1076500038352058312E3339392059312E333630D0
:107660000A4E313439302058312E333338205931D5
:107670002E3335340A4E313439352058312E3238D4
:10768000372059312E3332390A4E313530302058B7
:10769000312E3234382059312E3239340A4E3135B8
:1076A00030352058312E3231372059312E32353491
:1076B0000A4E313531302058312E32313420593193
:1076C0002E3235320A4E313531352058312E313790
:1076D000322059312E3139350A4E31353230205869
:1076E000312E3132382059312E3133390A4E31356D
:1076F00032352058312E3131302059312E31313749
:107700000A4E313533302058302E39353820593033
:107710002E3934310A4E313533352058302E383930
:10772000312059302E3837330A4E31353430205815
:10773000302E3832352059302E3830380A4E313517
:1077400034352058302E3735352059302E373437E0
:107750000A4E313535302058302E363139205930E7
:107760002E3633330A4E313535352058302E3437E6
:10777000372059302E3532360A4E313536302058C2
:10778000302E3437372059302E3532340A4E3135C9
:1077900036352058302E3431312059302E3437369A
:1077A0000A4E313537302058302E3333312059309E
:1077B0002E3435340A4E313537352058302E323795
:1077C000382059302E3432370A4E3135383020586F
:1077D000302E3233312059302E3339370A4E31357D
:1077E00038352058302E3138332059302E33373940
:1077F0000A4E313539302058302E3133352059304A
:107800002E3336350A4E313539352058302E303743
:10781000362059302E3334310A4E31363035204738
:107820003030204633302E300A4E31363130204D44
:107830003035200A4E313631352047393020583026
:10784000205930205A300A4E31363135204D3330F0
:107850000A28456E64206F6620434E432050726FA5
:107860006772616D2900284D53472A2A2A2A204D24
:107870006963726F737465702054657374205B76EE
:10788000315D202A2A2A2A290A47303020473137F9
:1078900020473231204734302047343920473830B0
:1078A000204739300A6730783079307A300A7B22C5
:1078B000316D69223A317D0A7B22326D69223A317B
:1078C0007D0A7B22336D69223A317D0A7B22346D39
:1078D00069223A317D0A6730207831300A7B2231C3
:1078E0006D69223A327D0A78300A7B22316D692235
:1078F0003A347D0A7831300A7B22316D69223A3878
:107900007D0A78300A6730207931300A7B22326D67
:1079100069223A327D0A79300A7B22326D69223A35
:10792000347D0A7931300A7B22326D69223A387D02
:107930000A79300A6730207A31300A7B22336D6948
:10794000223A327D0A7A300A7B22336D69223A3438
:107950007D0A7A31300A7B22336D69223A387D0AFA
:107960007A300A6730206131300A7B22346D692217
:107970003A327D0A61300A7B22346D69223A347DC5
:107980000A6131300A7B22346D69223A387D0A61FE
:10799000300A6D3200284D53472A2A2A2A20436F85
:1079A0006F7264696E617465206F66667365747367
:1079B0002074657374205B76315D202A2A2A2A2977
:1079C0000A673030673137673231673430673439AE
:1079D0006738306739300A6735340A6739327830AA
:1079E00079307A300A663630300A284D53472A2AD1
:1079F0002A2A207465737420473932206F666673B3
:107A00006574732A2A2A2A290A286D7367537465B4
:107A10007020313A204D6F76652066726F6D203090
:107A20002C3020746F2033302C30206D6D20696E27
:107A300020706F7369746976652058206469726577
:107A40006374696F6E290A286D73675374657020BB
:107A5000323A205265736574206F726967696E20CF
:107A6000746F20302E30207573696E67204739326D
:107A7000290A286D73675374657020333A204D6F5F
:107A8000766520746F2032302C302E2053686F754D
:107A90006C64206D6F7665203230206D6D20696ECC
:107AA00020706F7369746976652058206469726507
:107AB0006374696F6E20616E642073746174757392
:107AC000207265706F72742073686F756C642073B8
:107AD000746172742066726F6D20302C30290A2810
:107AE0006D73675374657020343A204D6F7665204E
:107AF000746F20302E3020202053686F756C642006
:107B00006D6F7665203230206D6D20696E206E6558
:107B10006761746976652058206469726563746969
:107B20006F6E20616E64207374617475732072656A
:107B3000706F72742073686F756C642073746172F7
:107B4000742066726F6D2032302C30290A673178CC
:107B500033300A67393278300A67317832300A6751
:107B600031783079300A2473720A67393278300AF2
:107B7000673470302E350A284D53472A2A2A2A2086
:107B80007465737420473535206F6666736574734A
:107B90002A2A2A2A290A286D7367537465702031AE
:107BA0003A2053657420436F6F7264696E61746527
:107BB0002073797374656D2032205B6735355D20E5
:107BC000746F206F6666736574206F662035302C85
:107BD0003530290A286D73675374657020323A2056
:107BE00053656C6563742047353520636F6F72642D
:107BF000696E6174652073797374656D290A286DE7
:107C000073675374657020333A204D6F7665207426
:107C10006F20302C302E20486561642073686F75AA
:107C20006C64206D6F766520646961676F6E616C4E
:107C30006C7920696E202B5820616E64202B5920AE
:107C4000616E6420737461747573207265706F72F5
:107C5000742073686F756C6420737461727420662D
:107C6000726F6D20302C30290A6731304C327032FF
:107C70007835307935300A6735350A6730783079AC
:107C8000300A673470302E350A284D53472A2A2A85
:107C90002A207465737420473533206162736F6CDA
:107CA000757465206F7665727269646573202A2A1F
:107CB0002A2A290A286D73675374657020313A2087
:107CC00052756E20612073717561726520696E2036
:107CD0004735352073797374656D290A286D73678C
:107CE0005374657020323A2052756E206120737192
:107CF0007561726520772F473533206F7665727214
:107D0000696465290A6730783079300A67307832DB
:107D10003079300A67307832307932300A6730781B
:107D2000307932300A6730783079300A6734703011
:107D30002E350A6735336730783079300A67353346
:107D4000673078323079300A6735336730783230CF
:107D50007932300A673533673078307932300A67E4
:107D600035336730783079300A6730783079300AC7
:107D7000673470302E350A284D53472A2A2A2A2084
:107D8000746573742052657475726E20746F206808
:107D90006F6D65202A2A2A2A290A286D7367537471
:107DA000657020313A2052657475726E20746F20B0
:107DB000686F6D65207573696E6720473238290AD0
:107DC000286D73675374657020323A20526573656D
:107DD0007420746F2047353420636F6F7264207392
:107DE000797374656D290A6732380A6735340A6D0C
:107DF000333000284D53472A2A2A2A2054657374A9
:107E0000206163637572616379206F6620736C6FA4
:107E100077206D6F766573205B76315D202A2A2A84
:107E20002A290A6735350A6730783079300A67348D
:107E300070302E350A673470302E350A673178314C
:107E4000306632320A6735340A6730783079300A62
:107E50006D333000284D53472A2A2A2A205465734F
:107E60007420766572792073686F7274206D6F76F6
:107E70006573205B76315D202A2A2A2A290A673019
:107E8000783079300A673470302E350A67317830AF
:107E90002E3166313030300A78300A78302E310A8F
:107EA00078300A78302E310A78300A78302E310A4C
:107EB00078300A78302E310A78300A78302E310A3C
:107EC00078300A78302E310A78300A78302E310A2C
:107ED00078300A78302E310A78300A78302E310A1C
:107EE00078300A78302E310A78300A78302E310A0C
:107EF00078300A78302E310A78300A78302E310AFC
:107F000078300A78302E310A673470302E350A788E
:107F1000300A78302E30310A78300A78302E3031FD
:107F20000A78300A78302E30310A78300A78302ECC
:107F300030310A78300A78302E30310A78300A78B9
:107F4000302E30310A78300A78302E30310A7830CD
:107F50000A78302E30310A78300A78302E30310AE3
:107F600078300A78302E30310A78300A78302E3066
:107F7000310A78300A78302E30310A78300A783079
:107F80002E30310A78300A78302E30310A67307856
:107F90003079300A6D3200284D53472A2A2A2A2088
:107FA000526F746172792041786973204D6F7469E2
:107FB0006F6E2054657374205B76315D202A2A2A07
:107FC0002A290A67303067313767323167343067C2
:107FD00034396738306739300A6730783079307A29
:107FE000306130623063300A6735350A6730783087
:107FF00079300A6633363030300A673061333630D4
:108000000A623336300A633336300A61300A62302E
:108010000A63300A673161313434300A62313434F2
:10802000300A63313434300A61300A62300A633016
:108030000A6731613134343062373230633336307D
:108040000A783079307A306130623063300A6731D3
:108050007836306131343430623732306333363021
:108060000A783079307A306130623063300A6731B3
:1080700078363079353061313434306237323063BC
:108080003336300A783079307A306130623063309C
:108090000A673178363079353078323561313434A9
:1080A0003062373230633336300A783079307A30A4
:1080B0006130623063300A6735340A67307830796E
:1080C000300A6D333000284D53472A2A2A2A204986
:1080D0006E76657273652054696D65204D6F7469A5
:1080E0006F6E2054657374205B76315D202A2A2AD6
:1080F0002A290A6730306731376732316734306791
:1081000034396738306739300A6735350A6730786F
:108110003079300A6739330A66302E30310A6731D8
:108120007831300A7931300A7A31300A6131300AD7
:1081300078300A79300A7A300A61300A673178314A
:10814000307931307A2D31306131300A6730783012
:1081500079307A3061300A66302E310A67327831F0
:1081600030792D31307A2D32306931300A673078EC
:108170003079307A300A6733783130792D31307A7E
:108180002D32306931300A6730783079307A300AF0
:10819000673278323079307A2D32306931300A677F
:1081A00030783079307A300A673378323079306914
:1081B00031300A6730783079307A300A6732783077
:1081C00079307A2D33306931300A6733783079303D
:1081D0007A306931300A6730783079307A300A671E
:1081E00032783079306932302028435720333630A6
:1081F0002064656772656573290A67337830793062
:108200006932302028434357203336302064656775
:1082100072656573290A6739340A6735340A67302D
:10822000783079300A6D3330007B226763223A223E
:1082300067303067313767323167343067343967D8
:108240003830673930227D0A7B226763223A226701
:108250003535227D0A7B226763223A2267307830E7
:108260007930227D0A7B226763223A2266353030DC
:10827000227D0A7B226763223A22284D534773717D
:10828000756172657329227D0A7B226763223A2217
:108290006730783230227D0A7B226763223A227966
:1082A0003230227D0A7B226763223A227830227D97
:1082B0000A7B226763223A227930227D0A7B226779
:1082C00063223A226731783130227D0A7B2267634C
:1082D000223A22793130227D0A7B226763223A22B8
:1082E0007830227D0A7B226763223A227930227D10
:1082F0000A7B226763223A22284D534763697263DF
:108300006C657329227D0A7B226763223A226732D9
:10831000783130792D3130693130227D0A7B226706
:1083200063223A22673078307930227D0A7B2267D7
:1083300063223A226733783130792D313069313018
:10834000227D0A7B226763223A22673078307930B7
:10835000227D0A7B226763223A22673278323079A3
:1083600030693130227D0A7B226763223A226730EE
:1083700078307930227D0A7B226763223A22673384
:108380007832307930693130227D0A7B226763226E
:108390003A22673078307930227D0A7B2267632267
:1083A0003A22673278307930693130227D0A7B2277
:1083B0006763223A22673378307930693130227D21
:1083C0000A7B226763223A22673534227D0A7B22A8
:1083D0006763223A22673078307930227D0A7B2227
:1083E0006763223A226D3330227D00284D53472A9D
:1083F0002A2A2A204D636F64657320746573742084
:108400005B76315D202A2A2A2A290A6735350A67D0
:1084100030783079300A6D330A673470310A6D353F
:108420000A673470310A6D340A673470310A6D3569
:108430000A673470310A6D370A673470310A6D3952
:108440000A673470310A6D380A673470310A6D3941
:108450000A663530300A67307832300A7932300AAD
:108460006D330A78300A6D340A79300A6D350A673F
:10847000317831300A6D370A7931300A6D380A782F
:10848000300A6D390A79300A6732783130792D3106
:10849000306931300A6D330A6730783079300A6DCF
:1084A000340A6733783130792D31306931300A6DD3
:1084B000350A6730783079300A6D370A673278329A
:1084C0003079306931300A6D380A67307830793068
:1084D0000A6D390A673378323079306931300A678A
:1084E00030783079300A6732783079306931300A43
:1084F0006733783079306931300A6735340A67304C
:10850000783079300A6D333000284D53472A2A2AB3
:108510002A2046656564686F6C6420546573742016
:108520005B76315D202A2A2A2A290A284D53472AB8
:108530002A2A2A204D616E75616C6C7920656E74F3
:108540006572202120616E64207E20647572696EE0
:1085500067206D6F76656D656E7420746F2074652D
:108560007374202A2A2A2A290A6735350A6730783F
:108570003079300A673470330A67303067313767D3
:1085800032316734306734396738306739300A66DA
:108590003630300A6730783130307637362E37361D
:1085A000350A783079300A6735340A67307830799F
:1085B000300A6D333000284D53472A2A2A2A204496
:1085C00077656C6C2054657374205B76315D202A6E
:1085D0002A2A2A290A6730306731376732316739EA
:1085E000300A6735350A6730783079300A663530B9
:1085F000300A67307831300A673470310A67307872
:1086000032300A673470310A67307831300A6734A3
:1086100070310A67307830300A673470310A793542
:108620000A6735340A6730783079300A6D330A6763
:108630003470310A67307831307931300A6D350A5B
:10864000673470310A67307832307932300A6D34ED
:108650000A673470310A67307833307933300A6D05
:10866000380A673470310A67307834307934300A28
:108670006D390A673470310A6730783530793530B2
:108680000A6730783079300A6D3330004E31206718
:1086900030306731376732316734306734396738A3
:1086A000306739300A4E3130206730783079300AFF
:1086B0004E323020663530300A4E33302067327803
:1086C0003130792D3130693130202843572032370D
:1086D000302064656772656573290A4E34302067FF
:1086E00030783079300A4E35302067337831307940
:1086F0002D313069313020284343572039302064F0
:10870000656772656573290A4E36302067307830A8
:1087100079300A4E3830206732783230793069311A
:1087200030202843572031383020646567726565F2
:1087300073290A4E3730206730783079300A4E3846
:108740003020673378323079306931302028434324
:1087500057203138302064656772656573290A4E89
:108760003930206730783079300A4E393920463137
:108770003230300A4E31303020673278307930690B
:1087800032302028435720333630206465677265C5
:108790006573290A4E31313020673278307930697B
:1087A0003230202843572033363020616761696EAC
:1087B000290A4E3132302066373030202843686134
:1087C0006E676520666565642072617465207768F0
:1087D000696C6520696E204732206D6F74696F6E19
:1087E000206D6F6465290A4E31333020673278304E
:1087F00079306932302028435720333630203372A5
:10880000642074696D65290A4E31343020673278EE
:1088100030793069323020284357203336302034C5
:1088200074682074696D65290A4E313530206635CB
:1088300030300A4E313630206733783079307A3430
:108840003069323020284343572033363020646566
:1088500067726565732077697468206C696E6561FD
:10886000722074726176656C290A4E313730206748
:1088700033783079307A30693230202843435720BA
:1088800033363020616761696E290A4E31383020F5
:108890006637303020286D73672A2A2A2A43686198
:1088A0006E6765206665656420726174652077680F
:1088B000696C6520696E204733206D6F74696F6E37
:1088C000206D6F64652A2A2A2A290A4E3139302000
:1088D000673378307930693230202843435720336A
:1088E0003630203372642074696D65290A4E323047
:1088F000302067337830793069323020284343574D
:1089000020333630203474682074696D65290A4E2E
:1089100032313020286D73672A2A2A2A47313820BD
:108920004576616C20746573742A2A2A2A290A4EB6
:10893000323230204731205833302E373037205AEA
:1089400035302E37323720463530300A4E3233300C
:108950002047313820473032205836372E373338C9
:10896000205A32332E3631372052323520463235B6
:10897000300A4E323430206738300A4E32353020DB
:108980006730783079307A300A4E323630206D33A5
:108990003000284D53472A2A2A2A205371756172C4
:1089A0006573204D6F74696F6E2054657374205B1E
:1089B00076315D202A2A2A2A290A67303067313722
:1089C0006732316734306734396738306739300A95
:1089D0006730783079300A67307832302028747206
:1089E00061766572736520612032306D6D20737120
:1089F0007561726520696E205820616E6420592966
:108A00000A7932300A78300A79300A6731783130A1
:108A10006635303020286472617720612031306DF6
:108A20006D2073717561726520696E205820616ECA
:108A30006420592061742046353030290A7931305C
:108A40000A78300A79300A67307A32302028747216
:108A500061766572736520612032306D6D207371AF
:108A60007561726520696E205820616E64205A29F4
:108A70000A7832300A7A300A78300A673178323030
:108A80007932307A32306635303020286665656458
:108A900020612032306D6D20646961676F6E616C9A
:108AA00020696E20582C205920616E64205A290AB2
:108AB000783079307A300A7834307934307A34301A
:108AC0002028747261766572736520612034306D80
:108AD0006D206375626520696E20582C20592061D5
:108AE0006E64205A290A78343079307A300A783026
:108AF0007934307A34300A7834307934307A300A44
:108B0000783079307A34300A78307934307A300AF3
:108B100078343079307A34300A783079307A300AE3
:108B20006738300A6730783079300A673078310A30
:108B3000673078300A6D333000284D53472A2A2A8F
:108B40002A20486F6D696E672054657374205B76C8
:108B5000315D202A2A2A2A290A6732382E327830B3
:108B600079307A300A6D333000284D53472A2A2A4B
:108B70002A20536D6F6B652054657374205B7631CA
:108B80005D202A2A2A2A290A4730302047313720F7
:108B9000473231204734302047343920473830209D
:108BA0004739300A6D33673470310A6D3567347078
:108BB000310A6D34673470310A6D33673470310AAD
:108BC0006D35673470310A6D37673470310A6D392D
:108BD000673470310A6D38673470310A6D390A674D
:108BE00030783079307A300A673030207832300A85
:108BF00078300A7932300A79300A7A32300A7A309B
:108C00000A6132300A61300A473030207832302031
:108C1000793230207A3230206132300A47303020C9
:108C20007830207930207A302061300A4730312086
:108C3000663330207832207932207A322061320A4D
:108C40007830207930207A302061300A67307831EE
:108C50000A673078300A6D32002C000A0025730054
:108C6000256C750025312E3066002573002C000A16
:108C70000025733A25730025733A256C750025731A
:108C80003A25312E30660025733A2573005B7476E1
:108C90005D20207465787420766572626F736974E4
:108CA0007925313564205B303D73696C656E742CB9
:108CB000313D766572626F73655D0A0025660A0054
:108CC000256C750A0025640A0025730A0074696E14
:108CD0007967205B25735D206572723A2025733AAF
:108CE000202573200074696E7967205B25735D20F1
:108CF0006F6B3E2000456E64206F6620636F6D6D64
:108D0000616E642066696C650A00FAC9A1C767CA0A
:108D100088CAE7CAE6C7BFCDA1C753CEBFCEEDCC48
:108D2000E6C70000400640061040B800B8BFCDA11D
:108D3000C753CEBFCEEDCCE6C700004006200608E4
:108D400040B800B828D0A1C748CFC4CF73D111CF45
:108D5000A0084006050609010828D0A1C748CFC4CD
:108D6000CFF9CAE6C7B00840060540B03080000021
:108D7000000000F0E0D0C0100100CF673322211FB7
:108D80001B1301016E616E00696E66004E414E4913
:108D90004E495459494E46CDCCCC3D0AD7233C17B9
:108DA000B7D13877CC2B329595E6241FB14F0A0006
:108DB0000020410000C84200401C4620BCBE4CCAF6
:108DC0001B0E5AAEC59D7400407A10F35A00A07273
:108DD0004E18090010A5D4E80000E87648170000F6
:108DE000E40B54020000CA9A3B000000E1F50500C4
:108DF0000080969800000040420F000000A086010D
:108E0000000000102700000000E8030000000064DC
:108E100000000000000A0000000000010000000047
:108E2000002C76D888DC674F0823DFC1DFAE59E11C
:108E3000B1B796E5E3E453C63AE651997696E8E68B
:108E4000C28426EB898C9B62ED407C6FFCEFBC9C5E
:108E50009F40F2BAA56FA5F490055A2AF75C936B70
:108E60006CF9676DC11BFCE0E40D47FEF520E6B52B
:108E700000D0ED902E0300943577050080841E0805
:108E80000000204E0A000000C80C333333330F9823
:108E90006E12831141EF8D2114893BE65516CFFEEA
:108EA000E6DB18D1844B381BF77C1D901DA4BBE476
:108EB00024203284725E228100C9F124ECA1E53DB8
:108EC000270011241FBECFEFCDBFDFE5DEBF00E0DE
:108ED0000CBF13E2A0E0B0E2E0E3FAEC01E00BBF6C
:108EE00002C007900D92A638B107D9F72CE5A6E885
:108EF000B3E201C01D92A237B207E1F70E94CA8017
:108F00000C9416E50C940000FC0160817181828153
:108F100093810E94C1D660933B350895FC01608126
:108F20007181828193810E94C1D660933A35089500
:108F3000AF92BF92CF92DF92EF92FF920F931F9367
:108F4000CF93DF937B018C018EEBC82E84E3D82E68
:108F5000E601AA24A394BC2EBC18F701619171917B
:108F6000819191917F012CEA35EC47E257E30E9411
:108F700050D818164CF4F8014081518162817381F8
:108F80008B2D0E943882A8820C5F1F4F2196F4E33C
:108F9000C43CDF0701F7DF91CF911F910F91FF9044
:108FA000EF90DF90CF90BF90AF900C944382FC0184
:108FB00060817181828193810E94C1D660933C352A
:108FC000613019F481E00E94E77781E00C94087821
:108FD000CF93DF93CDB7DEB76897CDBFDEBFFC017F
:108FE00060817181828193810E94C1D660933D35F9
:108FF00081E0613019F40E94E7770CC00E94087884
:10900000CE01019628E1FC0111922A95E9F7BC01F5
:109010000E94D7476896CDBFDEBFDF91CF910895FC
:109020000F931F93CF93DF93CDB7DEB72D97CDBFAF
:10903000DEBF27E0E8EDF0E28E010F5F1F4FD801A1
:1090400001900D922A95E1F7BC01660F771F680F1A
:10905000791F660F771F660F771F660F771F685699
:109060007A4E45E050E0CE0108960E947EE2688587
:1090700070E0C8010E94ACE2009739F46B8570E0A3
:10908000C8010E94ACE2009711F0801B01C08FEF75
:109090002D96CDBFDEBFDF91CF911F910F91089527
:1090A000EF92FF920F931F93CF93DF938C01F62ED5
:1090B000E72EEC012D96FC016185728583859485F0
:1090C0000E94C1D61F926F93DF93CF930F5E1F4F05
:1090D0001F930F93DF93CF93EF92FF92EEE6FCE5A1
:1090E00081818F9380818F930E944DE3EDB7FEB70E
:1090F0003C96EDBFFEBFDF91CF911F910F91FF9086
:10910000EF9008950F931F93CF93DF93EC01162FE9
:10911000072F8C819D810E94104883305CF58F3F22
:10912000A1F528C09E01235F3F4F9F938F938C85AD
:109130008F938B858F938A858F9389858F933F93A8
:109140002F936196DF93CF933F932F930F931F93AA
:1091500080916F5C8F9380916E5C8F930E944DE342
:109160008DB79EB740968DBF9EBFDF91CF911F9167
:109170000F910895E7E1F4E1659174914FE450E0B7
:1091800086E69FE30E947EE2CDCFE0913435F0E0A9
:10919000EE0FFF1FED5EFB4E659174914FE450E0C2
:1091A00086E69FE30E947EE2BDCF0F931F93CF938D
:1091B000DF93EC01162F072F8C819D810E941048B0
:1091C00083307CF58F3FC1F52CC0AE014F5E5F4F01
:1091D0009E01235F3F4F9F938F938C858F938B8549
:1091E0008F938A858F9389858F935F934F933F9356
:1091F0002F935F934F933F932F930F931F938091E0
:109200006F5C8F9380916E5C8F930E944DE38DB75E
:109210009EB742968DBF9EBFDF91CF911F910F9158
:109220000895E7E1F4E1659174914FE450E086E63A
:109230009FE30E947EE2C9CFE0913435F0E0EE0F6B
:10924000FF1FED5EFB4E659174914FE450E086E6A2
:109250009FE30E947EE2B9CFDF92EF92FF920F93DD
:109260001F93CF93DF93CDB7DEB72897CDBFDEBF77
:109270008B01E42ED52E37E0EFEDF0E2DE01119602
:1092800001900D923A95E1F728870E941048F82E38
:10929000288582E08F1518F0E22FF0E002C0E2E0AE
:1092A000F0E0EE0FFF1FED5EFB4E659174914FE411
:1092B00050E086E69FE30E947EE29F938F93F80141
:1092C00083818F9382818F9381818F9380818F930C
:1092D000E1E0F0E0EC0FFD1FEF0DF11D80811F922A
:1092E0008F93DF92EF9280916F5C8F9380916E5C91
:1092F0008F930E944DE3CDBFDEBF2896CDBFDEBF6A
:10930000DF91CF911F910F91FF90EF90DF90089523
:109310004F925F926F927F92AF92BF92CF92DF9205
:10932000EF92FF920F931F93CF93DF93CEEBD4E393
:1093300003E813E35C018991813009F042C0F80130
:10934000C480D580E680F780408051806280738041
:10935000A3019201C701B6010E94A4D49F772CEA11
:1093600035EC47E257E30E944DD687FD2AC020E046
:1093700034E244E759ECC701B6010E9450D81816F0
:109380005CF4F5012081318142815381C701B6012E
:109390000E9450D8181604F120E034E244E759EC5A
:1093A000C301B2010E9450D818165CF4F501208167
:1093B000318142815381C301B2010E944DD687FDA4
:1093C0000BC00B5C1F4FF4E0AF0EB11C84E3C43C38
:1093D000D80709F0B0CF02C08CED01C080E0DF916A
:1093E000CF911F910F91FF90EF90DF90CF90BF90A2
:1093F000AF907F906F905F904F9008958091BA34B6
:10940000811105C08091B9348093B83429C082306D
:1094100031F487E08093B8348091B93421C083302F
:1094200031F489E08093B8348091B93419C0843024
:1094300031F48AE08093B8348091B93411C08091BE
:10944000BB34813031F485E08093B8348091B934F5
:1094500007C0823019F486E08093B8348091B93423
:10946000863019F08091B83408958BE08093B83439
:1094700008958091B93408958093BB34813059F0B8
:1094800018F0823041F0089589EE94E38093E73438
:109490009093E834089585EB98E58093E7349093B2
:1094A000E8340895FC0184810895845B9F4FFC019A
:1094B00080810895855B9F4FFC0180810895825BC8
:1094C0009F4FFC0180810895815B9F4FFC0180814B
:1094D0000895875B9F4FFC01808108950C94399714
:1094E000CD96FC0160817181828193810895FC0198
:1094F000648308958B5A9F4FFC01608308958F5BAE
:109500009F4FFC014083518362837383089560936E
:10951000E9347093EA348093EB349093EC3480EE2A
:1095200091E20C94F061BF92CF92DF92EF92FF92A2
:109530000F931F93CF93DF93D09036357C010BE5CB
:1095400015E38091353590E0EC01CC0FDD1FC80F9D
:10955000D91FCC0FDD1FCC0FDD1FCC0FDD1FCE526E
:10956000DD4C81E0D816A9F0B881A981CA80BB8002
:109570004091AE35413091F4F80120813181428132
:1095800053816B2F7A2F8C2D9B2D0E94A5D49B018C
:1095900009C020E030E080E090E004C02B2F3A2F9B
:1095A0008C2D9B2DA901BC01F701458F568F678F2C
:1095B00070A3F4E0EF0EF11C0C5F1F4F249685E3BF
:1095C0000337180771F6DF91CF911F910F91FF902C
:1095D000EF90DF90CF90BF900895835B9F4FFC0189
:1095E000608389EE94E30C94934A4F925F926F925A
:1095F0007F928F929F92AF92BF92CF92DF92EF9223
:10960000FF920F931F93CF93DF93CDB7DEB7689789
:10961000CDBFDEBF8C016091AE3570E080E090E0A0
:109620000E94EFD62B013C01F8016081718182819B
:1096300093810E94C1D670E05B01AA0CBB1CA60EF0
:10964000B71EAA0CBB1CAA0CBB1CAA0CBB1CC501D8
:109650008E529D4C5C010BE515E3FE0131964F01E6
:10966000F501C190D190E190F1905F01F801619115
:109670007191819191918F01A30192010E94F2D881
:109680009B01AC01C701B6010E94A5D4F40161930E
:109690007193819391934F01F5E303371F0701F70E
:1096A000CE0101960E941C9789EE94E30E94934A92
:1096B0006896CDBFDEBFDF91CF911F910F91FF90D4
:1096C000EF90DF90CF90BF90AF909F908F907F9062
:1096D0006F905F904F900895895E944369F4E62FF0
:1096E000F0E0EE0FFF1FEE0FFF1FED5BFA4C608105
:1096F0007181828193810895862F0C941197CF9266
:10970000DF92EF92FF920F931F93CF93DF93EC01C1
:1097100084E3C93ED80709F04AC070E0FB01EE0FB0
:10972000FF1FEE0FFF1FED5BFA4CC080D180E2807F
:10973000F38080913635813059F18091353590E054
:10974000FC01EE0FFF1FE80FF91FEE0FFF1FE60FE2
:10975000F71FEE0FFF1FEE0FFF1FEE52FD4C0081B3
:109760001181B281A3812091AE352130B1F4FB018A
:10977000EE0FFF1FEE0FFF1FE55AFA4C20813181DB
:1097800042815381B8018B2F9A2F0E94A5D408C023
:1097900060E070E080E090E003C0B8018B2F9A2F6A
:1097A0009B01AC01C701B6010E94A4D403C0862F5F
:1097B0000E942597C55BDF4F2881211106C023E356
:1097C00033E34BEC51E40E9454D6DF91CF911F91CB
:1097D0000F91FF90EF90DF90CF90089588E1EEEE2B
:1097E000F4E3A3E4B5E301900D928A95E1F780914B
:1097F000323581110CC08091ED34813041F41092EA
:109800002635109227351092283510922935089563
:109810004F925F926F927F928F929F92AF92BF9280
:10982000CF92DF92EF92FF920F931F93CF93DF932C
:10983000CDB7DEB76997CDBFDEBF8091BA34811155
:1098400055C08091DF34813009F050C00E9440C77C
:1098500081114CC01092DF349AEE692E92E3792E7A
:1098600026E3822E912C8E010E5E1F4F36EEA32E24
:1098700030E2B32E33C0F70181917F011F928F93A5
:109880005F924F92BF92AF921F930F930E9418E482
:10989000B80184E493E20E94555F8D839E83F601B4
:1098A00081919191A191B1916F018A879B87AC873A
:1098B000BD87CE0101960E94445CCDBFDEBF9EED08
:1098C000E91690E2F906B9F6E8E16E0E711CFFEFB9
:1098D0008F1A9F0A8CE38816910441F0240189EDC8
:1098E000E82E80E2F82E630188E7C8CF80E0699611
:1098F000CDBFDEBFDF91CF911F910F91FF90EF9011
:10990000DF90CF90BF90AF909F908F907F906F909F
:109910005F904F9008952F923F924F925F926F9277
:109920007F928F929F92AF92BF92CF92DF92EF92EF
:10993000FF920F931F93CF93DF93CDB7DEB7299795
:10994000CDBFDEBF4C015B014090383550903635BD
:10995000209035356090AE35709034356B018EEEC9
:1099600094E3888799875AE7E52E53E3F52E98E12B
:10997000299E100111248401D6016D917D918D9154
:109980009D916D012CEA35EC47E257E30E944DD6DC
:1099900087FD80C0F70180818150823008F07AC055
:1099A00041104CC0F1E05F1609F1E885F985E20D40
:1099B000F31DEC51F2408081898391819D83B281B6
:1099C000A381E1E06E1217C0E885F985E359FF4FE6
:1099D0002081318142815381BC018B2F9A2F0E94BB
:1099E000A5D469837D838E839F8307C019821D82DE
:1099F0001E821F8202C0BE83AF8371100CC023E39E
:109A000033E34BEC51E4D8016D917D918D919C91A4
:109A10000E94F2D805C0F801608171818281938132
:109A200029813D814E815F810E94A5D4A885B98599
:109A30006D937D938D939C9313972CC0A885B985C6
:109A40008D919D910D90BC91A02D89839A83AB83BC
:109A5000BC8371100EC023E333E34BEC51E4F801F7
:109A600060817181828193810E94F2D89B01AC0157
:109A700005C0D8012D913D914D915C9169817A810C
:109A80008B819C810E94A5D4E885F98560837183D0
:109A9000828393838885998504968887998795E33F
:109AA000E90EF11C0C5F1F4FA885B985AA5FB4436E
:109AB00009F062CF6090343570903835F0913635CA
:109AC000F983C09035352091AE352D838CE0A80EFA
:109AD000B11CA9E1B4E3A887B9874AEFE42E44E3B7
:109AE000F42EB8E1CB9E600111248401F50161914F
:109AF0007191819191915F012CEA35EC47E257E336
:109B00000E944DD687FD8CC0A885B9858C9188238D
:109B100009F486C08150823030F4F8012484358401
:109B2000468457843BC0611016C023E333E34BECFB
:109B300051E4D8011C966D917D918D919C911F9758
:109B40000E94F2D820E030E044EB53E40E94F2D8C7
:109B50001B012C010DC020E030E044EB53E4F80180
:109B600064857585868597850E94F2D81B012C0136
:109B70002BED3FE049EC50E4A885B98591966D91B5
:109B80007D918D919C9194970E94F2D89B01AC019C
:109B9000C201B1010E9454D61B012C01711031C0C9
:109BA000B981B130E1F0F701EC0DFD1DEC51F2404F
:109BB000A081B18192808380ED81E130A1F4F70131
:109BC000E359FF4F2081318142815381BD01892DAD
:109BD000982D0E94A5D4DB01982E892E04C0A0E008
:109BE000B0E0912C812CA2019101BD01892D982D0D
:109BF0000E94A5D4D7016D937D938D939C93139769
:109C00000FC0A2019101F70160817181828193816E
:109C10000E94A5D4D7016D937D938D939C93139748
:109C2000E885F985F596E887F987F4E0EF0EF11CF1
:109C30000C5F1F4F88859985885B944309F056CF48
:109C40002996CDBFDEBFDF91CF911F910F91FF907D
:109C5000EF90DF90CF90BF90AF909F908F907F90CC
:109C60006F905F904F903F902F9008958091B63203
:109C70009091B7328F3E924111F08FE50895809117
:109C80006D3690916E368F3E9241B9F780913F3597
:109C9000909140358F3E924181F78091B5359091FA
:109CA000B6358F3E924149F780910D5990910E59EA
:109CB0008F3E924111F78091CA599091CB598F3EB6
:109CC0009241D9F680E00895CF93C82F0E943CA816
:109CD00082E08093B9348C2FCF9108958091BA346B
:109CE000811104C083E08093B93403C085E0809380
:109CF000B93480E00895CF93C82F0E94ADB380E0BF
:109D00000E944EAF8C2F0E943CA886E08093B9340D
:109D10008C2FCF9108958093333580E00895809300
:109D2000343580E008958093383580E008954F926F
:109D30005F926F927F929F92AF92BF92CF92DF928B
:109D4000EF92FF920F931F93CF93DF93C82FB62EFE
:109D50008A01F22ED32F8FEF8C0F863008F082C04D
:109D60006091413670E080E090E00E94EFD62CEAEE
:109D700035EC47E257E30E944DD687FD75C082E07F
:109D8000B81619F0E4E1BE1271C090903435CF2CB2
:109D9000DD2E8C2F90E0EC01CC0FDD1FC80FD91FFA
:109DA000CC0FDD1FCC0FDD1FCC0FDD1FCE52DD4CE5
:109DB000780103E415E3AA24A394F601619171915B
:109DC000819191916F012CEA35EC47E257E30E94B3
:109DD00050D81816DCF5F2E0BF1214C091100CC078
:109DE00023E333E34BEC51E4F7016081718182811D
:109DF00093810E94F2D824C0F70160817181828131
:109E000093811EC0F8014080518062807380911060
:109E10000EC023E333E34BEC51E4F7016081718121
:109E2000828193810E94F2D89B01AC0105C0F701A9
:109E30002081318142815381C301B2010E94A4D4A7
:109E4000688379838A839B83A092DF342496F4E02D
:109E5000EF0EF11C0C5F1F4F85E30B35180709F05F
:109E6000ACCF06C081EA05C08CEA03C08DEA01C010
:109E700080E0DF91CF911F910F91FF90EF90DF90E5
:109E8000CF90BF90AF909F907F906F905F904F90DA
:109E90000895CF93DF93CDB7DEB76897CDBFDEBF10
:109EA00080933535682F70E080E090E00E94EDD619
:109EB00069837A838B839C831D821E821F8218860E
:109EC00019861A861B861C861D861E861F86188A82
:109ED000198A1A8A1B8A1C8A1D8A1E8A1F8A188E52
:109EE000AE014F5F5F4FBA0185EF9AE40E947A831B
:109EF00080E06896CDBFDEBFDF91CF910895CF930C
:109F0000DF93E9EEF4E386E5DF011D928A95E9F738
:109F10008BE5A7EBB5E3ED01982F19929A95E9F738
:109F2000A2E1B6E3ED0119928A95E9F78FEE92E18D
:109F30008093B6329093B73280936D3690936E369D
:109F400080933F35909340358093B5359093B635E7
:109F500080930D5990930E598093CA599093CB5981
:109F6000E093E734F093E8348091CF328093343536
:109F70008091CD320E94494F8091CE32809333350B
:109F80008091D032809337358091D13280933835AB
:109F900081E0809332358093AF3594E09093ED3437
:109FA0001092E0341092E1341092E2348093B9348C
:109FB0008093B8340E94ECADDF91CF910C94BC84B7
:109FC000CF92DF92EF92FF92CF93C82F6A017B016D
:109FD000E82FF0E0DF01AA0FBB1FAA0FBB1FAD5B8C
:109FE000BA4C4D935D936D937C931397EE0FFF1FC7
:109FF000EE0FFF1FE251FB4C40835183628373835A
:10A000008C2F0E942D82B701A6018C2F0E943882CE
:10A01000CF91FF90EF90DF90CF900C9443829F926E
:10A02000AF92BF92CF92DF92EF92FF920F931F9366
:10A03000CF93DF93CDB7DEB76897CDBFDEBF962E47
:10A04000A72EC62ED72E7C0100E010E0B12CF60121
:10A0500061917191819191916F012CEA35EC47E208
:10A0600057E30E9450D81816A4F580913435811119
:10A070000EC023E333E34BEC51E4F70160817181BF
:10A08000828193810E94F2D8AB01BC0105C0F70127
:10A090004081518162817381E1E0F0E0EC0FFD1FAE
:10A0A000E00FF11F4083518362837383C8018A5498
:10A0B0009D4CFC01E357FD4F4083518362837383C2
:10A0C000E555F10940835183628373838B2D0E9490
:10A0D0002D82B3940C5F1F4FF4E0EF0EF11C08319A
:10A0E000110509F0B4CF492D5A2DBE016F5F7F4F86
:10A0F00088E997E40E947A8380E06896CDBFDEBF4E
:10A10000DF91CF911F910F91FF90EF90DF90CF9053
:10A11000BF90AF909F9008954F925F926F927F9201
:10A120008F929F92AF92BF92CF92DF92EF92FF9267
:10A130000F931F93CF93DF93CDB7DEB76897CDBF53
:10A14000DEBF21E02093AE358090353590903435D8
:10A150005B016C0103E415E3882D90E07C01EE0CBB
:10A16000FF1CE80EF91EEE0CFF1CEE0CFF1CEE0CA3
:10A17000FF1CC7018E529D4C7C01F50161917191CC
:10A18000819191915F012CEA35EC47E257E30E94FF
:10A1900050D8181664F5F70120813181428153812E
:10A1A000F80160817181828193810E94A4D42B0186
:10A1B0003C0191100EC023E333E34BEC51E4F60174
:10A1C00060817181828193810E94F2D89B01AC01F0
:10A1D00005C0F6012081318142815381C301B20162
:10A1E0000E94A4D4F801608F718F828F938FF4E066
:10A1F000CF0ED11C0C5F1F4F84E0E80EF11C95E3DD
:10A200000B35190709F0B9CF682D70E080E090E0B8
:10A210000E94EDD669837A838B839C831D821E8284
:10A220001F82188619861A861B861C861D861E8626
:10A230001F86188A198A1A8A1B8A1C8A1D8A1E8AF6
:10A240001F8A188EAE014F5F5F4FBA0185EF9AE407
:10A250000E947A8380E06896CDBFDEBFDF91CF9108
:10A260001F910F91FF90EF90DF90CF90BF90AF9034
:10A270009F908F907F906F905F904F900895CF93B5
:10A28000DF93CDB7DEB76897CDBFDEBF1092AE3596
:10A2900010925B3510925C3510925D3510925E35F0
:10A2A00010925F35109260351092613510926235D0
:10A2B00010926335109264351092653510926635B0
:10A2C00010926735109268351092693510926A3590
:10A2D00010926B3510926C3510926D3510926E3570
:10A2E00010926F3510927035109271351092723550
:10A2F0006091353570E080E090E00E94EDD6698392
:10A300007A838B839C831D821E821F821886198606
:10A310001A861B861C861D861E861F86188A198A29
:10A320001A8A1B8A1C8A1D8A1E8A1F8A188EAE01F1
:10A330004F5F5F4FBA0185EF9AE40E947A8380E015
:10A340006896CDBFDEBFDF91CF910895CF93DF93A5
:10A35000CDB7DEB76897CDBFDEBF1092AE35609146
:10A36000353570E080E090E00E94EDD669837A8315
:10A370008B839C831D821E821F82188619861A86F3
:10A380001B861C861D861E861F86188A198A1A8AB5
:10A390001B8A1C8A1D8A1E8A1F8A188EAE014F5F77
:10A3A0005F4FBA0185EF9AE40E947A8380E0689655
:10A3B000CDBFDEBFDF91CF910895CF93DF93CDB7AF
:10A3C000DEB76897CDBFDEBF81E08093AE35609188
:10A3D000353570E080E090E00E94EDD669837A83A5
:10A3E0008B839C831D821E821F82188619861A8683
:10A3F0001B861C861D861E861F86188A198A1A8A45
:10A400001B8A1C8A1D8A1E8A1F8A188EAE014F5F06
:10A410005F4FBA0185EF9AE40E947A8380E06896E4
:10A42000CDBFDEBFDF91CF910895CF931092ED3471
:10A430000E948B4C8091C032813069F48EEE94E39F
:10A440000E948849C82F882331F00E943CA882E0EE
:10A450008093B93417C089EE94E30E94934A85E053
:10A460008093B9348091BA34811105C081E0809322
:10A47000BA340E944FAC89EE94E30E9446970E9442
:10A48000EE4BC0E08C2FCF91089588E1E3E4F5E333
:10A49000A3E7B5E301900D928A95E1F780E0089576
:10A4A0000F931F93CF93DF93CDB7DEB76A97CDBFDE
:10A4B000DEBF8C0181E08093363589EE94E3698FAD
:10A4C0007A8F0E94934A698D7A8DC8010E94155235
:10A4D0000E94B4828823E1F388E1E0E0F0E2DE014B
:10A4E000119601900D928A95E1F7BE016F5F7F4F43
:10A4F00083E795E30E9415526A96CDBFDEBFDF91D8
:10A50000CF911F910F91089588E1E3E4F5E3ABE863
:10A51000B5E301900D928A95E1F780E008950F93DD
:10A520001F93CF93DF93CDB7DEB76A97CDBFDEBF62
:10A530008C0181E08093363589EE94E3698F7A8FC0
:10A540000E94934A698D7A8DC8010E9415520E941B
:10A55000B4828823E1F388E1E0E0F0E2DE011196C5
:10A5600001900D928A95E1F7BE016F5F7F4F8BE8F6
:10A5700095E30E9415526A96CDBFDEBFDF91CF9161
:10A580001F910F910895FB01DC01809132358111FB
:10A5900011C09B01AD0160E070E080E89FE30E9484
:10A5A00054D6609326357093273580932835909341
:10A5B000293518C080913435811109C023E333E374
:10A5C0004BEC51E4CD010E94F2D8FB0101C0CD015A
:10A5D000AF01BC0140932635509327356093283551
:10A5E0007093293580E008958093323580E0089596
:10A5F0008093373580E0089560932E3570932F3522
:10A6000080933035909331350E94D28380E0089555
:10A610000F931F93CF93DF93EC018B018091323521
:10A62000882399F08091263590912735A09128357F
:10A63000B0912935BC01CD019F772CEA35EC47E27A
:10A6400057E30E944DD687FD30C081E08093ED3402
:10A65000B801CE010E948B4C8091C032813069F4E8
:10A660008EEE94E30E948849C82F882331F00E941F
:10A670003CA882E08093B93419C089EE94E30E942B
:10A68000934A85E08093B9348091BA34811105C032
:10A6900081E08093BA340E944FAC89EE94E30E942B
:10A6A0004697C82F0E94EE4B01C0CEE88C2FDF9159
:10A6B000CF911F910F910895CF93DF93CDB7DEB760
:10A6C0006897CDBFDEBF682F70E080E090E00E9409
:10A6D000EDD669837A838B839C831D821E821F82C1
:10A6E000188619861A861B861C861D861E861F865E
:10A6F000188A198A1A8A1B8A1C8A1D8A1E8A1F8A2E
:10A70000188EAE014F5F5F4FBA0184E897E40E9454
:10A710007A8380E06896CDBFDEBFDF91CF91089548
:10A72000CF93DF93CDB7DEB76897CDBFDEBF609123
:10A730003B3570E080E090E00E94EDD669837A833B
:10A740008B839C831D821E821F82188619861A861F
:10A750001B861C861D861E861F86188A198A1A8AE1
:10A760001B8A1C8A1D8A1E8A1F8A188EAE014F5FA3
:10A770005F4FBA018EE897E40E947A8380E0689682
:10A78000CDBFDEBFDF91CF910895CF93DF93CDB7DB
:10A79000DEB76897CDBFDEBF682F70E080E090E045
:10A7A0000E94EDD669837A838B839C831D821E82EF
:10A7B0001F82188619861A861B861C861D861E8691
:10A7C0001F86188A198A1A8A1B8A1C8A1D8A1E8A61
:10A7D0001F8A188EAE014F5F5F4FBA0187ED97E475
:10A7E0000E947A8380E06896CDBFDEBFDF91CF9173
:10A7F0000895CF93DF93CDB7DEB76897CDBFDEBFA7
:10A80000682F70E080E090E00E94EDD669837A8343
:10A810008B839C831D821E821F82188619861A864E
:10A820001B861C861D861E861F86188A198A1A8A10
:10A830001B8A1C8A1D8A1E8A1F8A188EAE014F5FD2
:10A840005F4FBA0188EE97E40E947A8380E06896B1
:10A85000CDBFDEBFDF91CF910895CF93FC01608122
:10A860007181828193810E94C1D66093B934109224
:10A87000BB3489EE94E38093E7349093E83480917D
:10A88000BA34813011F41092BA341092BC34109260
:10A89000E2340E94FF96C091B934C430C9F40E94DA
:10A8A0003F518091CD320E94494F8091CE328093AA
:10A8B00033358091D1328093383580E00E944EAF9D
:10A8C00080E00E94F95381E080933235C093ED34EB
:10A8D00081E0CF910C9413AB8093AB358093AC3572
:10A8E0008093B43580E008952CEA35EC47E257E3D5
:10A8F0006091593670915A3680915B3690915C36F2
:10A900000E9450D81816B4F48091FE359091FF350E
:10A91000A0910036B0910136BC01CD019F772CEAA1
:10A9200035EC47E257E30E944DD687FF03C01092F3
:10A93000AB3503C081E08093AB3580E00895809310
:10A94000AB358091FE359091FF35A0910036B091E6
:10A9500001368093A3359093A435A093A535B09389
:10A96000A63580E008952CEA35EC47E257E3609184
:10A97000593670915A3680915B3690915C360E94C0
:10A9800050D81816B4F48091FE359091FF35A091FF
:10A990000036B0910136BC01CD019F772CEA35EC31
:10A9A00047E257E30E944DD687FF03C01092AC35B3
:10A9B00003C081E08093AC3580E008958093AC358E
:10A9C0008091FE359091FF35A0910036B09101360F
:10A9D0008093A7359093A835A093A935B093AA3555
:10A9E00080E008952CEA35EC47E257E36091593650
:10A9F00070915A3680915B3690915C360E9450D8A7
:10AA00001816B4F48091FE359091FF35A091003670
:10AA1000B0910136BC01CD019F772CEA35EC47E2BD
:10AA200057E30E944DD687FF03C01092B43503C090
:10AA300081E08093B43580E008958093B4358091AF
:10AA4000FE359091FF35A0910036B091013680938C
:10AA5000B0359093B135A093B235B093B33580E063
:10AA60000895BC018DEE90E20C94136281E0809316
:10AA7000E034089581E08093E134089581E080938B
:10AA8000E23408951F93CF93DF93CDB7DEB7689775
:10AA9000CDBFDEBF0E9439978130C9F10E94EBD251
:10AAA0000E94EFC90E94378380E00E9464AC10E0EE
:10AAB000812F0E941197AB01BC01812F0E94E04FB2
:10AAC0001F5F1630A9F780E090E0A0E4B0E489832E
:10AAD0009A83AB83BC831D821E821F8218861986CF
:10AAE0001A861B861C861D861E861F86188A198A52
:10AAF0001A8A1B8A1C8A1D8A1E8A1F8A188EBE010A
:10AB00006F5F7F4FCB010E942D5480E001C08AE629
:10AB10006896CDBFDEBFDF91CF911F9108958091E0
:10AB2000E0348130A9F42091BB34213079F4809154
:10AB3000BC3481110BC082E08093BB3485EB98E577
:10AB40008093E7349093E8342093BC341092E0343F
:10AB50008091E134813091F48091BB34882331F0CD
:10AB6000823061F49091BC34943051F40E94399752
:10AB7000811104C01092E1340E9442559091BC347E
:10AB80008091E2348130C1F42091E134211114C06C
:10AB90009150933088F01092E23495E09093BC3459
:10ABA0009093B9349091BA34911104C08093BA341F
:10ABB0000E944FAC0E94AB9F80E0089585E0809397
:10ABC000B9348091BA34811105C081E08093BA34E0
:10ABD0000C944FAC0895CF93DF93CDB7DEB7689751
:10ABE000CDBFDEBF8091BA34882311F180E090E0C0
:10ABF000A0E4B0E489839A83AB83BC831D821E8268
:10AC00001F82188619861A861B861C861D861E863C
:10AC10001F86188A198A1A8A1B8A1C8A1D8A1E8A0C
:10AC20001F8A188EBE016F5F7F4FCB010E942D548B
:10AC30006896CDBFDEBFDF91CF910895CF93DF93AC
:10AC4000CDB7DEB76897CDBFDEBF80E090E0A0E46F
:10AC5000B0E489839A83AB83BC831D821E821F82EA
:10AC6000188619861A861B861C861D861E861F86D8
:10AC7000188A198A1A8A1B8A1C8A1D8A1E8A1F8AA8
:10AC8000188EAE014F5F5F4FBA018DE294E50E94CE
:10AC90007A836896CDBFDEBFDF91CF910895CF93C1
:10ACA000DF93CDB7DEB76897CDBFDEBF80E090E021
:10ACB000A0E8B0E489839A83AB83BC831D821E82A3
:10ACC0001F82188619861A861B861C861D861E867C
:10ACD0001F86188A198A1A8A1B8A1C8A1D8A1E8A4C
:10ACE0001F8A188EAE014F5F5F4FBA018DE294E567
:10ACF0000E947A836896CDBFDEBFDF91CF91089521
:10AD0000CF93DF93CDB7DEB72797CDBFDEBF97E0F8
:10AD1000EFEDF0E2DE01119601900D929A95E1F7C8
:10AD2000873050F4E1E0F0E0EC0FFD1FE80FF11D7B
:10AD300087FDFA95808101C080E22796CDBFDEBFF6
:10AD4000DF91CF910895EF92FF920F931F93CF93CE
:10AD5000DF931F92CDB7DEB77C018B01642F70E0CB
:10AD600080E090E049830E94EDD6F7016187728709
:10AD70008387948782E087834981E42FF0E0EE0F98
:10AD8000FF1FE00FF11F659174914FE450E086E6DC
:10AD90009FE30E947EE2BC01C7010F90DF91CF913B
:10ADA0001F910F91FF90EF900C94B561CF93DF93BB
:10ADB000EC010E94FE49482F61E573E1CE01DF916D
:10ADC000CF910C94A3564091B93462E173E10C9495
:10ADD000A3564091BA3469EE72E10C94A3564091A7
:10ADE000BB3465ED72E10C94A3564091BC3467EA24
:10ADF00072E10C94A3564091BD346AE872E10C9460
:10AE0000A356E091E734F091E834E55BFF4F4081D1
:10AE100064EB73E10C94A356E091E734F091E834CD
:10AE2000E45BFF4F408160EC71E10C94A356E0912C
:10AE3000E734F091E834448166E271E10C94A35662
:10AE4000E091E734F091E834E65BFF4F408163EF37
:10AE500070E10C94A356E091E734F091E834E25BA2
:10AE6000FF4F408169EA70E10C94A356E091E7340A
:10AE7000F091E834E15BFF4F408168E670E10C94AB
:10AE8000A356E091E734F091E834E75BFF4F40814F
:10AE900069EF7FE00C94A356CF93DF93EC01E09130
:10AEA000E734F091E834EF5AFF4F608170E080E0C2
:10AEB00090E00E94EDD669877A878B879C8782E035
:10AEC0008F8380E0DF91CF910895CF93DF93EC01E2
:10AED0006091E9347091EA348091EB349091EC34D4
:10AEE0000E94EDD669877A878B879C8782E08F8363
:10AEF00080E0DF91CF910895CF93DF93EC01E09153
:10AF0000E734F091E83460817181828193810E94FD
:10AF1000EDD669877A878B879C8782E08F8380E074
:10AF2000DF91CF910895CF93DF93EC018091BB34F3
:10AF3000811105C019861A861B861C8614C00E94C2
:10AF4000089769877A878B879C8720910059211100
:10AF50000AC025E832E441E25DE30E94F2D8698745
:10AF60007A878B879C878C819D81FC01EE0FFF1F68
:10AF7000E80FF91FEE0FFF1FEE0FFF1FEE0FFF1F71
:10AF8000E156FA4E85919491888784E08F8380E022
:10AF9000DF91CF910895CF93DF93EC012091E734B7
:10AFA0003091E834F901FD9660817181828193814D
:10AFB00069877A878B879C873E96208121110AC0FA
:10AFC00025E832E441E25DE30E94F2D869877A879E
:10AFD0008B879C878C819D81FC01EE0FFF1FE80F02
:10AFE000F91FEE0FFF1FEE0FFF1FEE0FFF1FE156C1
:10AFF000FA4E85919491888784E08F8380E0DF9179
:10B00000CF910895CF93DF93EC018C819D810E94B5
:10B010001048682F8091E7349091E8340E947F4B6C
:10B0200069877A878B879C878C819D81FC01EE0FD5
:10B03000FF1FE80FF91FEE0FFF1FEE0FFF1FEE0FB0
:10B04000FF1FE156FA4E85919491888784E08F83A3
:10B0500080E0DF91CF910895CF93DF93EC018C8155
:10B060009D810E9410482091E7343091E834295E98
:10B07000344369F4E82FF0E0EE0FFF1FEE0FFF1FDF
:10B08000ED5BFA4C608171818281938102C00E94E4
:10B09000119769877A878B879C878C819D81FC01BA
:10B0A000EE0FFF1FE80FF91FEE0FFF1FEE0FFF1F40
:10B0B000EE0FFF1FE156FA4E85919491888784E048
:10B0C0008F8380E0DF91CF910895CF93DF93EC01E0
:10B0D0008C819D810E941048E091E734F091E83422
:10B0E00094E0899FE00DF11D1124458D568D678DEB
:10B0F00070A149875A876B877C878C819D81FC0171
:10B10000EE0FFF1FE80FF91FEE0FFF1FEE0FFF1FDF
:10B11000EE0FFF1FE156FA4E85919491888784E0E7
:10B120008F8380E0DF91CF910895CF93DF93EC017F
:10B130000E94285D69857A858B859C850E94C1D691
:10B14000462F60EE73E1CE01DF91CF910C94A356B0
:10B15000CF93DF93EC018C819D810E941048833056
:10B1600054F48F3FA9F407C0CE010E94D25D80E065
:10B170001CC08DE61AC020E030E040E450E4698550
:10B180007A858B859C850E9450D8181694F3ECCF55
:10B1900020E030E040E050E469857A858B859C852D
:10B1A0000E9450D818162CF3DFCFDF91CF9108956D
:10B1B00095E3899FF0011124E557FC4C6081718172
:10B1C000828193810895CF92DF92EF92FF92CF9385
:10B1D000DF936A017B0125E3829FC00111248A5419
:10B1E0009D4CFC01EB52FF4F40835183628373837C
:10B1F000EC01C352DF4F20E034E244E759E4C701D9
:10B20000B6010E94F2D89B01AC0160E070E080E8DA
:10B210009FE30E9454D6688379838A839B83DF915E
:10B22000CF91FF90EF90DF90CF900895CF92DF9273
:10B23000EF92FF92CF93DF93EC01C984DA84EB8421
:10B24000FC8420E034E244E759E4C701B6010E94DF
:10B2500050D8181664F420E034E244E759E4C701FA
:10B26000B6010E9454D669877A878B879C87CE0166
:10B270000E94CF62C984DA84EB84FC848C819D8136
:10B280000E94104825E3829FC00111248A549D4CDE
:10B29000FC01EB52FF4FC082D182E282F382EC01CB
:10B2A000C352DF4F20E034E244E759E4C701B6015E
:10B2B0000E94F2D89B01AC0160E070E080E89FE35F
:10B2C0000E9454D6688379838A839B8380E0DF91D0
:10B2D000CF91FF90EF90DF90CF900895CF92DF92C3
:10B2E000EF92FF92CF93DF93EC01C984DA84EB8471
:10B2F000FC8420E034E244E759E4C701B6010E942F
:10B3000050D8181664F420E034E244E759E4C70149
:10B31000B6010E9454D669877A878B879C87CE01B5
:10B320000E94CF6280E0DF91CF91FF90EF90DF909D
:10B33000CF90089581E08093E13480E008952CEA75
:10B3400035EC47E257E3FC0161857285838594857E
:10B350000E9450D8181614F40E94E06A80E0089504
:10B360006091E3347091E4348091E5349091E63457
:10B3700008950E94DE5E80E00E94636D80E0089583
:10B380000E94DE5E81E00E94636D80E008950E946D
:10B39000DE5E82E00E94636D80E008950E94DE5EC2
:10B3A00083E00E94636D80E00895CF93DF93EC010A
:10B3B000E091E734F091E834E55BFF4FE081F0E0A5
:10B3C000EE0FFF1FED5EFB4E659174914FE450E070
:10B3D00086E69FE30E947EE2AC0162EE7FE0CE0152
:10B3E000DF91CF910C9496C2CF93DF93EC01E09163
:10B3F000E734F091E834E55BFF4FE081F0E0EE0FD9
:10B40000FF1FED5EFB4E659174914FE450E086E6C0
:10B410009FE30E947EE2AC016AEC7FE0CE01DF9107
:10B42000CF910C9496C2CF93DF93EC0181EF90E221
:10B430000E94EBE3CE010E94D559CE010E94F4593F
:10B4400066EB7FE0CE010E945DC26DE97FE0CE0138
:10B450000E9428C264E87FE0CE010E9428C26BE609
:10B460007FE0CE010E9428C262E57FE0CE010E940B
:10B4700028C269E37FE0CE010E9428C260E27FE03B
:10B48000CE010E9428C267E07FE0CE010E9428C260
:10B490006EEE7EE0CE010E9428C265ED7EE0CE0118
:10B4A0000E9428C26CEB7EE0CE010E9428C263EAB3
:10B4B0007EE0CE010E9428C26AE87EE0CE010E94B2
:10B4C00028C261E77EE0CE010E9428C268E57EE0E6
:10B4D000CE010E945DC280E0DF91CF91089566EBBE
:10B4E0007FE00C945DC26DE97FE00C9428C264E8B3
:10B4F0007FE00C9428C26BE67FE00C9428C262E5E2
:10B500007FE00C9428C269E37FE00C9428C260E2DB
:10B510007FE00C9428C267E07FE00C9428C26EEEB6
:10B520007EE00C9428C265ED7EE00C9428C26CEBA2
:10B530007EE00C9428C263EA7EE00C9428C26AE89C
:10B540007EE00C9428C261E77EE00C9428C268E596
:10B550007EE00C945DC26CED7DE00C945DC26BEA04
:10B560007DE00C945DC266E77DE00C945DC26BE308
:10B570007DE00C945DC267E07DE00C945DC2CF93EA
:10B58000DF93EC01E091E734F091E834E55BFF4FA5
:10B59000E081F0E0EE0FFF1FED5EFB4E65917491D0
:10B5A0004FE450E086E69FE30E947EE2AC0163EE4A
:10B5B0007CE0CE01DF91CF910C9496C2CF93DF93C4
:10B5C000EC01E091E734F091E834E55BFF4FE08176
:10B5D000F0E0EE0FFF1FED5EFB4E659174914FE4BE
:10B5E00050E086E69FE30E947EE2AC0162EC7CE0E4
:10B5F000CE01DF91CF910C9496C265EA7CE00C9469
:10B600003EC2CF93DF93EC01E091E734F091E83450
:10B61000E55BFF4FE081F0E0EE0FFF1FED5EFB4EBC
:10B62000659174914FE450E086E69FE30E947EE2CC
:10B63000AC0166E87CE0CE01DF91CF910C9496C21C
:10B640000F931F93CF93DF938C01FC01618572856B
:10B65000838594850E94C1D6E62FF0E0EE0FFF1F90
:10B66000E052FC4E659174914FE450E086E69FE312
:10B670000E947EE2E8012D969F938F93F8016185E9
:10B680007285838594850E94C1D61F926F93DF9344
:10B69000CF930F5E1F4F1F930F93DF93CF938AE6D5
:10B6A0009CE09F938F93EEE6FCE581818F938081F0
:10B6B0008F930E944DE3EDB7FEB73E96EDBFFEBF00
:10B6C000DF91CF911F910F91089562E47CE00C947B
:10B6D00082486AE17CE00C94824868EF7BE00C943D
:10B6E000824866ED7BE00C94824864EA7BE00C942F
:10B6F000824863E77BE00C9482486AE37BE00C9429
:10B7000082486AE17BE00C94824868ED7AE00C9410
:10B71000504866E97AE00C9450486FE67AE00C9461
:10B72000824869E47AE00C94824868E27AE00C94FA
:10B73000824868E07AE00C9482486BEE79E00C94E1
:10B74000D5486CEC79E00C94D548BC01675F7F4F1D
:10B750002091343542E45EE0FC01848195810C94B3
:10B760002C49BC01675F7F4F21E048E25EE0FC01AD
:10B77000848195810C942C49BC01675F7F4F21E047
:10B780004FE05EE0FC01848195810C942C490F937D
:10B790001F93CF93DF93EC010C811D810E94826483
:10B7A00008171907C4F48C819D81FC01EE0FFF1F5F
:10B7B000E80FF91FEE0FFF1FEE0FFF1FEE0FFF1F29
:10B7C000EC55FA4E25913491CE01F901DF91CF91DC
:10B7D0001F910F91199485E1DF91CF911F910F91E6
:10B7E00008950F931F93CF93DF93EC010C811D817C
:10B7F0000E94826408171907C4F48C819D81FC01A2
:10B80000EE0FFF1FE80FF91FEE0FFF1FEE0FFF1FD8
:10B81000EE0FFF1FEE55FA4E25913491CE01F9013E
:10B82000DF91CF911F910F91199485E1DF91CF9115
:10B830001F910F9108950F931F93CF93DF93EC0106
:10B840000C811D810E94826408171907C4F48C8141
:10B850009D81FC01EE0FFF1FE80FF91FEE0FFF1F88
:10B86000EE0FFF1FEE0FFF1FE056FA4E25913491A9
:10B87000CE01F901DF91CF911F910F911994DF91C2
:10B88000CF911F910F910895CF93DF93EC018C819D
:10B890009D810E9495648823C9F08C819D81FC0163
:10B8A000EE0FFF1FE80FF91FEE0FFF1FEE0FFF1F38
:10B8B000EE0FFF1FE256FA4EE491E1FF05C0CE0104
:10B8C000DF91CF910C94538180E001C085E1DF913D
:10B8D000CF9108950F931F93CF93DF93EC0181E0F5
:10B8E0000E948F4E1C821D8280E090E08E010F5ED0
:10B8F0001F4F47C08C819D819C01220F331FF9018E
:10B90000E80FF91FEE0FFF1FEE0FFF1FEE0FFF1FD7
:10B91000E256FA4EE491E0FF2EC0280F391F220FA5
:10B92000331F220F331F220F331F28553A4EF901C0
:10B93000459155916591749149875A876B877C87AA
:10B94000BC01660F771F680F791F660F771F660FA0
:10B95000771F660F771F68567A4E45E050E0C801A2
:10B960000E947EE2CE010E94C75BCE010E94445C31
:10B970002C813D8101C09C012F5F3F4F2C833D8373
:10B98000C9010E9485648111B5CF81E00E94C2A8DF
:10B99000DF91CF911F910F910C94AAA8CF93DF93C1
:10B9A000EC012CEA35EC47E257E369857A858B8513
:10B9B0009C850E944DD687FF05C0CE01DF91CF91B7
:10B9C0000C94F579CE010E946A5C82E08F8340E09E
:10B9D00050E060E87FE349875A876B877C8780E087
:10B9E000DF91CF9108958091243C9091253C8F3E2A
:10B9F000924111F08AE508958091663C9091673CF0
:10BA00008F3E9241B9F78091FA369091FB368F3E86
:10BA1000924181F780911C3A90911D3A8F3E92415C
:10BA200049F780911E3A90911F3A8F3E924111F74B
:10BA30008091223C9091233C8F3E9241D9F6809197
:10BA4000B53F8111D7CF0895FC01178289E608958B
:10BA5000CF93DF93EC018C819D81FC01EE0FFF1FE2
:10BA6000E80FF91FEE0FFF1FEE0FFF1FEE0FFF1F76
:10BA7000EA55FA4EA591B4916C9170E080E090E0A7
:10BA80000E94EDD669877A878B879C8782E08F83B7
:10BA900080E0DF91CF910895CF93DF93EC018C810B
:10BAA0009D81FC01EE0FFF1FE80FF91FEE0FFF1F36
:10BAB000EE0FFF1FEE0FFF1FEA55FA4EA591B4914E
:10BAC0006D917D918D919C910E94EDD669877A87C9
:10BAD0008B879C8782E08F8380E0DF91CF910895F0
:10BAE000CF93DF93DC0114968D919C911597FC0107
:10BAF000EE0FFF1FE80FF91FEE0FFF1FEE0FFF1FE6
:10BB0000EE0FFF1FEA55FA4EC591D4914881598135
:10BB10006A817B8119964D935D936D937C931C97FD
:10BB200083E017968C9380E0DF91CF910895CF93B7
:10BB3000DF93DC0114968D919C911597FC01EE0F1B
:10BB4000FF1FE80FF91FEE0FFF1FEE0FFF1FEE0F95
:10BB5000FF1FEA55FA4EC591D491488159816A81F7
:10BB60007B8119964D935D936D937C931C97FC019B
:10BB7000EE0FFF1FE80FF91FEE0FFF1FEE0FFF1F65
:10BB8000EE0FFF1FE156FA4E8591949118968C9313
:10BB9000189784E017968C9380E0DF91CF910895F9
:10BBA00088E608950F931F93CF93DF93EC018C8168
:10BBB0009D81FC01EE0FFF1FE80FF91FEE0FFF1F25
:10BBC000EE0FFF1FEE0FFF1FEA55FA4E059114917D
:10BBD00069857A858B859C850E94C1D6F801608332
:10BBE00082E08F8380E0DF91CF911F910F910895C4
:10BBF000CF93DF93EC0169857A858B859C850E94C4
:10BC0000C1D66230B0F48C819D81FC01EE0FFF1F24
:10BC1000E80FF91FEE0FFF1FEE0FFF1FEE0FFF1FC4
:10BC2000EA55FA4EA591B4916C9382E08F8380E03F
:10BC300001C08EE6DF91CF910895CF93DF93EC01A1
:10BC400069857A858B859C850E94C1D66330B0F466
:10BC50008C819D81FC01EE0FFF1FE80FF91FEE0F95
:10BC6000FF1FEE0FFF1FEE0FFF1FEA55FA4EA591C3
:10BC7000B4916C9382E08F8380E001C08EE6DF9107
:10BC8000CF910895CF93DF93EC0169857A858B85F9
:10BC90009C850E94C1D66430B0F48C819D81FC01EA
:10BCA000EE0FFF1FE80FF91FEE0FFF1FEE0FFF1F34
:10BCB000EE0FFF1FEA55FA4EA591B4916C9382E006
:10BCC0008F8380E001C08EE6DF91CF9108950F93BE
:10BCD0001F93CF93DF93EC018C819D81FC01EE0FCC
:10BCE000FF1FE80FF91FEE0FFF1FEE0FFF1FEE0FF4
:10BCF000FF1FEA55FA4E0591149169857A858B8567
:10BD00009C850E94C1D6F8016083718382E08F8395
:10BD100080E0DF91CF911F910F9108950F931F93B2
:10BD2000CF93DF93EC018C819D81FC01EE0FFF1F0F
:10BD3000E80FF91FEE0FFF1FEE0FFF1FEE0FFF1FA3
:10BD4000EA55FA4E0591149169857A858B859C8513
:10BD50000E94C1D6F801608371838283938382E05D
:10BD60008F8380E0DF91CF911F910F910895CF9342
:10BD7000DF93DC0114968D919C911597FC01EE0FD9
:10BD8000FF1FE80FF91FEE0FFF1FEE0FFF1FEE0F53
:10BD9000FF1FEA55FA4EC591D49119964D915D91C8
:10BDA0006D917C911C97488359836A837B8383E0E0
:10BDB00017968C9380E0DF91CF910895CF93DF9316
:10BDC000DC0114968D919C911597FC01EE0FFF1FDD
:10BDD000E80FF91FEE0FFF1FEE0FFF1FEE0FFF1F03
:10BDE000EA55FA4EC591D49119964D915D916D9198
:10BDF0007C911C97488359836A837B83FC01EE0FF7
:10BE0000FF1FE80FF91FEE0FFF1FEE0FFF1FEE0FD2
:10BE1000FF1FE156FA4E8591949118968C931897CE
:10BE200084E017968C9380E0DF91CF9108951F9363
:10BE3000CF93DF93EC018091863C8823D1F01DE104
:10BE40000A80DB81C02D209711F480E013C08F8120
:10BE50008F3FD9F3811104C0CE010E94F15B06C06F
:10BE6000CE010E94C75BCE010E94445C115041F795
:10BE7000ECCF85E6DF91CF911F910895CF93DF93AB
:10BE8000EC01BC018FEF90E20E94B7E2892B41F0F8
:10BE9000BE0182E091E20E94B7E221E0892B09F421
:10BEA00020E0822FDF91CF9108950F931F93CF93BE
:10BEB000DF93CDB7DEB72997CDBFDEBF8B0144E05E
:10BEC00050E0BC01CE0101960E94D7E246E050E06E
:10BED000B801CE0101960E94C7E20E948264181642
:10BEE00019060CF03FC07981AA81BB811C810D81AC
:10BEF00028E935E140E050E0F9016491671327C07B
:10BF00003196E491E11103C0A11121C029C0EA13C7
:10BF10001EC0F9013296E491E11103C0B11117C0BE
:10BF20001FC0EB1314C0F9013396E491E11103C073
:10BF300011110DC015C0E1130AC0F9013496E49146
:10BF4000E11103C0011103C00BC0E01749F04F5FBE
:10BF50005F4F285E3F4F4817590709F0CDCF02C009
:10BF6000CA0102C08FEF9FEF2996CDBFDEBFDF91E0
:10BF7000CF911F910F910895CF93DF93FC012189F9
:10BF8000222371F1EC016196BE0186E091E20E94EC
:10BF9000B7E2892B39F1BE018FEF90E20E94B7E240
:10BFA000892B11F1BE0189E091E20E94B7E2892B51
:10BFB000D9F0BE018DEE90E20E94B7E2892BB1F07C
:10BFC000BE018CE091E20E94B7E2892B79F0BE01BC
:10BFD00080EE91E20E94B7E2892B51F485E009C01E
:10BFE00080E007C082E005C083E003C084E001C0B8
:10BFF00081E0DF91CF910895FC018FEF8783148258
:10C00000158211861286138614861086118A15866B
:10C01000178A108EA081B181109711F416820DC07D
:10C0200017968C911797873029F416968C918F5F0D
:10C03000868303C016968C918683CF010895EF9274
:10C04000FF920F931F93CF93DF93EC010C811D811F
:10C050000E948264081719070CF06FC00C811D81C3
:10C06000CE010E94FC5F0C831D837E0181E1E80EFE
:10C07000F11CB801660F771F600F711F660F771FE5
:10C08000660F771F660F771F68567A4EC7010E94AA
:10C090005FE28E01035F1F4F2C813D81B901660F66
:10C0A000771F620F731F660F771F660F771F660F6C
:10C0B000771F6C567A4EC8010E945FE28D858823F7
:10C0C00011F18C819D81FC01EE0FFF1FE80FF91F1C
:10C0D000EE0FFF1FEE0FFF1FEE0FFF1FE256FA4E8F
:10C0E000E491E2FF02C01D8610C0F801019000201B
:10C0F000E9F7BF01601B710B605F7F4F6C0F7D1F05
:10C10000C7010E94C0E28C819D81FC01EE0FFF1FE0
:10C11000E80FF91FEE0FFF1FEE0FFF1FEE0FFF1FBF
:10C12000EE55FA4E25913491CE01F901DF91CF9170
:10C130001F910F91FF90EF901994DF91CF911F9174
:10C140000F91FF90EF9008958F929F92AF92BF92C0
:10C15000CF92DF92EF92FF920F931F93CF93DF93D3
:10C1600000D01F92CDB7DEB76C015C0181E1A80E53
:10C17000B11C87E0F6018783A4E9EA2EA5E1FA2E37
:10C1800000E010E01DC0B701CE0101960E945FE201
:10C19000BE016F5F7F4FC5010E94B7E2892B59F442
:10C1A0004601F9E18F0E911CF601058F168FC4012F
:10C1B0000E941F6064010F5F1F4FF8E1EF0EF11C3A
:10C1C000C8010E9485648111DECF2496CDBFDEBFF9
:10C1D000DF91CF911F910F91FF90EF90DF90CF9063
:10C1E000BF90AF909F908F900895CF93DF93109260
:10C1F000203A1092213AA3EEB6E3ECEFF6E391E099
:10C200008FEFA083B18379965B96ED93FC935C9757
:10C210005D961D921C925E97EF016397988322961C
:10C220001882219788832A96188259962AE3EC313E
:10C23000F20739F71092053A1092063A1092FC363E
:10C240001092FD361092023787E08093033782E721
:10C2500090E080930D3790930E3785E197E3DF915F
:10C26000CF9108950F931F93CF93DF930E94F560B2
:10C27000EC018FEE92E18093243C9093253C8093D7
:10C28000663C9093673C8093FA369093FB3680939C
:10C290001C3A90931D3A80931E3A90931F3A8093D4
:10C2A000223C9093233C81E00E948F4E1C821D8291
:10C2B000CE010E942A8120916E3C30916F3C4091CA
:10C2C000703C5091713C69857A858B859C850E9474
:10C2D0004DD6882339F0CE01DF91CF911F910F9178
:10C2E0000C946A5C0E94AFA81C821D8280E090E0E2
:10C2F0008E010F5E1F4F2FC06C817D819B01220F2D
:10C30000331FF901E60FF71FEE0FFF1FEE0FFF1FA0
:10C31000EE0FFF1FE256FA4EE491E0FF17C0620FE6
:10C32000731F660F771F660F771F660F771F68569C
:10C330007A4E45E050E0C8010E947EE2CE010E94A4
:10C340002A81CE010E94C75B6C817D816F5F7F4F28
:10C350006C837D83CB010E9485648111CDCFDF91F9
:10C36000CF911F910F910C94C2A8EF92FF920F935F
:10C370001F93CF93DF938C012091203A3091213A83
:10C38000EB0109900020E9F72197C61BD70BAE01FE
:10C39000420F531F41305240D8F4F901EE5DF54C85
:10C3A0007F01AE014F5F5F4FCF010E9498E2409145
:10C3B000203A5091213A4F5F5F4F4C0F5D1F4093E1
:10C3C000203A5093213AF801E78AF08E80E001C0CC
:10C3D0008DE0DF91CF911F910F91FF90EF90089525
:10C3E000CF93DF932EE1C5E1D7E33F813F3F59F083
:10C3F0000A80DB81C02D209719F480E090E010C006
:10C40000215099F7FACFBC0184E493E20E94555F72
:10C410008C839D83019689F3CE010E941F60CE011B
:10C42000DF91CF910895EF92FF920F931F93CF93D7
:10C43000DF938B012EE1C5E1D7E33F813F3F59F008
:10C440000A80DB81C02D209719F480E090E01DC0A8
:10C45000215099F7FACF7E0121E1E20EF11C45E06F
:10C4600050E0BC01C7010E94D7E2B801CE010E9492
:10C47000B5618111EACFB70184E493E20E94555F70
:10C480008C839D8385E08F83CE01DF91CF911F91B7
:10C490000F91FF90EF9008952091863C213021F478
:10C4A0002091623F213029F4BC018DEE90E20C9482
:10C4B000136280E090E008959091863C913019F4E9
:10C4C000642F0C94A67F0C94A8C1CF93DF93EC014A
:10C4D00080917332811103C00E94E3D202C00E9496
:10C4E000F1C9682F70E080E090E00E94EDD6698786
:10C4F0007A878B879C8782E08F8380E0DF91CF9162
:10C5000008950F931F93CF93DF93CDB7DEB7C05835
:10C51000D109CDBFDEBFFC0161857285838594851D
:10C520000E94C1D68FEF860F863030F080E491E212
:10C530000E944C628EE62AC060936E3281E0809346
:10C540006F32E62FF0E0EE0FFF1FE15AFA4E6591D1
:10C5500074914FE450E086E69FE30E947EE29F9351
:10C560008F9386E294E19F938F938E010F5F1F4F0D
:10C570001F930F930E9441E4C8010E944C620F90E8
:10C580000F900F900F900F900F9080E0C058DF4FEA
:10C59000CDBFDEBFDF91CF911F910F9108950F9313
:10C5A0001F93CF93DF93EC0189EE94E30E945A4AE4
:10C5B000882329F009851A858B859C8511C023E382
:10C5C00033E34BEC51E469857A858B859C850E9429
:10C5D000F2D88B01AB01BC0149875A876B877C87F6
:10C5E0002C813D81F901EE0FFF1FE20FF31FEE0FCB
:10C5F000FF1FEE0FFF1FEE0FFF1FEA55FA4EA5912A
:10C60000B491A801BC014D935D936D937C931397F6
:10C61000F901EE0FFF1FE20FF31FEE0FFF1FEE0FEA
:10C62000FF1FEE0FFF1FE156FA4E85919491888708
:10C6300084E08F8380E0DF91CF911F910F91089567
:10C6400060E375E10C943EC26CE075E10C943EC26F
:10C6500060ED74E10C943EC26CE974E10C943EC24E
:10C660006FE474E10C943EC21F93CF93DF93EC010F
:10C6700010E08881882301F10E94F56045E050E0D8
:10C68000BE0186E297E30E94D7E266E277E384E4A4
:10C6900093E20E94555F8093193790931A3785E192
:10C6A00097E30E941F6042E063E080E00E945C62CA
:10C6B0001F5F26961D31E9F684E0DF91CF911F912F
:10C6C0000895CF93DF93CDB7DEB7EC97CDBFDEBF34
:10C6D0008CE3E8E1F0E2DE01119601900D928A957B
:10C6E000E1F7CE0101960E943463EC96CDBFDEBF28
:10C6F000DF91CF910895CF93DF93CDB7DEB7AA979F
:10C70000CDBFDEBF8AE2E4E5F0E2DE0111960190E2
:10C710000D928A95E1F7CE0101960E943463AA96A4
:10C72000CDBFDEBFDF91CF910895CF93DF93CDB71B
:10C73000DEB76E97CDBFDEBF8EE1EEE7F0E2DE0141
:10C74000119601900D928A95E1F7CE0101960E9413
:10C7500034636E96CDBFDEBFDF91CF910895CF9346
:10C76000DF93EC0143E759E763E770E0498B5A8BAD
:10C770006B8B7C8B0E94A46042E063E080E00E94AF
:10C780005C62CE010E949563CE010E947B6320E72C
:10C7900031E340E0298B3A8B4B8BCE010E94A460A1
:10C7A00042E063E080E00E945C62CE01DF91CF91C5
:10C7B0000C946163CF92DF92EF92FF92FC01C184EF
:10C7C000D284E384F48420E030E040E85FE3C701F2
:10C7D000B6010E9450D81816FCF0C701B6010E949D
:10C7E000C1D660937032C701B6019F772CEA35EC51
:10C7F00047E257E30E9450D818163CF460E470E01A
:10C8000080E00E94CFC780E008C060E870E080E070
:10C810000E94CFC780E001C08EE6FF90EF90DF90CE
:10C82000CF900895CF92DF92EF92FF92FC01C184E6
:10C83000D284E384F48420E030E040E050E4C70197
:10C84000B6010E9450D81816FCF0C701B6010E942C
:10C85000C1D660937232C701B6019F772CEA35ECDE
:10C8600047E257E30E9450D818163CF464E070E0A9
:10C8700080E00E94CFC780E008C068E070E080E000
:10C880000E94CFC780E001C08EE6FF90EF90DF905E
:10C89000CF900895CF92DF92EF92FF92FC01C18476
:10C8A000D284E384F48420E030E040E85FE3C70111
:10C8B000B6010E9450D81816FCF0C701B6010E94BC
:10C8C000C1D660937132C701B6019F772CEA35EC6F
:10C8D00047E257E30E9450D818163CF460E170E03C
:10C8E00080E00E94CFC780E008C060E270E080E096
:10C8F0000E94CFC780E001C08EE6FF90EF90DF90EE
:10C90000CF9008958DE891E0089521E0843491401E
:10C9100008F020E0822F08959C012056314081E0EC
:10C920002932310508F080E0089521E081369140F8
:10C9300008F020E0822F0895CF92DF92EF92FF92CD
:10C94000CF93DF93EC01C984DA84EB84FC84A701E4
:10C950009601C701B6010E9413DA81113CC0E89428
:10C96000F7F82FEF3FEF4FE75FE7C701B6010E94EF
:10C9700013DA81110AC02FEF3FEF4FE75FE7C701DE
:10C98000B6010E944DD6181634F18C819D81FC01B0
:10C99000EE0FFF1FE80FF91FEE0FFF1FEE0FFF1F37
:10C9A000EE0FFF1FE256FA4EE491E3FF14C089EE4A
:10C9B00094E30E945A4A81110EC025E832E441E214
:10C9C0005DE369857A858B859C850E94F2D86987AD
:10C9D0007A878B879C87DF91CF91FF90EF90DF90D4
:10C9E000CF90089580916F32882349F010926F3272
:10C9F00060916E3280E00E94D7C780E0089583E0A6
:10CA00000895CF93DF93E091A83CF091A93C04C036
:10CA1000E093A83CF093A93CEF018191982F9D7F72
:10CA20009032B1F38930A1F34FE750E0BE018CEAB8
:10CA30009EE30E94D7E21092A43C1092A53C109273
:10CA4000A63C1092A73C6881611105C08091863C8C
:10CA500081116DC039C0613221F4DF91CF910C9406
:10CA60003655653221F4DF91CF910C943A556E37EB
:10CA700021F4DF91CF910C943E556F3379F4FE0190
:10CA800001900020E9F73197EC1BFD0B329780F005
:10CA90002196C093A83CD093A93C49C06B3741F480
:10CAA00081E08093863CCE01DF91CF910C944B7A4C
:10CAB00070E080E791E20E94ACE2892B59F010927D
:10CAC000863CCE010E9400BE6CEA7EE3DF91CF91EE
:10CAD0000C9440BF8091863C811109C0CE010E9418
:10CAE0002D706CEA7EE3DF91CF910C9440BF0E94E1
:10CAF000F560EC0127E633E640E0298B3A8B4B8B5F
:10CB00006091A83C7091A93C0E94B56185E08F833B
:10CB10008091A83C9091A93C0E942D7042E060E079
:10CB20000E945C6280E0DF91CF910C9413ABDF91A7
:10CB3000CF910895FF920F931F93CF93DF931F928E
:10CB40001F92CDB7DEB7F82EE8E6FCE326EC32E024
:10CB5000DF01C9011D920197E9F72FEE32E1208331
:10CB6000318320932C3F30932D3F06E616E22CEDC7
:10CB700033E400936E3C10936F3C2093703C3093F1
:10CB8000713C0CEE11E528E73FE30093723C1093F3
:10CB9000733C2093743C3093753C00E010E020EA35
:10CBA00030E40093763C1093773C2093783C3093AC
:10CBB000793C00E010E020E83FE300937A3C1093DA
:10CBC0007B3C20937C3C30937D3C83E08093873C8E
:10CBD0008F2D4A8369830E94E7C76981862F0E944F
:10CBE000F2C74A81842F0E94FDC7F0926D32F09205
:10CBF0006B320F900F90DF91CF911F910F91FF90AB
:10CC00000895CF93DF931F921F92CDB7DEB780E6D2
:10CC1000F82E01E010E00E94B3788230E1F30E9428
:10CC2000BA788230C1F30E94394A863009F0D9C0FF
:10CC30000E94CAC580908D3C90908E3CA0908F3C05
:10CC4000B090903C86169706A806B90620F70E9479
:10CC5000CAC56C597F4F8F4F9F4F60938D3C709327
:10CC60008E3C80938F3C9093903C0E942978D3CF48
:10CC70000E94DBBC882329F08CEC0E947B4E823022
:10CC800051F20E948F55823031F20E94059E82300F
:10CC900011F20E94F35C8093B63F81112EC0809107
:10CCA000683C9091693C8F3E924109F0AAC0809106
:10CCB0002C3F90912D3F8F3E924109F0A2C097C02A
:10CCC0000E94FF818093B63F811117C00E9468B314
:10CCD0008093B63F811111C00E94F86F8093B63FD8
:10CCE00081110BC00E94F6C68093B63F811105C02A
:10CCF0000E943CB4823031F48ECF0E947B4E823051
:10CD0000B9F789CF0E9445AB823009F484CF0E94E5
:10CD1000B1AC823009F47FCF0E946DAD823009F44E
:10CD20007ACF09831A836AEA7CE3CE0101960E94D6
:10CD30000CC88093A83C9093A93C8F3F2FEF92079B
:10CD400039F48DE00E94644E823009F464CF04C04F
:10CD5000892B11F00E9401650E94648C823009F4D5
:10CD60005ACF0E942F6B823009F455CF0E94EE6D8E
:10CD7000823009F450CF0E94D36F823009F449CF3A
:10CD80000E94084C823009F444CF0E94B48284305F
:10CD9000F0F53FCF8091873C843038F484E0809375
:10CDA000873C0E943A550E94B4A883E090E08983B2
:10CDB0009A836AEA7CE3CE0101960E940CC88093B4
:10CDC000A83C9093A93C8F3F2FEF920721F48DE070
:10CDD0000E94644E1ECF892B09F41BCF0E9401656F
:10CDE00018CF0E94394A823009F44BCF41CF1092BC
:10CDF000B63F0E94364E8093B63F882309F460CF39
:10CE00007CCFF092B63F80E60E947B4E78CF809137
:10CE1000E0299091E1290E9457D1682F70E080E0CD
:10CE200090E00E94EFD620E030E048E451E40E9418
:10CE300050D887FFEECE0E94F264823009F0AACF6C
:10CE4000E8CE80916D3280936B32089580936B327F
:10CE5000089580936C320895CF93C82F80918F23CB
:10CE6000882379F040E050E0BA018C2F0E94E04F17
:10CE7000EC2FFF27E7FDF095E254FB4C81E0808327
:10CE80000AC06C2F85EB98E50E947F4BAB01BC017B
:10CE90008C2F0E94E04F4091B6235091B7236091B0
:10CEA000B8237091B9238C2F0E94E35885EF98E640
:10CEB000809390239093912382E0CF910895CF9215
:10CEC000DF92EF92FF920F931F93CF93DF93CDB733
:10CED000DEB7E097CDBFDEBF98E17E01A9E1EA0EA3
:10CEE000F11CF701A92F1192AA95E9F7FE013196DD
:10CEF0006F0111929A95E9F7F60194E08902E00D2D
:10CF0000F11D1124408F518F628F738F80E090E06C
:10CF1000A0E8BFE380839183A283B3830093263587
:10CF20001093273520932835309329350E94378375
:10CF30000E943E55B601C7010E9408538093B63F38
:10CF4000811101C082E0E096CDBFDEBFDF91CF91BD
:10CF50001F910F91FF90EF90DF90CF9008950F9366
:10CF60001F93E0918923FF27E7FDF095ED56FD4CD7
:10CF70009381913099F400919A2310919B232091F1
:10CF80009C2330919D234091A2235091A323609133
:10CF9000A4237091A5230E945F671DC0E0918A239E
:10CFA000FF27E7FDF095ED56FD4C9381913099F404
:10CFB00000919A2310919B2320919C2330919D23D3
:10CFC0004091A2235091A3236091A4237091A523A3
:10CFD00070580E945F6785EF97E680939023909347
:10CFE000912382E01F910F9108950F931F93CF9388
:10CFF000C82F85E3C802F0011124E157FC4C4081A1
:10D000005181628173818C2F0E94E35800919A2391
:10D0100010919B2320919C2330919D234091962336
:10D020005091972360919823709199238C2F0E949F
:10D030005F6784E898E6809390239093912382E041
:10D04000CF911F910F9108950F931F9300919A23F1
:10D0500010919B2320919C2330919D234091A623E6
:10D060005091A7236091A8237091A9230E945F6724
:10D070008CE297E6809390239093912382E01F9116
:10D080000F9108950E9437838091AF230E94494FEA
:10D090008091AE230E948F4E8091B0230E94934EC8
:10D0A0008091B1230E94F4528091B2239091B323D6
:10D0B000A091B423B091B523809326359093273562
:10D0C000A0932835B093293564E089EE94E30E945B
:10D0D000774A0E94EB551092BA3480E00895CF93BE
:10D0E000C82F4091B6235091B7236091B823709117
:10D0F000B9230E94E3588C2F0E94426880E00E946E
:10D1000013AB80EFCF9108950F931F93E091892384
:10D11000FF27E7FDF095ED56FD4C9381913039F0F6
:10D120008FE698E6809390239093912318C0009106
:10D130009E2310919F232091A0233091A123409101
:10D14000A2235091A3236091A4237091A5230E9450
:10D150005F6784E298E6809390239093912382E026
:10D160001F910F910895FF920F931F93CF93DF9319
:10D17000CDB7DEB7C058D109CDBFDEBFF82E0E94B3
:10D18000F5608EEFF81205C085E791E20E944C62CF
:10D1900019C08F2D0E9480561F928F932CEC3AE37A
:10D1A0003F932F938E010F5F1F4F1F930F930E948A
:10D1B00041E4C8010E944C620F900F900F900F90B5
:10D1C0000F900F9042E062E080EF0E945C628F2D32
:10D1D0000E94426880EFC058DF4FCDBFDEBFDF91B5
:10D1E000CF911F910F91FF9008954F925F926F9290
:10D1F0007F929F92AF92BF92CF92DF92EF92FF9277
:10D200000F931F93CF93DF938F3F09F045C02CEA14
:10D2100035EC47E257E360912136709122368091D8
:10D220002336909124360E9450D818160CF469C108
:10D230002CEA35EC47E257E36091193670911A36C3
:10D2400080911B3690911C360E9450D818160CF411
:10D250005DC12CEA35EC47E257E360911D367091D1
:10D260001E3680911F36909120360E9450D8181695
:10D270000CF455C12CEA35EC47E257E360912536B2
:10D280007091263680912736909128360E9450D88A
:10D2900018160CF43FC171C18230A1F52CEA35ECAF
:10D2A00047E257E36091193670911A3680911B3628
:10D2B00090911C360E9450D818160CF427C12CEA05
:10D2C00035EC47E257E360911D3670911E36809130
:10D2D0001F36909120360E9450D818160CF41FC1AA
:10D2E0002CEA35EC47E257E36091253670912636FB
:10D2F00080912736909128360E9450D818160CF449
:10D3000009C131C18823D9F2813051F32CC17E018A
:10D310008DEEE80EF11CF70180819181A281B3812D
:10D32000BC01CD019F772CEA35EC47E257E30E9420
:10D330004DD687FD46C06E01F1EFCF0ED11CF60130
:10D34000408051806280738020E030E0A901C301F9
:10D35000B2010E944DD687FD34C0FE01EF52FF4F4F
:10D360002081318142815381349760817181828132
:10D3700093810E94A4D49B01AC015F77C301B201E9
:10D380000E94A5D42B013C019F772CEA35EC47E2A3
:10D3900057E30E944DD687FD14C0AB2CAA0C8A2DF2
:10D3A0000E94D5BC80938723992493949A0C892D4D
:10D3B0000E94D5BC8093882320918723822780FDFB
:10D3C00002C08B2DDBC0B0928623F8018081918151
:10D3D000A281B381BF7780939A2390939B23A093DC
:10D3E0009C23B0939D23F701408151816281738119
:10D3F0007F7740939E2350939F236093A023709345
:10D40000A12320FF2DC0A092892390928A2377FA2E
:10D41000709477F87094409296235092972360927C
:10D42000982370929923F60180819181A281B38122
:10D430008093A2239093A323A093A423B093A52326
:10D44000CB50DF4F88819981AA81BB818093A6232D
:10D450009093A723A093A823B093A9238A2D2AC031
:10D4600090928923A0928A234092962350929723E8
:10D470006092982370929923F60180819181A28114
:10D48000B381B0588093A2239093A323A093A423A5
:10D49000B093A523CB50DF4F88819981AA81BB81AE
:10D4A000B0588093A6239093A723A093A823B0936A
:10D4B000A923892D0E94D5BC8D7F813039F085EF5D
:10D4C00098E6809390239093912369C080918A235A
:10D4D0000E94D5BC811103C08FEF80938A238B2DCE
:10D4E0000E94D8586093B6237093B7238093B823D3
:10D4F0009093B9238FEA97E680939023909391239A
:10D500004EC082E090E032E0B32E0DC080E090E0AB
:10D51000B12C09C083E090E023E0B22E04C081E08A
:10D5200090E0BB24B394FC01E254FB4C108225E351
:10D53000289FE001299FD00D1124CA54DD4C8E0193
:10D5400007511F4FF80180819181A281B381BC01F5
:10D55000CD019F772CEA35EC47E257E30E944DD688
:10D5600087FFD5CE2ECF81E08093BD3482E498E64C
:10D57000809390239093912312C08EEFDF91CF91EF
:10D580001F910F91FF90EF90DF90CF90BF90AF90E1
:10D590009F907F906F905F904F900C94B36882E063
:10D5A000DF91CF911F910F91FF90EF90DF90CF907F
:10D5B000BF90AF909F907F906F905F904F90089535
:10D5C000CF93DF93C7EED4E3888199810E945A4AB2
:10D5D0008093AE23888199810E94554A8093AF231E
:10D5E000888199810E94644A8093B02388819981BF
:10D5F0000E94694A8093B123888199810E94704A70
:10D600006093B2237093B3238093B4239093B52394
:10D6100081E00E948F4E81E00E94934E80E00E9444
:10D62000494F81E00E94F45281E080938F238FEF75
:10D630008093862385EF98E680939023909391239F
:10D6400083E08093BA341092BD3480E0DF91CF91B3
:10D6500008950E94E06A10928F2380E008958091DF
:10D66000BA34833059F40E946E4A813049F0E09117
:10D670009023F091912380918623199483E008955B
:10D6800082E008958AE49BE68093CB239093CC2399
:10D6900082E008952F923F924F925F926F927F9215
:10D6A0008F929F92AF92BF92CF92DF92EF92FF92B2
:10D6B0000F931F93CF93DF93CDB7DEB7CA54D10931
:10D6C000CDBFDEBF98E19E01275E3F4F29AB3AAB4D
:10D6D000D901E92F1D92EA95E9F72851310919017D
:10D6E000D9011D929A95E9F724E08202F0011124F4
:10D6F0002B96EEAFFFAF2B97E20DF31D80E090E08D
:10D70000A0E8BFE380839183A283B383C090C32347
:10D71000D090C423E090C523F090C6234090BF234F
:10D720005090C0236090C1237090C2238090BB238F
:10D730009090BC23A090BD23B090BE23A50194017E
:10D74000C301B2010E944DD618165CF080E090E053
:10D75000A0E8BFE329968CAF9DAFAEAFBFAF2997CE
:10D760000AC080E090E0A0E8BFEB29968CAF9DAFA7
:10D77000AEAFBFAF2997A3019201C501B4010E94CA
:10D78000A4D40E94BCD69B0177FF04C02227332774
:10D79000261B370BB901882777FD8095982F0E94AB
:10D7A000EFD625966CAF7DAF8EAF9FAF2597C09219
:10D7B0002635D0922735E0922835F09229350E94FF
:10D7C00037830E943E5520E030E040E050E425964B
:10D7D0006CAD7DAD8EAD9FAD25970E9450D81816CB
:10D7E0006CF08091C7239091C823A091C923B09178
:10D7F000CA238BAF9CAFADAFBEAFDBC02AE037ED25
:10D8000043E25CE325966CAD7DAD8EAD9FAD259773
:10D810000E9450D818162CF709E110E08AE0882EF3
:10D8200087ED982E83E2A82E8CE3B82E412C512C44
:10D8300032012B96AEADBFAD2B97A20DB31D5896FE
:10D840002196AEAFBFAF21974BAA5CAA6DAA7EAA64
:10D850008FAA98AEA9AEBAAE29962CAD3DAD4EAD0D
:10D860005FAD29976FA978AD89AD9AAD0E94F2D8C6
:10D870009B01AC016091BF237091C0238091C123B3
:10D880009091C2230E94A5D42196EEADFFAD2197C1
:10D890006083718382839383C0922635D09227352B
:10D8A000E0922835F0922935B101CE0149960E94C7
:10D8B00008538093B63F8111AAC020E030E040E8D1
:10D8C0005FE36BA97CA98DA99EA90E94A5D46BAB2F
:10D8D0007CAB8DAB9EAB20E030E048EC51E40E9485
:10D8E00054D69B01AC0160E070E080E291E40E94BC
:10D8F00055D92B013C018091C7239091C823A09159
:10D90000C923B091CA238BAF9CAFADAFBEAFC0905F
:10D91000C323D090C423E090C523F090C623A70171
:10D920009601BC01CD010E94A4D44B015C0120E012
:10D9300030E040E251E4C301B2010E9454D69B01A1
:10D94000AC01C501B4010E94F2D89B01AC01C70132
:10D95000B6010E94A5D46B017C012BA93CA94DA95D
:10D960005EA9CA01B9010E94A5D420E030E048ECCC
:10D9700051E40E9454D69B01AC016FA978AD89ADEA
:10D980009AAD0E94A5D46FAB78AF89AF9AAF9B01D7
:10D99000AC0125966CAD7DAD8EAD9FAD25970E94F7
:10D9A00050D8181634F4015011090115110509F069
:10D9B00053CF8BAD9CADADADBEAD8093263590936E
:10D9C0002735A0932835B09329352B96EEADFFADC2
:10D9D0002B97E20DF31D8091BB239091BC23A09166
:10D9E000BD23B091BE23808F918FA28FB38FB101E1
:10D9F000CE0149960E9408538093B63F811107C01B
:10DA00008EE19DE68093CB239093CC2382E0C65B8E
:10DA1000DF4FCDBFDEBFDF91CF911F910F91FF9000
:10DA2000EF90DF90CF90BF90AF909F908F907F90BE
:10DA30006F905F904F903F902F900895CF93DF931A
:10DA40001F92CDB7DEB789830E9437834091D523DB
:10DA50005091D6236091D7237091D82389810E9459
:10DA6000E3588091D2230E94494F8091D1230E9494
:10DA70008F4E8091D3230E94934E8091D4230E9495
:10DA8000F4528091CD239091CE23A091CF23B091D9
:10DA9000D0238093263590932735A0932835B093D3
:10DAA000293564E089EE94E30E94774A0E94EB55A1
:10DAB0001092BA3481EA91E20E94EBE380E00F9089
:10DAC000DF91CF9108950F931F93CF93C82F07EE47
:10DAD00014E3F801808191810E945A4A8093D123F6
:10DAE000F801808191810E94554A8093D223F801E8
:10DAF000808191810E94644A8093D323F8018081C0
:10DB000091810E94694A8093D423F8018081918198
:10DB10000E94704A6093CD237093CE238093CF23CD
:10DB20009093D0238C2F0E94D8586093D523709364
:10DB3000D6238093D7239093D82381E00E948F4EE1
:10DB400080E00E94934E80E00E94494F81E00E9455
:10DB5000F45240E050E060E271E44093C3235093FC
:10DB6000C4236093C5237093C62385E3C89FF00147
:10DB70001124E158FC4C40815181628173814093B2
:10DB8000C7235093C8236093C9237093CA236C2F73
:10DB900085EB98E50E946C4B6093BF237093C02384
:10DBA0008093C1239093C2230E94B0596093BB23FA
:10DBB0007093BC238093BD239093BE23C093BA235C
:10DBC00082E49BE68093CB239093CC2384E08093E4
:10DBD000BA3480E0CF911F910F9108958091BA34AB
:10DBE000843059F40E946E4A813049F0E091CB2391
:10DBF000F091CC238091BA23199483E0089582E0B8
:10DC00000895E091DB23F0E0ED56FD4C83818823FD
:10DC100041F08CE19EE68093D9239093DA2382E051
:10DC2000089568E274E280E194E20E9408538093D0
:10DC3000B63F882371F308951F93CF93DF93E0914C
:10DC4000DB23F0E0ED56FD4C81E09381913009F04B
:10DC500080E08093C434C5ECD4E310E0812F0E94AF
:10DC60002597AB01BC01812F0E94E04F612F80916D
:10DC7000E7349091E8340E946C4B699379938993CF
:10DC800099931F5F163051F78BEA91E20E944B7A0D
:10DC900088E89EE68093D9239093DA2382E0DF918F
:10DCA000CF911F9108951F93CF93DF930E943783E5
:10DCB0008091DC2380939332E091DB23F0E080912C
:10DCC000DD23ED56FD4C83870E94F2BCC0EED3E20B
:10DCD00010E04991599169917991812F0E94E358FF
:10DCE0001F5F1630B1F78091DF230E94494F80916A
:10DCF000DE230E94934E64E089EE94E30E94774A0B
:10DD00000E94EB551092BA34DF91CF911F91089584
:10DD10000E94536E80E008950F931F93CF93DF937B
:10DD2000CDB7DEB7C058D109CDBFDEBF182F0E94D6
:10DD3000F5601E3F29F488EB91E20E944C6219C005
:10DD4000812F0E9480561F928F938AEF9AE39F93B0
:10DD50008F938E010F5F1F4F1F930F930E9441E41B
:10DD6000C8010E944C620F900F900F900F900F907F
:10DD70000F9042E062E08AEF0E945C620E94536E64
:10DD80008AEFC058DF4FCDBFDEBFDF91CF911F912B
:10DD90000F910895FF920F931F93CF93DF931092EB
:10DDA000C43482E08093BA3400EE13E2CFE8D3E3C8
:10DDB000F12C8F2D0E94D858F801619371938193B3
:10DDC00091938F01488159816A817B818F2D0E94B7
:10DDD000E3586F2D8091E7349091E8340E946C4BAA
:10DDE000F801648B758B868B978BF394E596F6E040
:10DDF000FF12DFCF60E174E288EF93E20E94CDC2B0
:10DE00002AE43CE042E85EE30E944DD687FF03C06F
:10DE10008EEF0E948C6EC4E0D4E213E06991799198
:10DE2000899199912C893D894E895F890E94A4D45A
:10DE30009F772CEA35EC47E257E30E9450D818163A
:10DE40001CF4812F0E948C6E1F5F163039F784E01E
:10DE50008093DB238091A2328093DD2381E0809345
:10DE6000A232809193328093DC23109293320E94ED
:10DE7000F2BC8091E7349091E8340E94554A809337
:10DE8000DF238091E7349091E8340E94644A8093C4
:10DE9000DE2380E00E94934E80E00E94494F80E0A4
:10DEA0000E944EAF81E09EE68093D9239093DA23BF
:10DEB00082E0DF91CF911F910F91FF9008950F9312
:10DEC0001F93CF93DF938C01EB0180913235882330
:10DED00099F08091263590912735A0912835B09101
:10DEE0002935BC01CD019F772CEA35EC47E257E399
:10DEF0000E944DD687FD4FC088819981AA81BB8140
:10DF0000BC01CD019F772CEA35EC47E257E30E9434
:10DF100050D81816F4F48C819D81AE81BF81BC016C
:10DF2000CD019F772CEA35EC47E257E30E9450D8A9
:10DF300018167CF488859985AA85BB85BC01CD011E
:10DF40009F772CEA35EC47E257E30E9450D8181629
:10DF500024F188E1F801A0E1B4E201900D928A95E4
:10DF6000E1F788E1FE01A8E2B4E201900D928A9502
:10DF7000E1F788E1E5ECF4E3DF011D928A95E9F72A
:10DF800082E08093C4348AEC9EE68093D9239093F8
:10DF9000DA2380E003C08EE801C086E8DF91CF91EC
:10DFA0001F910F9108958091BA34823021F08091B1
:10DFB000C434823049F40E946E4A813039F0E091D5
:10DFC000D923F091DA23199483E0089582E008952B
:10DFD000EEE2FFE380E2DF011D928A95E9F78FEE22
:10DFE00092E180934C3F90934D3F808391830895BD
:10DFF00080914C3F90914D3F8F3E924111F08CE5C6
:10E00000089580912E3F90912F3F8F3E9241B9F716
:10E0100080E00895CF93DF93C82FCB01BA010E940F
:10E02000A1D927E0C29FE0011124C25DD04C0E941B
:10E03000BCD66D837E838F839887DF91CF910895BF
:10E0400097E0899FF0011124E25DF04C65817681B3
:10E05000878190850E94EFD608952F923F924F922C
:10E060005F926F927F928F929F92AF92BF92CF9268
:10E07000DF92EF92FF920F931F93CF93DF93CDB771
:10E08000DEB72797CDBFDEBF8C011B828091B934EC
:10E09000823009F43FC7D801DC90D11068C780E016
:10E0A0005E01B3E0AB0EB11C3DC0F5018081811172
:10E0B00008C0D72CD7011C925E01B3E0AB0EB11C97
:10E0C00053C7883239F4D72CF7011082FFEFAF1A0B
:10E0D000BF0A4AC78B33B9F3C82ED12CC6010E94A0
:10E0E00033E2892B39F4B60182EE91E20E94ACE270
:10E0F000892B51F047018FEF881A980AC6010E94B8
:10E1000057E2D7018C937401BFEFAB1ABB0AF7013A
:10E1100080818111CACFD72CD8018C915E01B3E0E8
:10E12000AB0EB11CF8011CC08E32E1F090E0C0973C
:10E130000A9790F08181803391F4828190E0C097BA
:10E140000A9760F4DF01119611968C9111978D93C7
:10E150008111FACF808104C0818101C080E33196B2
:10E160008111E2CFF501C080C11007C067C0D501A1
:10E170001196CC90BFEFAB1ABB0A75018C2C912C79
:10E18000C4010E9447E2892B91F7EBE7CE122EC023
:10E19000D50111968C9190E00E944FE28437910551
:10E1A00029F5F501828190E00E944FE289369105C0
:10E1B000E9F4D50113968C9190E00E944FE28436E9
:10E1C0009105A1F4C50105960E943DE1AA2797FD9E
:10E1D000A095BA2F8093A43C9093A53CA093A63C15
:10E1E000B093A73CF501C0808C2C912CC4010E94F7
:10E1F0004FE28D369105A1F4D50111968C9190E0F6
:10E200000E944FE28337910559F4F501828190E035
:10E210000E944FE28736910519F4F501339602C04A
:10E22000FE013396CC2061F08C2DD701893209F4A0
:10E230001C9211968C918111F9CF02C0FE01339688
:10E240008FE2D81609F468C68081882319F0CF01BF
:10E250000E94315580E1EEE4FFE3DF011D928A95D3
:10E26000E9F78BE5E2E1F6E3DF01982F1D929A953D
:10E27000E9F7E7EBF5E3DF011D928A95E9F789EE0F
:10E2800094E30E94524A8093B835812C912C80E807
:10E29000A82E8FE3B82E5524539492E0492E24E003
:10E2A000322E23C4C701B6010E94C1D6862F90E04A
:10E2B0008F35910508F034C6FC01EC50FF4F0C94EB
:10E2C00098DE1092B8355092133680914F3F8F5F91
:10E2D00080934F3F0AC45092B835509213368091C4
:10E2E0004F3F8F5F80934F3F00C44092B8355092AC
:10E2F000133680914F3F8F5F80934F3FF6C383E08B
:10E300008093B8355092133680914F3F8F5F809342
:10E310004F3FEBC38DE08093B73550921236E5C383
:10E3200088E0B2C01092E735509242368091503F5B
:10E330008F5F8093503FD9C35092E7355092423659
:10E340008091503F8F5F8093503FCFC34092E7351D
:10E35000509242368091503F8F5F8093503FC5C3AB
:10E360001092E835509243368091533F8F5F8093EF
:10E37000533FBBC35092E835509243368091533F90
:10E380008F5F8093533FB1C3C701B6010E940CDA7F
:10E390006C837D838E839F8320E030E040E251E4F4
:10E3A000C701B6010E94F2D86B017C0120E030E089
:10E3B00040E251E46C817D818E819F810E94F2D880
:10E3C0009B01AC01C701B6010E94A4D40E94C1D632
:10E3D000623001F128F4662341F0613089F0A0C574
:10E3E0006330E9F0643001F19BC5B5E0B093B73517
:10E3F0005092123680914E3F8F5F80934E3F75C38F
:10E400003092B7356093123680914E3F8F5F809384
:10E410004E3F6BC35092B7355092123666C340924E
:10E42000B7355092123661C383E08093B73550926E
:10E4300012365BC3C701B6010E940CDA6C837D8380
:10E440008E839F8320E030E040E251E4C701B601B3
:10E450000E94F2D86B017C0120E030E040E251E400
:10E460006C817D818E819F810E94F2D89B01AC01DD
:10E47000C701B6010E94A4D40E94C1D6662319F038
:10E48000613061F04DC587E08093B7355092123608
:10E4900080914E3F8F5F80934E3F27C3E6E0E0932D
:10E4A000B7356093123680914E3F8F5F80934E3F19
:10E4B0001CC3C701B6010E940CDA6C837D838E8376
:10E4C0009F8320E030E040E251E4C701B6010E94A2
:10E4D000F2D86B017C0120E030E040E251E46C8135
:10E4E0007D818E819F810E94F2D89B01AC01C70182
:10E4F000B6010E94A4D40E94C1D6623009F010C5B2
:10E500008EE08093B73550921236EFC25092EA35C2
:10E5100050924536EAC25092E93550924436809185
:10E52000573F8F5F8093573FE0C24092E93550924A
:10E5300044368091573F8F5F8093573FD6C283E028
:10E5400016C03092E935509244368091573F8F5F24
:10E550008093573FCAC2F5E0F093E93550924436B4
:10E560008091573F8F5F8093573FBFC286E0809373
:10E57000E935509244368091573F8F5F8093573FE3
:10E58000B4C2C701B6010E940CDA6C837D838E830E
:10E590009F8320E030E040E251E4C701B6010E94D1
:10E5A000F2D86B017C0120E030E040E251E46C8164
:10E5B0007D818E819F810E94F2D89B01AC01C701B1
:10E5C000B6010E94A4D40E94C1D6662319F061301E
:10E5D00059F0A6C41092EC35509247368091583FBE
:10E5E0008F5F8093583F81C26093EC3560934736CC
:10E5F0008091583F8F5F8093583F77C24092EC35AF
:10E60000509247368091583F8F5F8093583F6DC23C
:10E610003092B8355092133680914F3F8F5F809380
:10E620004F3F63C2C701B6010E940CDA6C837D8341
:10E630008E839F8320E030E040E251E4C701B601C1
:10E640000E94F2D86B017C0120E030E040E251E40E
:10E650006C817D818E819F810E94F2D89B01AC01EB
:10E66000C701B6010E94A4D40E94C1D6662319F046
:10E67000613059F055C41092ED3550924836809172
:10E68000513F8F5F8093513F30C21092EE356093BF
:10E6900049368091513F8F5F8093513F26C2C70119
:10E6A000B6010E940CDA6C837D838E839F8320E009
:10E6B00030E040E251E4C701B6010E94F2D86B019C
:10E6C0007C0120E030E040E251E46C817D818E816C
:10E6D0009F810E94F2D89B01AC01C701B6010E9444
:10E6E000A4D40E94C1D6662319F0613059F018C431
:10E6F0005092ED35509248368091513F8F5F809314
:10E70000513FF3C16093EE35609349368091513F9C
:10E710008F5F8093513FE9C1C701B6010E940CDAB7
:10E720006C837D838E839F8320E030E040E251E460
:10E73000C701B6010E94F2D86B017C0120E030E0F5
:10E7400040E251E46C817D818E819F810E94F2D8EC
:10E750009B01AC01C701B6010E94A4D40E94C1D69E
:10E76000613089F028F06230A1F06330C1F0D8C385
:10E7700099E09093B7355092123680914E3F8F5F5B
:10E7800080934E3FB2C1AAE0A093B7356093123692
:10E79000ACC1BBE0B093B73550921236A6C1ECE0E5
:10E7A000E093B73550921236A0C11092E2355092E4
:10E7B0003D368091523F8F5F8093523F96C1509279
:10E7C000E23550923D368091523F8F5F8093523FA9
:10E7D0008CC1C701B6010E94C1D6862F90E08D334F
:10E7E000910508F09BC3FC01ED5AFE4F0C9498DE96
:10E7F0001092B935509214368091593F8F5F8093B3
:10E80000593F73C15092B935509214368091593F97
:10E810008F5F8093593F69C15092F43550924F36C3
:10E8200080915B3F8F5F80935B3F5FC14092F43587
:10E8300050924F3680915B3F8F5F80935B3F55C115
:10E840001092F43550924F3680915B3F8F5F8093EA
:10E850005B3F4BC15092F13550924C3646C15092BD
:10E86000F23550924D3680915C3F8F5F80935C3FD4
:10E870003CC15092F33550924E3680915C3F8F5F91
:10E8800080935C3F32C11092F33550924E368091A6
:10E890005C3F8F5F80935C3F28C15092E53550927A
:10E8A000403680915D3F8F5F80935D3F1EC1109227
:10E8B000E5355092403680915D3F8F5F80935D3F9C
:10E8C00014C15092E33550923E3680915D3F8F5F88
:10E8D00080935D3F0AC15092FD3550925836809129
:10E8E0005D3F8F5F80935D3F00C1C701B6010E940D
:10E8F0000CDA0E94C1D66093F03550924B36F5C0C9
:10E90000C092D635D092D735E092D835F092D9352D
:10E910008092313690923236A0923336B0923436AD
:10E92000E4C0C092FE35D092FF35E0920036F092FE
:10E9300001368092593690925A36A0925B36B09248
:10E940005C36D3C0C092F535D092F635E092F735FB
:10E95000F092F8358092503690925136A09252360D
:10E96000B0925336C2C0C092BE35D092BF35E0924D
:10E97000C035F092C1358092193690921A36A09225
:10E980001B36B0921C36B1C0C092C235D092C3358E
:10E99000E092C435F092C53580921D3690921E36B5
:10E9A000A0921F36B0922036A0C0C092C635D09239
:10E9B000C735E092C835F092C935809221369092E1
:10E9C0002236A0922336B09224368FC0C092CA3528
:10E9D000D092CB35E092CC35F092CD358092253671
:10E9E00090922636A0922736B09228367EC0C092EA
:10E9F000CE35D092CF35E092D035F092D13580929D
:10EA0000293690922A36A0922B36B0922C366DC0C1
:10EA1000C092D235D092D335E092D435F092D5352C
:10EA200080922D3690922E36A0922F36B0923036AC
:10EA30005CC0C0920636D0920736E0920836F0925B
:10EA400009368092613690926236A0926336B09217
:10EA500064364BC0C0920A36D0920B36E0920C3628
:10EA6000F0920D368092653690926636A0926736A7
:10EA7000B09268363AC0C0920E36D0920F36E0920D
:10EA80001036F09211368092693690926A36A092D2
:10EA90006B36B0926C3629C0C0920236D0920336E3
:10EAA000E0920436F092053680925D3690925E36A2
:10EAB000A0925F36B092603618C0C701B6010E94BE
:10EAC000C1D66093BA357093BB358093BC359093B3
:10EAD000BD3581E090E0A0E0B0E0809315369093E2
:10EAE0001636A0931736B0931836D8012C902220F2
:10EAF00009F424C2822D90E00E943EE2892B09F4A1
:10EB00002FC23801BFEF6B1A7B0AF8018181803375
:10EB100049F48281883531F40E5F1F4FC12CD12C0E
:10EB2000760100C2BE016F5F7F4FC3010E94B8DE55
:10EB30006B017C0109811A816016710609F0F2C12E
:10EB400011C28091E2350E94F452182F01C010E0EA
:10EB500060913136709132368091333690913436EF
:10EB60000E94C1D6662359F06091D6357091D73591
:10EB70008091D8359091D9350E94C352182F609159
:10EB800035367091363680913736909138360E94FE
:10EB9000C1D6662371F06091DA357091DB358091D2
:10EBA000DC359091DD350E94C1D6862F0E949F549E
:10EBB000182F6091393670913A3680913B3690919A
:10EBC0003C360E94C1D6662371F06091DE357091AB
:10EBD000DF358091E0359091E1350E94C1D6862FD6
:10EBE0000E94DE54182F60915036709151368091FA
:10EBF0005236909153360E94C1D6662359F06091E7
:10EC0000F5357091F6358091F7359091F8350E9481
:10EC100082AF182F609154367091553680915636D8
:10EC2000909157360E94C1D6662371F06091F935F4
:10EC30007091FA358091FB359091FC350E94C1D6D8
:10EC4000862F0E941D55182F80914B36882329F05E
:10EC50008091F0350E945C53182F80914C368823A8
:10EC600029F08091F1350E949053182F80914F36F2
:10EC7000882329F08091F4350E944EAF182F80919F
:10EC80004D36882329F08091F2350E94C553182F04
:10EC900080914E36882329F08091F3350E94F953F4
:10ECA000182F80913E36882329F08091E3350E9409
:10ECB0007454182F80913F36882329F08091E435D1
:10ECC0000E94B354182F80915836882329F08091E0
:10ECD000FD350E94F254182F80914036882329F088
:10ECE0008091E5350E946C54182F8091B7358D3096
:10ECF00029F0809142368823A9F00FC06091FE353B
:10ED00007091FF3580910036909101360E94FC523F
:10ED10008093B63F882369F32FC18091E7350E9425
:10ED20008B4E182F80914336882329F08091E83547
:10ED30000E948F4E182F80914436882329F08091AD
:10ED4000E9350E94494F182F80914736882329F0D2
:10ED50008091EC350E94F852182F80914836882314
:10ED600029F08091ED350E94934E182F4091B735D0
:10ED700050E04F30510508F0B6C0FA01E057FE4FA1
:10ED80000C9498DE0E944552182FADC069E176E3DD
:10ED90008EEB95E30E945052182FA5C00E9484521A
:10EDA000182FA1C069E176E38EEB95E30E948F52A4
:10EDB000182F99C00E94E06A182F95C069E176E388
:10EDC0008EEB95E30E940F50182F8DC00E94296B87
:10EDD000182F89C069E176E38EEB95E30E945F6F9F
:10EDE000182F81C06091FE357091FF3580910036FB
:10EDF000909101360E94C1D6862F29E136E34EEB71
:10EE000055E36091E6350E94974E182F6CC069E17A
:10EE100076E38EEB95E30E948C50182F64C00E941D
:10EE20003F51182F60C00E94A651182F5CC00E944D
:10EE3000DD51182F58C06091EA3589EE94E30E94A5
:10EE4000ED4A8091B835843038F48230D8F4882384
:10EE500049F0813079F047C0843009F044C0809394
:10EE6000ED3441C069E176E38EEB95E30E941552E3
:10EE7000182F39C069E176E38EEB95E30E940853C1
:10EE8000182F31C0A0900E36B0900F36C0901036BB
:10EE9000D0901136E0900A36F0900B3600910C3687
:10EEA00010910D3620910636309107364091083684
:10EEB000509109368F93809105368F938091043657
:10EEC0008F93809103368F93809102368F9369E1FF
:10EED00076E38EEB95E30E94C784182F0F900F9076
:10EEE0000F900F900F9060E089EE94E30E94ED4A3E
:10EEF00080911436813061F48091B935811104C05C
:10EF00000E941E56812F38C00E944F56812F34C058
:10EF1000812F32C08BEC30C083E02EC084E82CC03F
:10EF200083E82AC0822D90E0FC01E154F109EA3126
:10EF3000F105B0F7E156FE4F0C9498DE1092B63F03
:10EF40006091BA357091BB358091BC359091BD35DB
:10EF50000E94874A80913D36882309F4F8CDF1CD8F
:10EF600085E60AC086E608C0D8018C91DBC8580146
:10EF70008D2D78017D2CA5C82796CDBFDEBFDF91F2
:10EF8000CF911F910F91FF90EF90DF90CF90BF90A6
:10EF9000AF909F908F907F906F905F904F903F9039
:10EFA0002F900895CF93DF93EC016CEA7EE30E94EB
:10EFB000B5618093B63F811102C095E09F83DF91D8
:10EFC000CF910895FC018789908D0C942D7083FF5B
:10EFD00006C0E0918B32F0918C3290E2958382FFF3
:10EFE00006C0E0918D32F0918E3290E2958381FFE0
:10EFF00006C0E0918F32F091903290E2958380FFCD
:10F0000006C0E0919132F091923280E285830895BA
:10F0100083FF06C0E0918B32F0918C3290E29683B0
:10F0200082FF06C0E0918D32F0918E3290E296839D
:10F0300081FF06C0E0918F32F091903290E296838A
:10F0400080FF06C0E0919132F091923280E2868397
:10F0500008958091883C811107C084E00E94E77781
:10F0600081E08093883C089584E00E9408781092A3
:10F07000883C0895CF92DF92EF92FF920F931F93F7
:10F08000CF93DF93C12C26E0D22EC0927B32D09258
:10F090007C3230EAE32E36E0F32EE0927D32F092BD
:10F0A0007E3200E816E000937F3210938032C0E693
:10F0B000D6E0C0938132D0938232C0928332D09214
:10F0C0008432C0938532D093863200938732109376
:10F0D0008832E0928932F0928A322DEC3CEC4CED91
:10F0E00050E40E9450D8C0928B32D0928C32E09281
:10F0F0008D32F0928E3218164CF4C0938F32D0932A
:10F100009032009391321093923208C000938F3264
:10F1100010939032C0939132D0939232DF91CF917D
:10F120001F910F91FF90EF90DF90CF9008950E9474
:10F13000F7D360E070E080E091E40E943A780C94AC
:10F1400016D481E08093913C089520E093E088ED0F
:10F1500008B618BE84BF909380002091820021FDE4
:10F16000FCCF08BEFFCF8091913C81110E94A57811
:10F1700083E008958091923C882341F0F89461E007
:10F1800089E790E00E94F9D382E0089583E0089532
:10F19000CF93DF93CDB7DEB7AD97CDBFDEBF21E212
:10F1A000E5EEF1E2DE01119601900D922A95E1F76C
:10F1B00022E02093CA01DE019296E8E0F0E024917B
:10F1C0002D933196EE30F105D1F72DE228A7E0E13D
:10F1D000F0E0E491EF7121E030E02C0F3D1F2E0FA5
:10F1E000311DF901208129A7E2E1F0E0E491EF71FE
:10F1F0009E012E0F311DF90121812AA7E4E1F0E0E3
:10F20000E491EF719E012E0F311DF90121812BA791
:10F210001CA61092CA0125E0FC012783BE016E5D89
:10F220007F4F0E94B5618093B63FAD96CDBFDEBFE4
:10F23000DF91CF91089581E08093923C80E0089522
:10F24000CF93DF93EC0120E030E040E051E46985AA
:10F250007A858B859C850E9450D818166CF0CE015B
:10F260000E94DE5E69857A858B859C850E943A784E
:10F270000E94F2BC80E001C08DE6DF91CF9108953D
:10F280006CE97BE30C947DC26EE77BE30C947DC25A
:10F290006FE57BE30C947DC261E47BE30C947DC25B
:10F2A0006DE27BE30C9428C2CF93DF9382EE96E469
:10F2B0009F938F93CEE6DCE589818F9388818F932E
:10F2C0000E944DE38CEA94E49F938F9389818F93FE
:10F2D00088818F930E944DE384E294E49F938F93FF
:10F2E00089818F9388818F930E944DE38AE593E40F
:10F2F0009F938F9389818F9388818F930E944DE391
:10F300000E94B4A88DB79EB740968DBF9EBF80E087
:10F31000DF91CF910895CF93DF9385E393E49F939B
:10F320008F93CEE6DCE589818F9388818F930E944D
:10F330004DE387EC91E49F938F9389818F9388812C
:10F340008F930E944DE38CE390E49F938F93898188
:10F350008F9388818F930E944DE384E294E49F937E
:10F360008F9389818F9388818F930E944DE38AE5E3
:10F3700093E49F938F9389818F9388818F930E94C9
:10F380004DE38DB79EB744968DBF9EBF80E0DF9161
:10F39000CF910895CF93DF938BE190E49F938F9368
:10F3A000CEE6DCE589818F9388818F930E944DE3BF
:10F3B0008DE99CE39F938F9389818F9388818F93AD
:10F3C0000E944DE38AE593E49F938F9389818F9305
:10F3D00088818F930E944DE38DB79EB70C968DBFA9
:10F3E0009EBF80E0DF91CF910895CF93DF9385E7B3
:10F3F0009CE39F938F93CEE6DCE589818F93888190
:10F400008F930E944DE384E09CE39F938F938981C7
:10F410008F9388818F930E944DE38AE593E49F93B5
:10F420008F9389818F9388818F930E944DE38DB74D
:10F430009EB70C968DBF9EBF80E0DF91CF9108955F
:10F44000CF93DF9381EE9BE39F938F93CEE6DCE532
:10F4500089818F9388818F930E944DE388EB9BE392
:10F460009F938F9389818F9388818F930E944DE31F
:10F470008AE593E49F938F9389818F9388818F93FB
:10F480000E944DE38DB79EB70C968DBF9EBF80E066
:10F49000DF91CF9108952F923F924F925F926F929A
:10F4A0007F928F929F92AF92BF92CF92DF92EF9214
:10F4B000FF920F931F93CF93DF93CDB7DEB76A9779
:10F4C000CDBFDEBF5C010E94F5602C011F86188A4B
:10F4D000198A1A8AF50101900020E9F73197EA1993
:10F4E000FB09E130F24008F002C2D5018C9188237B
:10F4F00059F17501BFEFEB1AFB0A850120E02111DC
:10F5000015C0883229F08132C8F08F37B9F001C0B8
:10F5100021E06801EFEFCE1ADE0A90E02A8F0E9408
:10F520004FE2D8018C9386012A8D08C021E08932F0
:10F5300009F420E0F80180830F5F1F4FD7018D9100
:10F540007D018111DCCF01C08501F801108210928C
:10F55000B63FFDE19F2EAAE36A2EA2E27A2E812C0D
:10F56000B6E02B2E03C09A9409F49CC18BE79CE271
:10F57000A2E2B0E08B879C87AD87BE876B8A7C8ACE
:10F580008D8A8DE79CE2A2E2B0E08F839887A987FD
:10F59000BA87E6E0F2E2DE011196822D01900D922B
:10F5A0008A95E1F7C2010E94FC5F8501075F1F4F4A
:10F5B00075019FEFA91AB90AD7016C9170E0CE01CD
:10F5C0000B960E94ACE2892B21F487010E5D1F4F40
:10F5D00004C0A016B10661F793C16501BFEFAB1A75
:10F5E000BB0AF601608170E0CE0143960E94ACE256
:10F5F000892B91F0D6011D928D0192012F5E3F4F14
:10F60000288F398F46E050E0B701C9010E94D7E248
:10F610003AE0C30ED11C04C0A016B106F1F670C1C9
:10F620005801D8013D908D01E32CF12CC7010E94B7
:10F6300033E2892B59F4B701CE0101960E94ACE266
:10F64000892B21F40C151D0559F75AC18501BEE619
:10F650003B1641F0E2E23E120CC0D50111968C91AE
:10F660008232A9F5F201178211861286138614865A
:10F67000A3C0B0E3EB1AF108EAE0EE16F10418F0CB
:10F68000FDE23F1217C0BE016A5E7F4FC5010E94B6
:10F69000B8DED20119966D937D938D939C931C9740
:10F6A0008E899F898A159B0509F42DC1E4E0179680
:10F6B000EC9382C0FBE73F124FC0E7E0D201179600
:10F6C000EC93FFEFAF1ABF0AE2E0FE2E95C02FEFDA
:10F6D000A21AB20AE5E0D2011796EC9362E270E05A
:10F6E000C5010E94ACE28E8B9F8B009709F408C184
:10F6F000DC011C92F50101900020E9F73197EA192D
:10F70000FB093397C8F0F80181818033A9F4828125
:10F71000883791F440E050E060E070E0C5010E945D
:10F7200029E0D20119966D937D938D939C931C973C
:10F7300083E017968C9308C0B501C2010E94B561A1
:10F740008093B63F811153C0AE88BF88BFEFAB1A1C
:10F75000BB0AAE8ABF8A30C0E4E73E120EC0E1E0C9
:10F76000D2011796EC9380E090E0A0E8BFE3F201AD
:10F7700081879287A387B4871FC0F6E63F120CC02B
:10F78000E1E0D2011796EC93179719961D921D92FE
:10F790001D921C921C9710C0BBE53B12B1C0F20138
:10F7A0002782B501C2010E94B5618093B63F8111E5
:10F7B0001EC077E6F72E7DC0BE01695F7F4FC50191
:10F7C0000E94F1E25C01009709F49AC0DC018C917F
:10F7D0008D3729F411968C91F50131965F018C32A9
:10F7E00009F48BC0FFEFAF1ABF0AF12C05C0F82E49
:10F7F00022E0281708F45DC08F858201035F1F4F48
:10F80000882341F043E050E0BE01615F7F4FC801B3
:10F810000E94D7E2688D798DC8010E94555FD201A0
:10F8200014968D939C9315978F3FBFEF9B07B9F16B
:10F830000E948C64882371F0888D998D0E943E5FB0
:10F84000882341F043E050E0688D798DCE010F961A
:10F850000E94D7E2F201428053804114510411F119
:10F86000F11081CE80911C37811108C085E197E3AA
:10F870000E94F15B8093B63FF82E1BC08091B93493
:10F88000823099F085E197E30E94C75B8093B63F91
:10F8900081110EC085E197E30E94445C0AC064E6D2
:10F8A000F62E07C050E7F52E04C04BECF42E01C035
:10F8B000F82E42E060E08F2D0E945C6281E00E94A1
:10F8C00013AB6A96CDBFDEBFDF91CF911F910F9131
:10F8D000FF90EF90DF90CF90BF90AF909F908F9070
:10F8E0007F906F905F904F903F902F9008958BE6A0
:10F8F0008093B63F3BE6F32EDCCF22E0F22E7CCFA6
:10F900009FE6F92ED6CF86E6F82ED3CF2F923F92E0
:10F910004F925F926F927F928F929F92AF92BF921F
:10F92000CF92DF92EF92FF920F931F93CF93DF93CB
:10F9300000D000D0CDB7DEB78C0169837A834B83CA
:10F940005C835A0128E0A21AB108A60EB71EDC019A
:10F9500016967C907B01BFEFEB1AFB0A8BE7FB014D
:10F96000808380E0912C95E0692E20E1422E22E2F6
:10F97000522E3CE0232E32E2332E4DE7842EED82D0
:10F98000FE82D80117969C919F3F09F429C18823D4
:10F9900039F02CE2ED81FE8120833196ED83FE83E8
:10F9A0008091603F811119C0C80141969F938F9348
:10F9B0003F922F923E813F938D818F930E9418E456
:10F9C000AD81BE81A80FB91FAD83BE830F900F908C
:10F9D0000F900F900F900F9018C0C80141969F9301
:10F9E0008F935F924F92BE81BF93ED81EF930E9400
:10F9F00018E42D813E81280F391F2D833E830F90FF
:10FA00000F900F900F900F900F90D80117968C9138
:10FA10001797843059F51996CD90DD90ED90FC90B4
:10FA20001C97A7019601C701B6010E9413DA811144
:10FA300017C0E894F7F82FEF3FEF4FE75FE7C701F4
:10FA4000B6010E9413DA811121C12FEF3FEF4FE77A
:10FA50005FE7C701B6010E944DD618160CF016C11B
:10FA6000F801118612861386148610C1811113C005
:10FA7000E6E1F2E2AD81BE81862D01900D928A957C
:10FA8000E1F72D813E812C5F3F4F2D833E83D801CE
:10FA900017968C9199C0823061F4F80184858F9318
:10FAA00083858F9382858F9381858F93ABE1B2E2BB
:10FAB00014C0833029F5D8011C968C911C978F9324
:10FAC0001B968C911B978F931A968C911A978F93F4
:10FAD00019968C918F93A1E2B2E2BF93AF93FE810E
:10FAE000FF932D812F930E9418E4AD81BE81A80F52
:10FAF000B11DAD83BE83F8018781CDBFDEBF64C079
:10FB0000853059F4D80158968C9158978F93579611
:10FB10008C918F93A9E2B2E20CC0863009F5D8012E
:10FB200058968C9158978F9357968C918F93AEE2FD
:10FB3000B2E2BF93AF93FE81FF932D812F930E947A
:10FB400018E4AD81BE81A80FB11DAD83BE83F8015D
:10FB500087810F900F900F900F900F900F9034C0EF
:10FB6000813091F52CEA35EC47E257E3D80119963C
:10FB70006D917D918D919C911C970E944DD687FF30
:10FB800012C0E3E3F2E2AD81BE8186E001900D9206
:10FB90008A95E1F7ED81FE813596ED83FE83D801EC
:10FBA00017968C9111C0E9E3F2E2AD81BE81862DFA
:10FBB00001900D928A95E1F7ED81FE813496ED83F7
:10FBC000FE83D80117968C91873049F42BE7ED819D
:10FBD000FE8120833196ED83FE8380E001C081E0C9
:10FBE000AD81BE81AA15BB0518F08FEF9FEF65C0F0
:10FBF000F801028113810115110549F0D80116960B
:10FC00009C912FEF290D99153CF0992EBACEED80DD
:10FC1000FE807914B4F020C0ED81FE81D801CF01BF
:10FC20000196808216969C9016973FEF320F92169F
:10FC30001CF4232FFC01F3CF8D839E838D0181E083
:10FC4000A0CEF7012DE7CF01019620839A94791475
:10FC500014F4FC01F8CF7C018DE79AE0A0E0F701F5
:10FC600080839183A283F2E0EF0EF11C89819A8157
:10FC70002B813C81820F931F8E159F0508F4B5CF11
:10FC8000C701A981BA818A1B9B0B17C0C8010E94BA
:10FC90009C64F801418552856385748520858D813A
:10FCA0009E810E94C1C42D813E81280F311D2D836C
:10FCB0003E83D80117968C9187CF2696CDBFDEBFA5
:10FCC000DF91CF911F910F91FF90EF90DF90CF9038
:10FCD000BF90AF909F908F907F906F905F904F906C
:10FCE0003F902F90089540E052E06CEA7CE30E9440
:10FCF000867C60916E5C70916F5C8CEA9CE30C94E6
:10FD00009CE3BF92CF92DF92EF92FF920F931F93EB
:10FD1000CF93DF93CDB7DEB76297CDBFDEBFB82EEE
:10FD200080915E3F882309F404C18FE6B81212C0A7
:10FD30000E94F5606CEA7EE38091A83C9091A93C1A
:10FD40000E94A1C4BC018CE091E20E94136205E113
:10FD500017E339C08091B93405E117E3882399F19D
:10FD6000FF24FA94C8010E94BC5F882361F18230AD
:10FD700029F48091653F811120C01DC0843029F491
:10FD80008091623F811119C016C08530B1F4809115
:10FD9000643F882381F0F80181859285A385B4852D
:10FDA000BC01CD019F772CEA35EC47E257E30E9476
:10FDB0004DD687FF02C0F801F782F8010281138156
:10FDC0000115110579F66091A43C7091A53C8091D4
:10FDD000A63C9091A73C0E94EDD66B017C012CEAD9
:10FDE00035EC47E257E30E9450D818165CF14EC03C
:10FDF000F801028113810115110521F581E70E94A7
:10FE00003CA86091A43C7091A53C8091A63C909147
:10FE1000A73C0E94EDD669B97AB98BB99CB984E741
:10FE200099E6A4E6B0E081BB92BBA3BBB4BB83E080
:10FE300087B940E052E06CEA7CE38CEF96E30E94E5
:10FE4000867C77C0F80187818F3F91F6C186D28684
:10FE5000E386F48684E799E6A4E6B0E0818B928B92
:10FE6000A38BB48B82E08783028113810FC0F801DA
:10FE7000028113810115110549F440E052E06CEA5A
:10FE80007CE38CEF96E30E94867C53C0F801878167
:10FE90008F3F69F78091733281111AC08091AB3C1A
:10FEA0008F938091AA3C8F931F92BF928EE392E230
:10FEB0009F938F93CE0101967C01FF928F930E94B6
:10FEC00018E41092AA3C1092AB3CCDBFDEBF13C029
:10FED0000E94F1C91F928F931F92BF9286E492E213
:10FEE0009F938F93CE0101967C01FF928F930E9486
:10FEF00018E4CDBFDEBFB701C8010E94B561F801AB
:10FF0000168286E0878386E690E0818B928B128250
:10FF1000138240E052E06CEA7CE38CEF96E30E94AF
:10FF2000867C60916E5C70916F5C8CEA9CE30E94B1
:10FF30009CE36296CDBFDEBFDF91CF911F910F9101
:10FF4000FF90EF90DF90CF90BF900895613019F04F
:10FF5000623029F0089585E197E30C94737E0C9448
:10FF6000817ECF92DF92EF92FF92FC01C184D28416
:10FF7000E384F48420E030E040EA50E4C701B601B5
:10FF80000E9450D818160CF453C0C701B6010E9445
:10FF9000C1D660935E3F1092613F1092623F109213
:10FFA000633F1092643F1092653F20E030E040E8EC
:10FFB0005FE3C701B6010E9450D887FD03C081E00E
:10FFC0008093613F20E030E040E050E4C701B6019B
:10FFD0000E9450D887FD03C081E08093623F20E0FB
:10FFE00030E040E450E4C701B6010E9450D887FDDC
:10FFF00003C081E08093633F20E030E040E850E4BC
:020000021000EC
:10000000C701B6010E9450D887FD03C081E08093EC
:10001000643F20E030E040EA50E4C701B6010E94AE
:1000200050D887FD07C081E08093653F80E003C022
:100030008EE601C080E0FF90EF90DF90CF900895B2
:1000400064E877E40C943EC26DE277E40C943EC21F
:1000500069EF76E40C943EC2BF92CF92DF92EF92AA
:10006000FF920F931F93CF93DF93CDB7DEB76897BF
:10007000CDBFDEBF6B0128E1FC01DE0111960190CE
:100080000D922A95E1F78AE7E82E83E3F82E8E0198
:100090000F5F1F4FB12CF7018081823029F4F801E6
:1000A00010821182128213828091F05A8B1114C037
:1000B0002091035B3091045B4091055B5091065B9E
:1000C000F80160817181828193810E94F2D8F601EA
:1000D000608371838283938380910F5B8B1114C043
:1000E0002091225B3091235B4091245B5091255BF2
:1000F000F80160817181828193810E94F2D8F601BA
:10010000648375838683978380912E5B8B1114C0E3
:100110002091415B3091425B4091435B5091445B45
:10012000F80160817181828193810E94F2D8F60189
:10013000608771878287938780914D5B8B1114C094
:100140002091605B3091615B4091625B5091635B99
:10015000F80160817181828193810E94F2D8F60159
:100160006487758786879787B394F5E3EF0EF11C54
:100170000C5F1F4F86E0B8128ECF6896CDBFDEBFF2
:10018000DF91CF911F910F91FF90EF90DF90CF9073
:10019000BF900895F8940E9497780E9421810E9450
:1001A00016D40E94B4C60E94ADB30E94E86F0E94AC
:1001B000F2BC0E9409A640E060E080E00E949A65DF
:1001C0000E9432610E940F810E9413830E947F4F20
:1001D0000E940ED48091A20084608093A20080913E
:1001E000A20082608093A2008091A200816080932F
:1001F000A20078940E94B4A80E94FFBD0E940166EC
:10020000FDCFE82FF0E0EE0FFF1FE055F84B6591B2
:1002100074914FE450E086E69FE30C947EE2809177
:10022000853C823041F440E060E081E00E949A65C4
:1002300080E00E9429670C94EACA682F81E00C9440
:1002400091C71092B73F1092B83F1092B93F1092E9
:10025000BA3F0895CF93DF93EC018C819D81880F85
:10026000991F880F991F2091B93F3091BA3F820F93
:10027000931F8093BB3F9093BC3F44E050E061EC00
:100280007FE30E940ED34091C13F5091C23F6091E5
:10029000C33F7091C43F49875A876B877C8780E052
:1002A000DF91CF9108958F929F92AF92BF92CF929C
:1002B000DF92EF92FF92CF93DF93EC018091BA34FB
:1002C000882369F089E0DF91CF91FF90EF90DF9074
:1002D000CF90BF90AF909F908F900C943CA8898551
:1002E0009A85AB85BC858093BD3F9093BE3FA0931C
:1002F000BF3FB093C03FCE010E942A818093B63F9A
:1003000081116EC0C984DA84EB84FC84A701960154
:10031000C701B6010E9413DA81112FC046015701AF
:10032000E894B7F82FEF3FEF4FE75FE7C501B4015F
:100330000E9413DA81110AC02FEF3FEF4FE75FE70A
:10034000C501B4010E944DD61816BCF08090BD3F87
:100350009090BE3FA090BF3FB090C03FA5019401D8
:10036000C701B6010E94A4D49F772CEA35EC47E27E
:1003700057E30E9450D8181674F58091BD3F9091B4
:10038000BE3FA091BF3FB091C03F8093C13F9093CB
:10039000C23FA093C33FB093C43F8C819D81880F1F
:1003A000991F880F991F2091B93F3091BA3F820F52
:1003B000931F8093BB3F9093BC3F44E050E061ECBF
:1003C0007FE30E949FD38090BD3F9090BE3FA0905E
:1003D000BF3FB090C03F89869A86AB86BC8680E0DE
:1003E000DF91CF91FF90EF90DF90CF90BF90AF90D3
:1003F0009F908F9008950E9408B980E008958091A1
:10040000C53F9091C63F8F3E924111F08EE5089511
:100410008091EB3F9091EC3F8F3E9241B9F78091F4
:10042000ED3F9091EE3F8F3E924181F7809176575C
:10043000909177578F3E924149F7809178579091EC
:1004400079578F3E924111F780910B5990910C5939
:100450008F3E9241D9F680E0089594E0899FF001A3
:100460001124EB53F04C42835383648375830895C6
:1004700094E0899FF0011124E858F84A45AB56AB47
:1004800067AB70AF08955F926F927F928F929F9249
:10049000AF92BF92CF92DF92EF92FF920F931F9392
:1004A000CF93DF93CDB7DEB76097CDBFDEBFBE0180
:1004B0006F5F7F4F8DEA97E50E942C80CE010196F9
:1004C0004C0185E2A82E88E5B82E95E3C92E98E563
:1004D000D92E25E4E22E28E5F22E05E618E537E8C8
:1004E000632E3BE5732E512CF401419151916191A2
:1004F00071914F01F50141935193619371935F01A4
:10050000F60141935193619371936F01F701419308
:100510005193619371937F01852D0E940A70F801B8
:1005200011921192119211928F01F3011082118296
:10053000128213825394F8E16F0E711C84E05812FA
:10054000D3CF6096CDBFDEBFDF91CF911F910F91CA
:10055000FF90EF90DF90CF90BF90AF909F908F90E3
:100560007F906F905F9008958091EF3F08951F9363
:10057000CF93DF938BE897E1EDEEFFE3DF019C0182
:100580001D9221503040E1F78FEE92E18093ED3FD4
:100590009093EE3F8093765790937757C6EFDFE3C3
:1005A000C093F03FD093F13FC093F23FD093F33F1D
:1005B000C093F43FD093F53F81E090E06AEB76E59D
:1005C00020E030E01CEB129FA001139F500D11247E
:1005D000FA01E351F04CD90111961A9F90011B9F2B
:1005E000300D11242A50304C23873487618772875D
:1005F000BA016A50704C9C0101968032910519F73E
:100600008CEB829FF001839FF00D1124E351F04C9D
:10061000C387D4876187728780E28093EF3FDF9141
:10062000CF911F910895CF93DF93E8E7F7E585E930
:1006300091E0DF01EC011D922197E9F7A5ECBFE302
:1006400088E2ED0119928A95E9F78FEE92E18D9398
:100650009C938093EB3F9093EC3F808391838093B6
:100660000B5990930C59DF91CF910C94B7820E9453
:10067000308D0E94B78280E00C943C4AE091F03FBC
:10068000F091F13F848581111BC0228133818081EB
:1006900091814CEBDF011D924A95E9F72283338368
:1006A0008083918381E084878091EF3F81508093A4
:1006B000EF3F828193818093F03F9093F13F05C09B
:1006C0008CE10E943CA8E0E0F0E0CF010895A2EFA9
:1006D000BFE3ED91FC911197858781E0878782E0E8
:1006E0008487828193818D939C9381E00E9464AC86
:1006F0000C944EB6EF92FF920F931F93CF93DF931C
:1007000000D01F92CDB7DEB78C014B835C83698329
:100710007A830E943E83FC014B815C8169817A81EE
:10072000009761F48EE02496CDBFDEBFDF91CF91BC
:100730001F910F91FF90EF900C947B4E83E0858783
:100740008BEF91E884839583068317838B017A016D
:1007500026E0D8014D915D916D917D918D01CF0184
:1007600085599F4FDC014D935D936D937C93139757
:10077000D7014D915D916D917D917D01418B528BA2
:10078000638B748B215034962111E3CF83E0249640
:10079000CDBFDEBFDF91CF911F910F91FF90EF9002
:1007A0000C946783CF92DF92EF92FF926B017C01F2
:1007B0000E943E83009739F48EE0FF90EF90DF9027
:1007C000CF900C947B4E25E534E8FC0124833583DF
:1007D000E556FF4FC082D182E282F38221E0FC0124
:1007E000278782E00E94678380E0FF90EF90DF9090
:1007F000CF9008958091F43F9091F53FFC012485BE
:100800003EEF320F323018F424E02487089524306C
:1008100011F080E090E00895E091F43FF091F53F11
:1008200022813381808191814CEBDF011D924A95B9
:10083000E9F72283338380839183E091F43FF09141
:10084000F53F0280F381E02DE093F43FF093F53F14
:100850008485823011F483E084878091EF3F8F5F3D
:100860008093EF3F8FEF0E9464AC81E04091F03FB6
:100870005091F13F2091F43F3091F53F42175307DB
:1008800009F080E00895BC016F5E7F4FDC01169691
:10089000ED91FC91179785599F4F19950E940C84F3
:1008A00081110E94EB5580E0089585569F4F20E00E
:1008B00034E244E759E4FC016081718182819381D3
:1008C0000E94F2D80E94C1D60E94EDD60E9412B9B1
:1008D0000E940C8481110E94EB5580E00895809164
:1008E000F43F9091F53FFC0124853EEF320F32300A
:1008F00018F424E024870895243011F080E090E07B
:100900000895CF93DF93C091F43FD091F53F8C854C
:100910009EEF980F923018F484E08C8705C08430E5
:1009200019F080E090E010C02097D9F3DE01129614
:10093000ED91FC9113978785882329F0EC17FD072B
:1009400011F0DF01F4CFCD01DF91CF910895CF9366
:10095000DF93EC012A813B81888199814CEBFB017B
:10096000DE0101900D924A95E1F72A833B8388834B
:100970009983DF91CF9108958FEE92E180930D5985
:1009800090930E598093CA599093CB5908952F9202
:100990003F924F925F926F927F928F929F92AF920F
:1009A000BF92CF92DF92EF92FF920F931F93CF935C
:1009B000DF93CDB7DEB76A97CDBFDEBF4C011B0119
:1009C00029013A01E986FA860B871C871A2D0B2D1F
:1009D000E8A8B9A8AAA82BA9298380913235882331
:1009E00099F08091263590912735A0912835B091C6
:1009F0002935BC01CD019F772CEA35EC47E257E35E
:100A00000E944DD687FD11C780915D3690915E366C
:100A1000A0915F36B0916036BC01CD019F7731E087
:100A20003D832CEA35EC47E257E30E9450D8181674
:100A300014F01D8210C02DEC3CEC4CEC5DE3609199
:100A400002367091033680910436909105360E94EB
:100A50004DD687FDECC6F10180819181A281B381E1
:100A6000BC01CD019F77F1E0FD872CEA35EC47E230
:100A700057E30E9450D818160CF01D86F1018481AE
:100A80009581A681B781BC01CD019F77F1E0F98BFB
:100A90002CEA35EC47E257E30E9450D818160CF0C8
:100AA000198AF10180859185A285B38520916136EF
:100AB0003091623640916336509164362E8B3F8B75
:100AC000488F598F20916536309166364091673650
:100AD000509168362A8B3B8B4C8B5D8B40916936ED
:100AE00050916A3660916B3670916C36F090333568
:100AF000F11021C01092555981E08093565982E03F
:100B0000809357593D81332341F04D85411195C65E
:100B10005989511192C68CE9C1C6CB01BA019F77A0
:100B20002CEA35EC47E257E30E9450D818160CF037
:100B300089C68BE9B3C6BC01CD019F77A1E0AA8F1E
:100B40002CEA35EC47E257E30E9450D818160CF017
:100B50001A8EB1E0FB1216C01092555982E08093B4
:100B60005659F0925759ED81EE2339F0FD85F11178
:100B700064C62A8D222379F260C66A897B898C89B2
:100B80009D89CDCF32E0F31217C081E08093555993
:100B9000F0925659109257594D81442341F059898A
:100BA00051114BC68A8D882309F4B5CF46C66E898C
:100BB0007F89888D998DB3CFB101C4010E948B4C80
:100BC0009D81992309F451C02091EE343091EF3486
:100BD0004091F0345091F134609143357091443537
:100BE00080914535909146350E94A4D49F772CEA98
:100BF00035EC47E257E30E944DD687FF36C020917F
:100C0000F2343091F3344091F4345091F5346091E2
:100C10004735709148358091493590914A350E9409
:100C2000A4D49F772CEA35EC47E257E30E944DD6D7
:100C300087FF1BC02091F6343091F7344091F8348F
:100C40005091F93460914B3570914C3580914D3510
:100C500090914E350E94A4D49F772CEA35EC47E260
:100C600057E30E944DD687FDE4C58CA98093ED34EF
:100C700089EE94E30E94934A86E5E9EEF4E3A4E763
:100C8000B9E501900D928A95E1F788E1E3E4F5E397
:100C9000A0E1B9E501900D928A95E1F78091343594
:100CA0008111D5C523E333E34BEC51E46E2D7B2D4D
:100CB0008A2D99810E94F2D84B015C0160934059C2
:100CC00070934159809342599093435923E333E3FE
:100CD0004BEC51E4C301B2010E94F2D86093285951
:100CE0007093295980932A5990932B5923E333E326
:100CF0004BEC51E469857A858B859C850E94F2D8FE
:100D000060932C5970932D5980932E5990932F599D
:100D100023E333E34BEC51E4612F702FC6010E94B3
:100D2000F2D8162F072F412F502FBC014093305976
:100D30005093315960933259709333598091FE35F5
:100D40009091FF35A0910036B0910136BC01CD01E4
:100D50009F770E942AD70E94C1D660935159709301
:100D600052598093535990935459A0915559A98B36
:100D7000B0915659BA8BEB2FF0E0ED83FE837F01E3
:100D8000EE0CFF1CEE0CFF1CF101EE0DFF1D80812F
:100D90009181A281B381BC01CD019F772CEA35EC12
:100DA00047E257E30E944DD6D82EDD1CDD24DD1C22
:100DB0003989232F30E029833A838901000F111FDD
:100DC000000F111FF101E00FF11F80819181A281BD
:100DD000B381BC01CD019F772CEA35EC47E257E3A4
:100DE0000E944DD6881F8827881F8D2180935059D7
:100DF0002CEA35EC47E257E3C501B4019F770E9426
:100E000050D818160CF0F9C0F801E251FB4CD8018B
:100E1000AD5BBA4C2D913D914D915C91608171819A
:100E2000828193810E94A4D46B017C01ED81FE81BB
:100E3000EE0FFF1FEE0FFF1FE251FB4CAD81BE8195
:100E4000AA0FBB1FAA0FBB1FAD5BBA4C2D913D91E2
:100E50004D915C9160817181828193810E94A4D4C3
:100E600069877A878B879C87A5019401C501B401A6
:100E70000E94F2D820E030E040E850E40E94F2D82E
:100E80006D877E878F87988BA7019601C701B60172
:100E90000E94F2D82B013C0129853A854B855C855F
:100EA000CA01B9010E94F2D89B01AC01C301B20191
:100EB0000E94A5D49B01AC016D857E858F859889A4
:100EC0000E94A4D42B013C0120E030E0A9010E9443
:100ED00050D81816C4F4C301B2010E94CBD92B011B
:100EE0003C0129853A854B855C85C701B6010E9486
:100EF0005DD89B01AC01C301B20190580E9454D649
:100F00002B013C0103C0412C512C32018091ED3466
:100F1000833021F477FA709477F8709420E030E011
:100F2000A901C501B4010E944DD687FF04C077FA1C
:100F3000709477F8709409811A81000F111F000FC7
:100F4000111FA801435F564A5A01A3019201698506
:100F50007A858B859C850E94F2D89B01AC01C701E4
:100F6000B6010E94A4D420E030E040E05FE30E949C
:100F7000F2D8D5015B966D937D938D939C935E978C
:100F8000AD80BE80AA0CBB1CAA0CBB1CF501E35FA4
:100F9000F64A4F01A3019201C701B6010E94F2D89F
:100FA0009B01AC0169857A858B859C850E94A5D4BF
:100FB00020E030E040E05FE30E94F2D8D4015B968D
:100FC0006D937D938D939C935E97E0915759F0E0DC
:100FD000EE0FFF1FEE0FFF1FE35FF64A138E148E16
:100FE000158E168EB0914059B987E0914159ED8721
:100FF000209042593090435925C05701F701E35FD3
:10100000F64A838D948DA58DB68D9C01AD01505807
:10101000F801E35FF64A838D948DA58DB68DBC01F2
:10102000CD0190580E945DD89B01AB01BC0140935B
:1010300040595093415960934259709343592987BD
:101040003D871C01D801A35FB64A5B96CD90DD9029
:10105000ED90FC905E97E981FA81EE0FFF1FEE0F95
:10106000FF1FE758F64A13962D913D914D915C91E3
:10107000169760817181828193810E94A4D4A70117
:1010800096010E94A4D469837A838B839C83D501C3
:10109000A35FB64A5B964D905D906D907C905E9795
:1010A000ED81FE81EE0FFF1FEE0FFF1FE758F64A9E
:1010B00013962D913D914D915C91169760817181B0
:1010C000828193810E94A4D4A30192010E94A4D49E
:1010D0006D837E838F8398879B01AC0169817A81C0
:1010E0008B819C810E945DD829853D85A1010E944C
:1010F000A4D44B015C01E894B7F820E030E040E86C
:101100005FE3C501B4010E9450D818160CF4C3C3A4
:101110002AE037ED43EA5BE3C501B4010E9450D8F1
:10112000181694F42FE632E143E85AE369857D8589
:10113000C1010E94F2D89B01AC01C501B4010E941B
:1011400050D818160CF4A7C3A30192015058C70138
:10115000B60190580E9418D54B015C016093385934
:101160007093395980933A5990933B598091333514
:10117000813039F4412C512C30E8632E3FEB732E33
:1011800006C0412C512C20E8622E2FE3722E809154
:1011900050598823D1F160915159709152598091E1
:1011A0005359909154590E94EDD66B017C012CEA61
:1011B00035EC47E257E30E944DD687FD10C01091F1
:1011C000ED342BED3FE049EC50E4C701B6010E943D
:1011D000F2D89B01AC01C12CD12C7601B9C081E0C1
:1011E00090E0A0E0B0E08093515990935259A093C1
:1011F0005359B09354591091ED342BED3FE049EC25
:1012000050E4C12CD12C7601A3C02D813E814F81A9
:10121000588569817A818B819C810E9418D5698368
:101220007A838B839C8360933C5970933D59809360
:101230003E5990933F59A50194010E94A4D46B019B
:101240007C019F772CEA35EC47E257E30E944DD6AC
:1012500087FF18C01091ED34609151597091525927
:1012600080915359909154590E94EDD62BED3FE057
:1012700049EC50E40E94F2D89B01AC01C12CD12C66
:10128000760166C029813A814B815C81C501B40138
:101290000E9450D81816F4F42BED3FE049EC50E4CE
:1012A000C301B2010E94F2D89B01AC0169817A812D
:1012B0008B819C810E94A5D460933C5970933D59C9
:1012C00080933E5990933F59A50194010E94A4D464
:1012D0006B017C011091ED34133099F060915159FC
:1012E0007091525980915359909154590E94EDD662
:1012F0002BED3FE049EC50E40E94F2D89B01AC0199
:1013000027C02BED3FE049EC50E4C301B2010E943D
:10131000F2D89B01AC01C701B6010E94A4D47B01A5
:101320008C0160915159709152598091535990910B
:1013300054590E94EDD62BED3FE049EC50E40E9459
:10134000F2D89B01AC01C701D8016C017D010BC033
:10135000123049F4C301B2010E94F2D8A7019601EC
:101360000E94A5D40AC0C301B2010E94F2D89B0119
:10137000AC01C701B6010E94A4D47B01AB01BC0142
:101380004093445950934559609346597093475937
:101390008C0150905759A52DB0E0FD01EE0FFF1FB5
:1013A000EE0FFF1FE758F64AAA0FBB1FAA0FBB1F7D
:1013B000A35FB64A13962D913D914D915C9116977E
:1013C00060817181828193810E94A4D44B015C0170
:1013D000609348597093495980934A5990934B5957
:1013E0009701A80169857D85C1010E94F2D86B0132
:1013F0007C0160934C5970934D5980934E59909352
:101400004F59A50194010E945DD869837A838B832B
:101410009C836093345970933559809336599093D7
:10142000375980913235811117C0F0912635FD83EF
:1014300040902735209128352E8B309129353A8FD1
:1014400010922635109227351092283510922935A2
:1014500081E08093323512C02091263530912735B6
:10146000409128355091293569817A818B819C8101
:101470000E9454D66D83472E8E8B9A8F598945E3EF
:10148000549FF0011124E558FC4C208131814281A8
:101490005381C701B6010E9454D6662E072F182F1C
:1014A000792E2D81342D4E895A8D0E944DD687FF7D
:1014B00004C06D80042D1E897A8C9A8985E3989FDB
:1014C000F0011124E558FC4C208131814281538187
:1014D000C701B6010E9454D66B017C019B01AC018F
:1014E000662D702F812F972D0E9450D8181624F04A
:1014F0006C2C0D2D1E2D7F2C862D902FA12FB72DFE
:101500008093585990935959A0935A59B0935B5965
:1015100020E030E0A901C501B4019F770E9450D8B6
:10152000181684F5A5E35A9EF0011124E558FC4CE9
:101530002081318142815381C501B4010E9454D67A
:101540004B015C01E894B7F8A5019401662D702F5A
:10155000812F972D0E9450D8181614F4A72C04C080
:10156000682C092D1A2DAB2C862D902FA12FBA2D6A
:101570008093585990935959A0935A59B0935B59F5
:10158000B62C02C0B62CA72CC090BC32D090BD3275
:10159000E090BE32F090BF3220E030E040E850E40E
:1015A000C701B6010E94F2D82B013C0129853D8577
:1015B000A10169857D85C1010E94A5D4A70196017D
:1015C0000E94A4D49B01AC01C301B2010E94F2D8D5
:1015D0000E94CBD92B013C0120EC31EE44E65CE4C7
:1015E0006B2D702F812F9A2D0E94F2D820E030E4CD
:1015F0004CE156E40E9454D66B017C012091C53227
:101600003091C6324091C7325091C83269817A8197
:101610008B819C810E9454D64B015C01A3019201F5
:1016200069817A818B819C810E9454D687017601E1
:10163000A50194010E94A9C30E942AD77B018C01B5
:1016400020E030E040E85FE30E9450D818163CF4F8
:10165000B701C8010E94BCD64B015C0108C0812CB7
:10166000912C54018394E12CF12C00E81FE3C70175
:10167000D80180935C5990935D59A0935E59B093C3
:101680005F599701A80160915859709159598091FB
:101690005A5990915B590E9454D66093A9597093FE
:1016A000AA598093AB599093AC598092605990920B
:1016B0006159A0926259B09263599701A801609153
:1016C00044597091455980914659909147590E94CB
:1016D00054D660936459709365598093665990937A
:1016E00067599701A80160914859709149598091B3
:1016F0004A5990914B590E9454D6609368597093FF
:10170000695980936A5990936B5980903859909099
:101710003959A0903A59B0903B59C501B4010E9483
:10172000C1D9C0904059D0904159E0904259F090B1
:1017300043590091555910E0000F111F000F111F60
:10174000035F164AA70196010E94F2D89B01AC01E3
:10175000F80163817481858196810E94A4D460938D
:101760006C5970936D5980936E5990936F59C50160
:10177000B4010E9451D69B01AC010091565910E072
:10178000000F111F000F111F035F164AC701B6019A
:101790000E94F2D89B01AC01D80113966D917D9106
:1017A0008D919C9116970E94A4D460937059709368
:1017B00071598093725990937359A0915759B0E021
:1017C000FD01EE0FFF1FEE0FFF1FE758F64AAA0FAD
:1017D000BB1FAA0FBB1FA35FB64A13968D919D91A5
:1017E0000D90BC91A02D80839183A283B38310922E
:1017F000B63F8091345990913559A0913659B091A6
:101800003759BC01CD019F772CEA35EC47E257E30D
:101810000E944DD687FD0FC00E94DE5582E0809366
:101820000F590E94EE4B80E039C08EE837C08EE938
:1018300035C08FE933C089EC31C0B101C4010E94C9
:101840008B4CC2C9B101C4010E948B4C0ECA8E2DB3
:101850009B2DAA2DB9818093405990934159A09313
:101860004259B09343594092285950922959609255
:101870002A5970922B5929853A854B855C8520938E
:101880002C5930932D5940932E5950932F594C0178
:101890005D01C60148CA8BE98093B63F6A96CDBF09
:1018A000DEBFDF91CF911F910F91FF90EF90DF90FE
:1018B000CF90BF90AF909F908F907F906F905F90F0
:1018C0004F903F902F9008958F929F92AF92BF922A
:1018D000CF92DF92EF92FF92CF93DF9380910F59D7
:1018E000882309F4B1C00E94B482843010F482E0ED
:1018F000ACC020916459309165594091665950911E
:101900006759609138597091395980913A5990913D
:101910003B590E94A5D46B017C01609338597093A8
:10192000395980933A5990933B590E94C1D980907C
:10193000405990904159A0904259B0904359C0915C
:101940005559D0E0CC0FDD1FCC0FDD1FC758D64A4C
:10195000A50194010E94F2D89B01AC0160916C59E1
:1019600070916D5980916E5990916F590E94A5D4D4
:10197000688379838A839B83C701B6010E9451D60D
:101980009B01AC01C0915659D0E0CC0FDD1FCC0FAC
:10199000DD1FC758D64AC501B4010E94F2D89B0189
:1019A000AC01609170597091715980917259909108
:1019B00073590E94A5D4688379838A839B83C091DD
:1019C0005759D0E0CC0FDD1FCC0FDD1FC758D64ACA
:1019D000209168593091695940916A5950916B59D9
:1019E000688179818A819B810E94A5D468837983EB
:1019F0008A839B8384E799E50E94469788E1E9E71B
:101A0000F9E5A0E1B9E501900D928A95E1F78091A1
:101A1000605990916159A0916259B09163590197B1
:101A2000A109B1098093605990936159A0936259BB
:101A3000B0936359181619061A061B060CF457CFF3
:101A400010920F5980E001C083E0DF91CF91FF90A9
:101A5000EF90DF90CF90BF90AF909F908F900895C0
:101A600010920F5908954F925F926F927F928F92CA
:101A70009F92AF92BF92CF92DF92EF92FF92CF935D
:101A8000DF93CDB7DEB76497CDBFDEBF69837A83BE
:101A90008B839C8369017A0120E030E040E751E4C8
:101AA0000E94F2D84B015C0120E030E040E751E4B5
:101AB000C701B6010E94F2D89B01AC01C501B40177
:101AC0000E94A4D46D877E878F87988B20E030E0BA
:101AD00040E251EC69817A818B819C810E94F2D82D
:101AE0004B015C0120E030E040E251E4C701B60167
:101AF0000E94F2D89B01AC01C501B4010E94A5D49B
:101B0000698B7A8B8B8B9C8B20918D5830918E5862
:101B100040918F585091905860E070E080E89FE3CA
:101B20000E9454D64B015C0120E030E040EC50ECC8
:101B300069817A818B819C810E94F2D82B013C01C2
:101B400020E030E040EC50E4C701B6010E94F2D83A
:101B50009B01AC01C301B2010E94A5D4A50194016F
:101B60000E94F2D8A50194010E94F2D8A501940127
:101B70000E94F2D8A50194010E94F2D8A501940117
:101B80000E94F2D86B017C01A50194016D857E85D0
:101B90008F8598890E94F2D8A50194010E94F2D8FD
:101BA000A50194010E94F2D8A50194010E94F2D8E7
:101BB0006D837E838F839887A501940169897A89D3
:101BC0008B899C890E94F2D8A50194010E94F2D8C9
:101BD000A50194010E94F2D869877A878B879C8738
:101BE00020E030E042EF50E4C701B6010E94F2D895
:101BF0002B013C0120E030E040EA50E46D817E8121
:101C00008F8198850E94F2D89B01AC01C301B2017B
